:020000040800F2
:10000000008000208D700008F97C00081D26000883
:10001000FB7C0008FD7C0008FF7C0008000000005D
:10002000000000000000000000000000C1CA00083D
:10003000017D00080000000051CB000895CB0008AE
:10004000037D0008057D0008077D0008097D000884
:100050000B7D00080D7D00088D7C0008937C000856
:10006000997C00089F7C0008A57C00080F7D000893
:10007000117D0008137D0008157D0008177D00081C
:10008000197D00081B7D00081D7D00081F7D0008EC
:10009000217D0008237D0008257D0008AB7C000839
:1000A000277D0008297D00082B7D00082D7D000894
:1000B0002F7D0008317D0008337D0008357D000864
:1000C000377D0008397D00083B7D00083D7D000834
:1000D0003F7D0008D5840008B5860008417D0008F2
:1000E000CF7C0008797D0008437D0008457D00082D
:1000F000477D000800000000000000000000000034
:1001000000000000000000005FF808F110B5054C89
:10011000237833B9044B13B10448AFF300800123B3
:10012000237010BDD805002000000000A0F10108D8
:1001300008B5034B1BB103490348AFF3008008BD6A
:1001400000000000DC050020A0F1010810B5044605
:10015000C06910B1012106F097FF206910B101219B
:1001600006F092FF204610BD30B585B003F054FF75
:10017000002304468DF80F3003F0FEFA204606F007
:100180002DF82149204606F087FD10B901238DF88E
:100190000F30002302221D49CDE9003220461C4BBE
:1001A0000DF10F0203F0BAFD0A233221194DCDE9FA
:1001B00000310DF10F02184B1849204603F0AEFD37
:1001C0002B1F0DF10F0216492046009503F0E6FDA6
:1001D000A5F1200300930DF10F02A5F124031149AD
:1001E000204603F0DBFD1049204603F05BFD9DF83F
:1001F0000F30287733B10D480AF000FB69210C4815
:1002000002F07AF905B030BD0400002010A9010801
:100210005200002038000020530000201EA90108D1
:100220002DA9010838A9010843A9010850A901080E
:100230007EBA0108F8B50025C0E901120570C0E9D1
:100240000335C0E90555C0E90755456206990446DE
:10025000164600F11C0702F0F5FD38B93146074893
:100260000AF0CCFA2021064802F046F9069A3946EF
:10027000204602F0AFFD2046F8BD00BF63A901088B
:100280007EBA0108F8B50025C0E901120570C0E981
:100290000335C0E90555C0E907554562069904468E
:1002A000164600F11C0702F0E9FC38B93146074850
:1002B0000AF0A4FA2021064802F01EF9069A3946EF
:1002C000204602F0C5FC2046F8BD00BF63A9010826
:1002D0007EBA010870B58CB003F09EFE0446384D1E
:1002E00000F0CCFE214601F029FC204606F026FD58
:1002F000344B354A0095032102A8FFF79BFF02A962
:10030000204603F02FFF02A8FFF720FF00950025ED
:100310002E4B2F4A032102A8FFF78CFF02A920468B
:1003200003F020FF02A8FFF711FF2A4B2A4A0221FF
:10033000009502A8FFF7A6FF02A9204603F012FFCE
:1003400002A8FFF703FF3223244A00930221244B23
:1003500002A8FFF797FF02A9204603F003FF02A8B7
:10036000FFF7F4FE01211F4E1F4B02A88DF8085025
:1003700003910496CDE90535CDE90755CDE9095539
:100380000B9502F07BFB38B9314618480AF036FA73
:100390002021174802F0B0F8012209A902A802F0B2
:1003A0005BFB02A9204603F0DDFE02A8FFF7CEFEAC
:1003B00000F064FE0122214601F0C8FC0CB070BDC3
:1003C00026A80108F0A7010838A9010833A80108E8
:1003D0002DA9010877A8010810A901081EA9010884
:1003E000CAA8010843A90108F2A8010863A90108E5
:1003F0007EBA0108012A03D0022A03D000207047E8
:100400000160FBE70B680360F8E7006812F0F2B9DF
:1004100008B5402010F0DEFA202010F0E1FA10F0CC
:1004200047FC014B187808BD580C002008B510F0A7
:1004300095FF012871F1000306DB04480AF0DEF99C
:10044000BDE808400FF062B808BD00BFD3AB01089B
:10045000F8B5194E194F1A4D4EF6602010F03EFCBB
:10046000044640B917480AF0C9F92E21164802F08F
:1004700043F82046F8BD0178022904D113480AF058
:10048000BDF93521F2E7427E30460AF0B7F923780C
:10049000032B04D138460AF0B1F90FF037F8637E28
:1004A000002BE6D028460AF0A9F9204612F0A2F95E
:1004B00010F074FCD0E700BFD9AA0108D3AB010843
:1004C00004AB010889AA01087EBA0108A2AA0108A2
:1004D000F8B5254D254E264F10F040FF012871F14B
:1004E000000304DB28460AF089F90FF00FF810F03A
:1004F0000DFC18B17E21304601F0FEFF01230022E1
:100500000421384610F00CFDFFF7A2FFD0F8A03010
:100510000446CBB11A7F597F16480AF06FF9D4F818
:10052000A0305A7FE02A0FD11A7F042A0CD19B6E8B
:100530001A78012A08D15A78012A05D19A78012A15
:1005400002D1DB78012B06D00B480AF057F9204680
:1005500012F050F9C0E709480AF050F9204612F0AD
:1005600049F9074B1878F8BDD3AB01087EBA0108EA
:1005700077AB01087CAB0108C6AB0108A8AB01084A
:10058000F405002007B58DF8041001A98DF80520A9
:100590008DF8063004F0EEFB03B05DF804FB10B5F7
:1005A0008368044613B1032201469847204610BDD4
:1005B00070B50646D0F8A000C0B060B1437FE02B14
:1005C0003AD1057F836E012D1C7806D12CB93048B5
:1005D0000AF014F9022040B070BD022C53D0032C55
:1005E00053D0042C2AD12B480AF008F9FF2200210D
:1005F000684617F02EFC01238DF800409D4208DD6F
:10060000D6F8A020926ED25C01320DF8032001339F
:10061000F4E7FFF70BFF10F079FB18B1C6211E4875
:1006200001F06AFFE02300222946684610F078FCBA
:10063000E0B91A480AF0E2F80020CCE7052C17D1FF
:1006400017480AF0DBF80023ADF8003001238DF8DD
:10065000023010F05BFB18B1D5210F4801F04CFFC0
:100660000021009BE022084610F0B0FB0320B2E717
:10067000012DE1D1062CDFD10A480AF0BFF808F0BD
:1006800009F92846A7E70420A5E70520A3E700BF4E
:100690008EA90108ABA901087EBA0108BBA901080F
:1006A000CDA90108E5A901082DE9F047DFF8F080A0
:1006B0000024C146354FC0B001F04EFE21466846C9
:1006C0000AF0B1F9FFF7B2FE10F020FB20B14FF4B1
:1006D0008171384601F010FFE02398F800200221D4
:1006E000684610F01DFC38B929480AF087F84FF425
:1006F0007A700DF07DFCDFE7FFF7AAFED0F8A0309E
:1007000005462BB10134A4B2214622480AF076F8FE
:10071000DFF880A02846FFF74BFF0646284612F078
:1007200069F8052E22D801A353F826F0B90600086F
:100730006D070008810700084507000861070008E9
:1007400069070008FFF784FED0F8A0300546002BAB
:10075000E0D00134A4B2214650460AF04FF8D9E760
:10076000012389F80030A7E70023FAE731460A4859
:100770000AF044F84FF49471384601F0BDFE9BE74F
:10078000064B187840B0BDE8F08700BF7EBA01087C
:100790001DAB01083FAB01085CAB0108580C002001
:1007A000F50500206E232DE9F04F85B00193324B03
:1007B00088460293002301A904469346039304F05C
:1007C00013F961262D4BDFF8DC9002932C4B89F84E
:1007D000000001A920460196039304F00DFA294B6D
:1007E00082460293284B01A920460196039304F008
:1007F00003FA264B05460293254B01A92046019694
:10080000039304F0F9F9234B07460293224B01A905
:1008100020460196039304F0EFF906464146DFF8BF
:10082000888053465A462046FFF7ACFE2B4698F880
:10083000002051462046FFF7A5FE184A2B462946C0
:1008400020461278FFF79EFE154A3B462946204671
:100850001278FFF797FE334699F800203946204674
:10086000FFF790FE3B4698F8002031462046FFF700
:1008700089FE05B0BDE8F08FF6A9010809AA0108B4
:100880001104000813AA0108C10800081DAA0108E4
:10089000D104000832AA0108A90600085A0C002059
:1008A0005C0C0020F4050020580C0020826810B574
:1008B0000AB915F08CFDC368BDE810401847000068
:1008C000F0B5234D234E244F89B010F04DF818B9E0
:1008D000224B187809B0F0BD10F024FAFFF7B8FDEC
:1008E00000230446022204A9049068460293CDE93D
:1008F0000665FFF77FFD079B04A80393069B029301
:10090000FFF74DFE237804226178384609F076FF20
:100910006378042B03D05F21114801F0EDFD2378AB
:10092000032B01D10EF0F2FD237E4BB90D4809F0E7
:1009300065FF6846FFF7BAFF6846FFF730FEC4E779
:100940006846FFF7B3FF6846FFF729FEC0E700BF20
:100950000B040008F503000840AA01085C0C002005
:100960007EBA010875AA0108FF22014B1A70704770
:10097000F405002010B50020002105F073FB0446AB
:1009800028B9124809F03AFF114B187810BD417987
:10099000104809F033FF6179802905D0842911D0EE
:1009A0000D4809F02BFF05E00C4B227921681868EF
:1009B00002F070FE204605F0BDFE0821204606F03C
:1009C00063FBE1E70122064B1A76F3E70EAE01085E
:1009D000580C002016AE01081FAE010820060020AA
:1009E0005800002010B501F089F90446084809F0C4
:1009F00005FF204600F0E2FE064916F01BFC16F04B
:100A000005FE4FF40043044C6085238510BD00BFF4
:100A1000B7AF010800007A4458000020054B30B4FD
:100A20001C6823689D681346AC460A46014620466A
:100A300030BC604718060020054B30B41C682368A2
:100A40005D681346AC460A460146204630BC604706
:100A500018060020034B01461B681A6818461269E5
:100A6000104700BF1806002008B5044809F0C6FE6C
:100A7000BDE80840112007F008BF00BF2FB00108F3
:100A800008B5044809F0BAFEBDE80840132007F095
:100A9000FCBE00BFD6AF010808B5044809F0AEFEA1
:100AA000BDE80840122007F0F0BE00BF06B0010804
:100AB00008B5044809F0A2FEBDE80840102007F080
:100AC000E4BE00BF19B00108064B1B685B6833B970
:100AD000054B187A08B15B7A13B100F075BD01209F
:100AE000704700BF200600205800002070B5144C4D
:100AF000237E0BB3637EFBB90125124809F07EFE0D
:100B000004F0BDFF06F03EF8022106F049F806F0B9
:100B100039F8012106F044F8D4E900236576C4E9E8
:100B2000082314F06EFD064630B9074809F066FE4A
:100B300084F82C5025726672044B187870BD00BF83
:100B400058000020A4AD0108C5AD0108580C0020D4
:100B5000F7B5194F04463B680E465B688BB1174DDD
:100B6000174809F04BFE0DF1070332462946386855
:100B700002F01EFB9DF8073025606371207103B001
:100B8000F0BD104D2B7A7BB16B7A6BB90E4809F032
:100B900035FED5E90023C5E904230123314620466B
:100BA0006B7200F0DBFCEAE7084809F027FE3146EB
:100BB000204600F02BFDE2E7200600205807002029
:100BC000E4AC0108580000200AAD010827AD010877
:100BD0002DE9F8434FF0004700268046894605F08E
:100BE00033F9144BD3E90045BD4208BFB44205D0E8
:100BF00014EB080045EB0901C3E90001D3E9044502
:100C0000BD4208BFB44205D014EB080045EB090112
:100C1000C3E90401D3E90801B1F1004F08BF00287E
:100C200005D018EB000449EB0105C3E90845BDE810
:100C3000F88300BF58000020D0B501F05FF8C36B07
:100C40003C301B689847254CC4E9000109F056FD6B
:100C50000146234809F0D2FDFFF7C4FED4E904237E
:100C6000B3F1004F08BF002A2DD0D4E900671D481A
:100C700009F06AFC864277EB0103ACBF0123002335
:100C8000237200236372D4E90823B3F1004F08BF35
:100C9000002A1AD0D4E90067134809F055FC8642AF
:100CA00077EB0103ACBF012300230022627684F8B6
:100CB0002C20227A237662B14BB10C4809F09EFDBC
:100CC0000B4B1878D0BD0123DAE70123EDE7094883
:100CD000F4E70BB10848F1E70848EFE758000020B7
:100CE00042AD0108180000203800002058AD01086E
:100CF000580C002072AD010883AD010892AD0108C7
:100D0000F8B53F4D14F0FCF9D5E90823B3F1004FD5
:100D100008BF002A2C4611D1D5E90023C5E90823D4
:100D2000384B93F8503033B1374809F067FD012351
:100D30002B76364B4DE0364809F060FD00F0DEFFC3
:100D4000C36B3C301B689847D4E90023461C41F133
:100D50000007B3F1004F08BF002A3CD12D4809F02D
:100D60004DFD01232372D4E90023B3F1004F08BFE6
:100D7000002A38D1284809F041FD01232376237A3F
:100D800013B1637A002B36D0237E0BB1637E93B30D
:100D900000F0B4FFC36B3C301B68984702460B461B
:100DA00004461E480D4609F0CFFB09F0A7FC01469A
:100DB0001B4809F023FD2B4622461A4809F0C4FBC4
:100DC00009F09CFC0146184809F018FD01F0C4FA2E
:100DD000164B1878F8BD114809F0B6FB864277EB40
:100DE0000103C0DBBAE70F4809F0AEFB864277EBA0
:100DF0000103C4DBBEE70E4809F000FD99E700BF20
:100E000058000020040000209CAE01085B0C00206C
:100E1000C2AE0108EDAE010821AF010818000020A4
:100E200053AF01083800002074AF0108580C0020AF
:100E300095AF01081FB56123CDE9013101A90392E6
:100E400003F0DAFE05B05DF804FB00002DE9F04F79
:100E500087B0FFF73FFAFA200DF0CAF8FFF784F9E0
:100E600000F04CFF6A4B6B4D03646B4809F0C6FC05
:100E70002B686A4C13F0010F06D100F03FFF00F021
:100E800099FF012320602B60654D26682A6B654918
:100E900003A803F04FFD03A9304603F0A5FD266823
:100EA0002A698DF80500604903A803F043FD03A9F2
:100EB000304603F099FD5D4A8DF806005C492068D4
:100EC000FFF7B8FF8246206804F0F8FD594A8DF814
:100ED000070059492068FFF7ADFF584A06465849B0
:100EE0002068FFF7A7FF574B8346574A57492068AA
:100EF00005F022FB564A804656492068FFF79AFFC4
:100F0000554A8DF8040055492068FFF793FF9DF876
:100F1000053081468DF80C309DF8063003AA8DF817
:100F20000D304F490223206804F00AFF07464D4D5B
:100F300020689DF8073080F828A02A785146FFF7EE
:100F400021FB494B51461A782068FFF72BFC474A92
:100F500033469DF8071020681278FFF713FBDFF87F
:100F600018A143462A7831462068FFF70BFB434619
:100F70002A789DF804102068FFF704FB9DF80430E0
:100F80009AF8002041462068FFF7FCFA4B462A7881
:100F900041462068FFF7F6FA354A3346494620684D
:100FA0001278FFF7EFFA3B462A7849462068FFF7A8
:100FB000E9FA9DF804309AF8002039462068FFF7D6
:100FC000E1FA5B469DF8052039462068FFF7DAFA1A
:100FD0005B469DF8062039462068FFF7D3FA334672
:100FE0002A7859462068FFF7CDFA206804F07EF889
:100FF000204809F003FC01224FF41671206804F028
:101000000FF800200CF05AFD07B0BDE8F08F00BFCC
:10101000D10B0008000600203FAE01081C0600208E
:10102000040000202DA9010838A9010811110008A9
:1010300047C20108ED0A00085CAE0108390C00083F
:1010400064AE0108510B0008C90A00086BAE010824
:101050007509000876C10108010D000878AE010885
:101060002AC20108580C0020040600205C0C002055
:101070005B0C002082AE0108220D002000F03EBE75
:1010800013B500F03BFE044603689B68984723684D
:101090002046DB6801219847236820461B694FF4EE
:1010A000FA71984723682046DB680021984700249E
:1010B00001234FF496720B49CDE900340A482346C8
:1010C0000CF0FCFB094809F099FB094809F096FB74
:1010D0000CF0E4FD40F20121064801F00DFA204633
:1010E00002B010BD44B001084D0E00084DB001081B
:1010F00060B001087EBA010810B50446006810B15E
:10110000012105F0C1FF204610BD000000000000D5
:101110002DE9F04FB64C9BB02368DB0708D402F0F2
:1011200095FF80220146B34801F0E8FF01232360C8
:10113000B04AB14BB14E1A6000F0E0FD34460127D1
:10114000AF4BB04D8365B04B1AA80D93AF4B0C93CA
:10115000AF4B0B93AF4B40F8403D05F0C3FA0FCDBA
:101160000FC40FCD0FC495E80F00377284E80F004D
:1011700000F0C4FDC36B3C301B689847002300227D
:1011800033764FF00043A44DC6E908232B68C6E927
:10119000000113F0010FA14C04D100F0AFFD4C3061
:1011A00020602F60206803681B689847044618B9C0
:1011B000EE219B4801F0A0F99A4B11939A4B0F93A3
:1011C0009A4B0E939A4B10939A4B07939A4B099311
:1011D0009A4B089300F092FD02AB07AA00F13C0580
:1011E00007CA83E8070010AB93E803008DE803000B
:1011F0000EAB0CCB2146284605F08EFC904905F03D
:1012000085FD05F0BFFC13F07BFFFFF7EBFB00F063
:1012100075FD16AA044617468A4B00F14C0503F1EA
:10122000100C164618685968083303C663453246E1
:10123000F7D1E36C01211B6928469847E36C3A46D5
:101240009E687B2110232846B04712AE1022002151
:10125000304616F0FEFDE36C3246D3F804807B2165
:1012600010232846C04710223946304616F0BEFDEE
:10127000E36CB0FA80FAD3F80C80212210237B2192
:101280002846C047E36C3246D3F804807B21102304
:101290002846C04700234FEA5A1AF25C0133212A3C
:1012A00018BF4FF0000A102BF7D1E36C00211B6927
:1012B00028469847204600F081FA15F04BFB48A3DA
:1012C000D3E900238046894615F022FE002800F06D
:1012D000D78045A3D3E90023404649464FF0010596
:1012E00015F00CFE00B90546EDB204F14F025F3473
:1012F00012F8013F002B40F0C580A242F8D11C46F5
:10130000BAF1000F00F0C080002D14BFA3464FF0CB
:10131000000BDFF86481DFF864914B4809F06EFA46
:101320003F4BBAF1000F14BF4A464246474948486E
:1013300009F064FA3A4B002D14BF4A46424645492B
:10134000434809F05BFA364B002C14BF4A4642462C
:1013500041493F4809F052FA40494148BBF1000F6A
:1013600008BF414609F04AFA3E4809F047FA02F040
:101370006DFE3D4A0146304602F09DFC00230820E8
:10138000CDE91633189309F0D5FA384A00F108036D
:101390001690189312F8011F00B1017001308342BA
:1013A000F8D1DDE9120216991793121A5B1A9A42C4
:1013B0006CD11AB116F01AFD002867D12C4809F03B
:1013C0001DFA2C4B1C783846FFF796FE3046FFF787
:1013D00093FE20461BB0BDE8F08F00BFAFF3008046
:1013E000CDCCCCCCCCCC004033333333333313406F
:1013F000F8050020080600202006002058000020E4
:1014000049600008F0AB0108690A0008810A000879
:10141000990A0008B10A0008FC05002018060020FF
:101420007EBA0108FDA700081D0A0008390A000855
:10143000550A00083D630108DD620108A163010847
:101440000400002020AC010845AC010855AC01089F
:101450005AAC010871AC010875AC010842AC010836
:101460007CAC010891AC01089FAC01082FAC0108CD
:10147000A6AC0108040600203DAC010838AC010808
:10148000054632E701243BE7D34642E7004B99E7A4
:10149000580C0020FF22014B1A70704704060020F0
:1014A000054B1A68054B93F84F30B2FBF3F003FB82
:1014B000102303B1013070475407002004000020BE
:1014C00030B5CDB005F05EFB04A905F081FA1E4CE5
:1014D000002836D04FF496721C49684605F035FD59
:1014E00001231B4D8DF80C3095F84E307BB1002355
:1014F000059A684605F070FD95F84E30022B06D12E
:101500009DF8241068464942C9B205F049FD0CA96E
:101510000B9A684605F026FD684605F04EFD002250
:101520000C4B206068461A6005F045FD044668468D
:1015300005F043FD21460246074805F0BDFC4DB0CD
:1015400030BD2060FBE700BF5407002024060020C8
:101550000400002050070020880000207FB50126ED
:101560000A4604461649684605F0EFFC0221684623
:10157000144D8DF80C6005F013FD0521684605F04B
:101580000FFD0D21684605F00BFD698D684605F0DD
:101590002FFDB5F92810684605F011FD95F82C10BF
:1015A000684605F0FDFC684605F005FD0546684601
:1015B00005F003FD66712560207104B070BD00BFA9
:1015C000580700205800002038B50E4C23683BB95E
:1015D00014F003F8002801DDFFF772FF236863B100
:1015E00014F00FF8054613F0F8FF2D1A14F009F85F
:1015F00029460246044809F001F92068003018BF66
:10160000012038BD54070020CCB001082DE9F3417A
:10161000364E074696F84E500A4634468DB1022D96
:101620005CD8334D334C2946204605F017FC96F81C
:101630004E30387164337B71D4E902233D609A42A5
:1016400040E0FFF72DFF2C4E3368984241D994F8C3
:101650004F502A4A03FB0525294B1978FFF720FF35
:10166000336894F84F20984294BF00235343C91A1B
:10167000CCB2944228BF14461CB97321214800F013
:101680003BFF31684FF00A080131FFF709FF08FB03
:1016900001085FFA88F3024600931B48234609F0CD
:1016A000ADF82146284609F00FF9184809F0A6F8C8
:1016B000316887F8058001313D603C713160FFF78A
:1016C000EFFE814202D100220D4B1A6002B0BDE84C
:1016D000F08171210B4800F00FFFBDE7A8210948F8
:1016E00002B0BDE8F04100F007BF00BF04000020D9
:1016F0005807002088000020500700202406002002
:10170000540700207EBA010891B001087DBA010893
:10171000704710B504465C2105F0B6FC204610BDAC
:1017200081F001020148032106F0D4B90000024013
:1017300007F0B0B810B50C460CF0C8FE022808D16E
:101740004FF47A704443B4FBF0F0BDE810400CF065
:101750004FBC2046BDE8104005F022BF08B5034845
:1017600009F04CF8BDE8084007F094B844B401080B
:101770007FB5F82300F1440504AC0646284604F87A
:10178000013D00F017FD0223214600930122A02312
:10179000284600F013FD4FF400430822009306F1A1
:1017A0005001A0230446284600F032FD0440E4B274
:1017B000284600F001FD204604B070BD05F0B8BD1C
:1017C0002DE9F047044605F0B3FD2149054615F023
:1017D000CFFE002836D00FF27009D9E900892368BE
:1017E0000121DB6820469847DFF870A0194F284692
:1017F00015F0B0F842464B4615F076FB0646B8B1F8
:101800005146284615F016FD15F0DAFE40F6C412D2
:10181000014640F62823384608F0F0FF23684FF4CD
:101820007A711B692046984705F082FD0546DEE780
:10183000094808F0E3FF236831462046BDE8F04739
:10184000DB681847BDE8F087CDCCCCCCCCCC0440CD
:101850000000204014B101084DB1010800007A4495
:1018600030B5524B8BB019680446514808F0C6FF9A
:1018700006F0E8FF01464F4808F0C0FF00F090FB7B
:101880004D484E4908F0BAFF04F1440000F08CFCCA
:1018900030B94B4808F0B2FF6E214A4800F02CFEE8
:1018A00005F064FE2046FFF763FF18B97321454831
:1018B00000F022FE94F8570094F85230049094F807
:1018C000560094F85120039094F8550094F8501065
:1018D000029094F85400019094F8530000903A4814
:1018E00008F08CFF04F14C0000F01AFC00F06CFBD7
:1018F000364808F083FF4FF4FA7016F047FA0546B1
:1019000000284BD1324808F079FF324808F076FFC2
:10191000314808F073FF314808F070FF304808F094
:101920006DFF304808F06AFF2F4808F067FF2F4826
:1019300008F064FF2E4808F061FF2E4A2E492F4818
:1019400008F05CFF2E492F4808F058FF2E4808F099
:1019500055FF2E4B2E4A1B682E4900932E4B1268C2
:101960001B682E4817F0F2F92C492D4808F046FF65
:101970002C492D4808F042FF07A806F0B7FA07A83F
:1019800008F092FE0146294808F038FF124808F096
:1019900035FF2046FFF714FF0BB030BD244808F098
:1019A0002DFF284616F0FAF9AFE700BF9C00002093
:1019B00060B1010876B101088CB10108A086010070
:1019C000A7B101087EBA0108BDB10108F2B1010852
:1019D00020B201087CBA01085EB201088FB201088A
:1019E0009EB20108C0B20108E3B2010807B30108C2
:1019F0007DBA01082AB3010835B3010849B30108CB
:101A00005AB3010864B301086FB301086400F81FFA
:101A10005000F81F8FB301085400F81F4008002041
:101A2000A1B30108ACB30108B2B30108CCB30108FB
:101A300054B2010870B50446344E354808F0DEFE55
:101A4000204605F0EBF914F049FC0FF0EBF80DF02F
:101A50003FFB0EF057F9012230460C2105F0C2FF82
:101A600006F0DCFB23680021DB682A4D20469847FE
:101A700006F096F8284808F0C1FE06F0FDFC05F0D7
:101A800067FD284601220D2105F0ACFF2846012202
:101A90000E2105F0A7FF01222846032105F0A2FF31
:101AA0000021084606F066FB002328461A4603215B
:101AB00005F05AFF01220321284606F00BF804F135
:101AC000440000F071FB4FF4E13006F0E7FD1348ED
:101AD00008F094FE30460C2105F0F0FF002330465C
:101AE0001A460C2105F040FF0021084606F0BAFB1B
:101AF0000EF01AF90DF012FA06F08EFB2046FFF7F1
:101B00005FFE2046BDE8704005F098B90004024031
:101B1000DEB301080000024002B4010849B5010823
:101B200038B50C46113105460EF02AFF214651F812
:101B3000503F28462B604B686B6038BD30B50D4672
:101B40009DB0044601466846FFF7EAFF694628460D
:101B50000EF054FC04F1110321346B632C631DB0AF
:101B600030BD00002DE9FF4100F14405284600F09A
:101B700021FB04240226284F013C14F0FF0432D03C
:101B8000A123012239460096284600F017FB4FF4A6
:101B90000043804600930422A12302A9284600F0B6
:101BA00037FBB8F1000FE7D00028E5D09DF80830EA
:101BB000442B1FD19DF809306E2B1BD10DF10A006B
:101BC00008F00BFF013084B221460DF109008DF8B9
:101BD000086008F028FF002303220093A02302A935
:101BE000284600F0EBFA284600F0E6FA204604B05A
:101BF000BDE8F0814FF488430024ADF808306E232F
:101C000000210DF10B008DF80A3008F00CFF009454
:101C1000A0230522E3E700BFE9B00108F7B50446B9
:101C200005F0F2F81B4B1C4A23601C4B6264E36313
:101C300000231B4A1B4E236484F84830E264C4E945
:101C40001433A365184808F0D9FD3368174F019382
:101C50003B68174D00932B68164A1B2104F12100A5
:101C600017F040F8296804F1110008F0D3FE396834
:101C700004F1150008F0CEFE316804F1190008F0F7
:101C8000C9FE296804F11D0008F0C4FE204603B017
:101C9000F0BD00BF30B40108E0B4010824B501086C
:101CA000C4B401086400F81F10B401085400F81F00
:101CB0005000F81F8FB3010810B506F069FD0A4CFB
:101CC0000A4B186000F038F92368DB0709D408488C
:101CD000FFF7A4FF0123074A07490548236014F0D2
:101CE00071FB034810BD00BF380800209C00002095
:101CF0005C080020000000201117000838B5064DD0
:101D0000064C2B6813F0010F04D1FFF7D5FF012318
:101D100020602B60206838BD3C080020B8080020F7
:101D200010B5FFF7EBFF836D2BB1FFF7E7FFBDE8C1
:101D30001040836D1847BDE8104006F0ABBD08B5F4
:101D4000FFF7DCFFBDE80840FFF774BE30B508467A
:101D50008DB014460F4B104A104902F0C5F800210F
:101D60000F4A0A9107920F4A069108920E490F4AAC
:101D70000F4D09920494059104AA01AC07CA0B9572
:101D800084E8070007AB00950FCB02F0E3FB0DB032
:101D900030BD00BF31170008EAB001080EB10108DC
:101DA0005D760008E5750008000008085D1700086A
:101DB000211D000838B5054602F004FF074B044614
:101DC0001A784AB1002205F13C011A7002F0C8FDF0
:101DD0000349204602F0C6FD204638BDA000002081
:101DE0003F1D0008032006F0A5BC10B50446FFF710
:101DF00085FF2146BDE81040FFF7B4BE38B5384D29
:101E00000DF0B8F928460222002105F0EBFD284626
:101E10000222012105F0E6FD002328461A4603218F
:101E200005F0A2FD28460222082105F0DBFD284628
:101E300002220B2105F0D6FD284602220C2105F0D6
:101E4000D1FD284602220D2105F0CCFD28460222B4
:101E50000E2105F0C7FD284602220F2105F0C2FD24
:101E60000222204C1146204605F0BCFD20460222ED
:101E7000032105F0B7FD20460022062105F0B2FD42
:101E800020460222082105F0ADFD2046022209214C
:101E900005F0A8FD204602220C2105F0A3FD2046F6
:101EA00002220D2105F09EFD0F2328460222082163
:101EB00005F038FC204601220C2105F093FD204658
:101EC00002220D2105F08EFD204602220E2105F092
:101ED00089FD2046BDE8384002220F2105F082BD71
:101EE000000002400004024008B50D49012005F041
:101EF000BBFE0C490B2005F0B7FE0B490A2005F08C
:101F0000B3FE0A49042005F0AFFE0949072005F099
:101F1000ABFEBDE808400749052005F0A5BE00BF9F
:101F200069C50008DDC800082DC7000825CA0008DB
:101F30005DC90008F1C9000808B5022005F08EFA55
:101F400005F0F0FAFFF75AFF05F002FBFFF7CCFFB0
:101F500006F034F80C4800F099FA4FF4E13006F03E
:101F60009DFB0A4B1A680AB9094A1A60094B1A689C
:101F70000AB9074A1A60084808F040FCBDE8084062
:101F8000064808F03BBC00BFE51D0008600E0020BD
:101F90003D850008640E002066B401087EB4010887
:101FA000002307B5ADF804308DF8063001238DF815
:101FB000053001980DF03AF805F0CAFA03B05DF863
:101FC00004EB0DF085B800002DE9F04FA5B00DF041
:101FD00079FCDFF800A1374EDFF8FC80DFF8FC90D9
:101FE0001CAF50B9CDE91F66CDE91D98CDF870A0A2
:101FF000009697E80F000DF07FFC2F4B00241593FF
:102000002E4B06A914932E4B14A816932D4BCDE9F5
:102010001A9817932C4B6D46CDE918360423CDE959
:10202000063409F017F909F009F908F043FD032314
:1020300021460994142224AC1FA8089315F009FF27
:1020400044F8188D0FCCCDE91C690FC594E8030046
:1020500085E803000DF1200B97E80C009BE80300D6
:1020600014F088F818B9F421184800F045FA002255
:10207000CDE90B220D92164A0AAB139203220A9263
:10208000012202AC8DF82E200FCBCDE91198CDE9BD
:102090000E66CDF840A084E80F0012AB93E8030071
:1020A0008DE803000EAB0FCB0EF0BEFC25B0BDE8F3
:1020B000F08F00BFFDA7000855F000081DEF0008D5
:1020C0002DEE0008C5ED0008D9ED00087EBA010824
:1020D000EB1D0008A97F000809A9000835A9000820
:1020E0000DF036BD084611461A460DF0CFBD084624
:1020F00011461A460DF04CBD084611461A460DF021
:1021000081BD09B10DF010BE0DF0FCBD0C2110B168
:10211000024805F0D3BC014805F0D6BC00040240DB
:1021200000B50C2189B0194805F0C8FC00230C212A
:102130001A46164805F018FC0021084606F092F8E9
:1021400000220592124A02AB0292124A0692124AE9
:102150000392124A04924FF40042079208AA12E92D
:1021600003008DE803000FCB0DF0F6FD40B10DF03C
:10217000EFFC01460A4809B05DF804EB08F03EBBED
:10218000084809B05DF804EB08F038BB00040240D1
:102190000D210008A175000819830008FDA700089B
:1021A00094B40108AAB40108014805F0E7BC00BFD7
:1021B000A086010005F0B2BC05F0CCBC2DE9F041D1
:1021C000069F1E4607F00303032B80460C46154668
:1021D00003D119210D4800F08FF92046BC07324683
:1021E00029460AD505F004FD10B10120BDE8F081B3
:1021F0000123002088F80430F8E7FB0702D505F03A
:1022000005FDF1E705F0E6FCEEE700BF7EBA010848
:102210002DE9F041069C0D46E107804616461F4613
:1022200003D536210D4800F067F9A20703D53921FF
:102230000A4800F061F923043A46314628460AD597
:1022400005F0F2FC10B10120BDE8F081012300206F
:1022500088F80430F8E705F0AFFCF3E77EBA010830
:1022600005F0A2BE1FB501A808F0E0F901A805F02D
:102270007BFF05B05DF804FB05F0E4BE05F0FCBE95
:10228000084605F073BDDFB50023CDE90133ADF895
:102290000C3001238DF807308DF808306FF01D03E6
:1022A0008DF809300723044601A88DF80A3008F09C
:1022B000E2F9236806461B6820460F469847864287
:1022C00077EB0103B4BF0120002004B0D0BD70B58E
:1022D0000646194610461D4614460DF057FB736816
:1022E00023B120462946BDE87040184770BD000064
:1022F0002DE9FF4714461D46824605F055FE8046EF
:102300008946261A22462B4601A865EB010708F0EC
:102310008DF94046494608F0F1F9294680462046A5
:1023200008F0ECF939460446304608F0FDF922463B
:1023300003464146074808F061FA01A805F0C6FDCA
:1023400020B132463B465046FFF7C1FF04B0BDE81E
:10235000F08700BFF4B401082DE9F04741488AB086
:1023600008F04CFA0BF0FAFC2425079007993E4838
:1023700008F044FA0798684308F0DCFA04463B4842
:1023800008F03CFA94B107990DEB050220460CF0D9
:1023900045F80023DFF8F0A0354F07900893089A1E
:1023A000079B9A421DD3204608F0AEFA0AF0DEFCE5
:1023B00004460AF0E9FC214602462E4808F01EFABF
:1023C0002D4B2E4819889A888B1A08F017FA2C4B37
:1023D0001B6803B198472B4808F010FA0AB0BDE813
:1023E000F087089B05FB03431B7B042B98BF1AF85F
:1023F0000320099B88BF3F22642B83BF6420B3FB6B
:10240000F0F30899002382BF05FB01418969B1FB04
:10241000F3F308990898DDF820C0DDF820E0DDF836
:102420002080DDF8209005FB004005FB0949D9F824
:102430001C6005FB0141CDE9033605FB08439B69A0
:10244000029305FB0E439B68019305FB0C431B8C19
:10245000009303694968384608F0D0F9089B0133B6
:1024600008939CE745B5010851B501085CB5010822
:1024700091B50108C3B50108A2190020E2B5010811
:102480003409002085B0010840B50108014B1860EF
:10249000704700BF5009002073B5124C06462378E0
:1024A0000D46114A1BB913780BB172B6FEE7012332
:1024B000002113700D48642215F0CBFC2B460096CA
:1024C0000B4A6421094816F00DFC0A4B1B6803B146
:1024D00098470125054E304608F0D4F972B62570AC
:1024E000F9E700BF2C090020C0080020C208002026
:1024F00019B6010850090020F7B5184C0646237894
:102500000D46174A1BB913780BB172B6FEE70123CB
:10251000002113701348642215F09BFC2B46009693
:10252000114A64210F4816F0DDFB104B1B680BB1FC
:102530000C4898470E4B1B6803B198470125094E7C
:102540000C4F304608F09EF9384608F09BF972B6F9
:10255000094B257000BF013BFCD1F2E72D0900209B
:10256000C1080020C208002041B60108BC080020B4
:102570005009002050B60108FFFF0F00F8B5DFF842
:1025800098C003681A4FCCF800304368194E3B607E
:102590008368194D3360C368184C2B600369184970
:1025A0002360436982690B60164BC0691A60164A42
:1025B0001060DCF8000038683068286820681C4625
:1025C0000968124D1968124E1268642200212846CB
:1025D00015F03FFC236832466421284616F082FB42
:1025E000284608F04FF90B4B00BF013BFCD1ECE74C
:1025F00040090020480900204C090020440900201F
:10260000280900203009002038090020C2080020D5
:1026100006B60108FFFF0F003C090020074B1B68AE
:1026200003B198471EF0040F0CBFEFF30880EFF3DF
:1026300009808169004A10477D2500085009002063
:1026400010B1012104F020BD704708B108F072B943
:10265000704780687047406870474368012B08D115
:10266000D0E90432934204D01878003018BF01201A
:102670007047002070474B6870B5042B04460E4627
:102680004FF0000304D0C0E900338360204670BDE2
:10269000D1E90425AD1AC0E9003383602846FFF76D
:1026A000D4FFC4E900000544A560D6E904530246FE
:1026B00029468B4205D00AB10E78167001310132DD
:1026C000F7E75B1B18446060E0E742680346022AB4
:1026D00006D1D3E904031B1A032B01D908F08BB9E7
:1026E000002070474368032B06D1D0E904329A4298
:1026F00008BF0023184670470023FBE7037870B536
:1027000081680446B3B1284A284808F077F863681E
:10271000022B12D12046FFF7D8FF0146244808F0CB
:102720006DF8E1680B78002B3CD02248BDE8704082
:1027300008F064B8204A2148E7E7032B05D120467A
:10274000FFF7D0FF01461E48E9E7042B0ED1002514
:102750001C4ED4E90431C91A8D4205D2595D304668
:1027600008F04CF80135F4E71748D8E7012B08D1F9
:102770002046FFF772FF1549154B002818BF194670
:10278000E1E700250F4ED4E904239B1A9D4205D2B0
:10279000515D304608F032F80135F4E70D4808F095
:1027A0002DF8BEE70C48C1E731A80108F4B60108CE
:1027B00008B701082AB701087EBA0108FEB6010869
:1027C00062B801081FDA010812B70108EEB6010865
:1027D000E9B6010818B701087DBA0108B1F5A04FA4
:1027E0002DE9F84304460F4602D9174804F00CFCC3
:1027F000066883689B1B994219D9D0F80490084653
:10280000FFF723FF05460346A9EB0608B14505D0AF
:102810000BB132781A7001360133F7E72068FFF701
:102820000FFF05EB080325603D446360A560256844
:102830003DB92846C4E90155FFF702FF2846BDE827
:10284000F8830120FBE700BF6CB601082DE9F041D9
:102850000368561A904682680446D21A96420D467C
:1028600015D93046FFF7F1FE07460346A84505D0C7
:102870002A7803B11A7001350133F7E720683E4426
:10288000FFF7DEFEC4E901662760BDE8F081476816
:10289000481EFF1ABE420ED81A469D19A91A0029D1
:1028A00004DD10F8011F02F8011BF7E7002EA8BF96
:1028B0009B196360E9E73D441F44FA1A002A04DDCE
:1028C00010F8012F03F8012BF7E763682E4618462E
:1028D000B04505D0327800B1027001360130F7E71B
:1028E000A8EB05084344E4E708B509C81B1AC3F57B
:1028F000A040884202D2104604F086FB994238BFBD
:102900001946581805D2B0F5A04F28BF4FF4A04083
:1029100008BD4FF4A040FBE72DE9F8430C46591CD5
:10292000204615461F46FFF759FF064680B14FF077
:102930000003EA1929462046FFF788FFD4E901532E
:102940009D4208D00DB100232B7063680133636092
:102950003046BDE8F8831B4A01212046FFF7C4FF3B
:1029600023680746A5EB0309FFF76FFE10EB090F7D
:102970001CBF002300F80930236880461A46014630
:10298000954205D009B11078087001320131F7E79E
:10299000D31A01334344104619466568954207D05F
:1029A00019B192F800C081F800C001320131F5E799
:1029B0002D1A1D4420684744FFF742FEC4E90085F4
:1029C000A760C5E7A7B601082DE9F04105460E4608
:1029D00061B1D0E90132D21A8A4209D300221E44E1
:1029E00003B11A700133B342FAD16B60BDE8F081D4
:1029F000114AFFF779FF8046FFF727FED5E900145B
:102A000007460A460346944205D00BB11078187069
:102A100001320133F7E70023641A3C44264404B131
:102A200023700134B442FAD12868FFF709FEC5E9E2
:102A300000744744AF60D9E7DBB70108D0E9003242
:102A4000D21A914210B503D9891AFFF7BDFF10BD04
:102A50003CBF5B184360FAE770B50C460121204685
:102A60001646FFF7BBFE054628B101212046FFF7B9
:102A7000E5FF23681E70284670BD0000426808B557
:102A8000012A06D1BDE808400A4600F11001FFF70F
:102A9000E3BF8168024807F0B1FE002008BD00BF17
:102AA0006AB7010810B50C1A134605D00146224634
:102AB000184615F0B5F90346181910BD2DE9F04177
:102AC0000446A2EB01081646A368226808469B1A32
:102AD00098450F4615D94046FFF7B7FD0546034612
:102AE000BE4205D00BB13A781A7001370133F7E7CF
:102AF0002068FFF7A5FD25604544C4E90155BDE800
:102B0000F0816568AD1AA84504D83146FFF7CAFFC1
:102B10006060F4E70D442946FFF7C4FF6368294667
:102B20001A468E4205D00AB1087810700131013280
:102B3000F7E7751B1D446560E1E770B50E46D2E905
:102B400000313046C91A1446FFF748FE054630B139
:102B5000D4E900124FF000033046FFF7AFFF2846DC
:102B600070BD000070B5D0E9043100F110060446D4
:102B7000C91A3046FFF732FE054640B1D4E90712C4
:102B8000914206D1A168064807F038FE0025284684
:102B900070BD4FF000033046FFF790FFF7E700BF2E
:102BA000C1B601082DE9F0418368A2EB0108174680
:102BB000026804469B1A98450E4615D94046FFF711
:102BC00044FD05460346B74205D0327803B11A707A
:102BD00001360133F7E72068FFF732FD25604544F1
:102BE000C4E90155BDE8F0814568AD1AA84505D88E
:102BF00039463046FFF756FF6060F3E70D4429463B
:102C00003046FFF74FFF636829461A468F4205D0CA
:102C1000087802B1107001310132F7E77D1B1D44C5
:102C20006560DFE737B50D4601A8114607F000FFE4
:102C300004212846FFF7D2FD044630B14FF00003CF
:102C400002AA01A92846FFF7ADFF204603B030BD18
:102C5000FFF7E8BF426808B5022A06D1BDE8084080
:102C60000A4600F11001FFF7DDBF8168024807F056
:102C7000C5FD002008BD00BFA2B70108FFF7EABFED
:102C80002DE9F0410E4600211C4617468AB00DF191
:102C900008082022C0E9001181600546404615F071
:102CA000D8F81E2C94BF22461F223946404615F004
:102CB000ACF87368013B032B14D8DFE803F0023053
:102CC000404722462F49384616F0BFF828B1224621
:102CD0002D49384616F0B9F840B901222946304648
:102CE000FFF7BAFE28460AB0BDE8F0812246274920
:102CF000384616F0AAF828B122462549384616F07B
:102D0000A4F808B90022E9E700220AA941F8242D15
:102D1000404616F0BFF9021C18BF0122DEE7002270
:102D20000AA941F8242D404616F0B4F9019B024649
:102D30004345D7D029463046FFF774FFD2E72346F4
:102D40003A4629463046FFF7E7FDCBE714F0010687
:102D5000C8D1640821462846FFF740FD0028C1D0AD
:102D600021462846FFF76AFEB442BBD0022107EB9A
:102D7000460007F079FE0028B4DB2B689855013631
:102D8000F2E700BFE9B601087CB60108EEB601081B
:102D900081B6010830B51346426885B0032A04465F
:102DA00000F110050A460FD0014601A8FFF768FFA1
:102DB000204601AA2946FFF7C0FE04460198FFF706
:102DC0003FFC204605B030BD2946FFF7A5FD04466F
:102DD000F7E70000F0B5044685B0104616460F46EA
:102DE00016F02BF862680346032A16D032462146B5
:102DF00001A8FFF745FFDDE9011291420BD04FF02A
:102E000000033846FFF75AFE01250198FFF718FC2A
:102E1000284605B0F0BD0025F7E7441C214638469A
:102E2000FFF7DCFC054618B9054807F0E7FCEFE7BB
:102E30004FF00003321931463846FFF707FDE7E748
:102E400087B601080A4600F11001FFF7C3BFF8B5C5
:102E50000D461946284616461F46FFF7BFFC044696
:102E600030B14FF00003F21931462846FFF79AFEC1
:102E70002046F8BD1346426810B5042A06D1BDE8C5
:102E800010400A4600F11001FFF7E1BF81680248D7
:102E900007F0B4FC002010BD31B701082DE9F04166
:102EA0000C4690461D46064640B139B108491846C1
:102EB00004F0E6F8074618B930602060BDE8F081FC
:102EC0002A46414614F0A1FF37602560F6E700BFAF
:102ED0004EEC010870B5054610460E46144615F036
:102EE000ACFF2246034631462846BDE87040FFF756
:102EF000D5BF000010B50C4631B1044900F00CFDFF
:102F0000231A5842584110BD0846FCE756B901083B
:102F100010B500B121B9064807F070FC002010BDC3
:102F20001AB9044AFFF7D6FFF8E70120F7E700BF18
:102F3000F5B7010802B801082DE9F74305460E462A
:102F400017469846FFF7E4FFC0B10F49222004F06E
:102F500097F80446A8B13846FFF77BFB8146384610
:102F6000FFF7C0FB15F069FF4346CDE90090074A23
:102F70002221204615F0B6FE30602C6003B0BDE87B
:102F8000F0833060F9E700BF4EEC010819B8010882
:102F90002DE9F8430E46984616F8013B02F1FF3939
:102FA00003704660C0F80890044615463D214A4625
:102FB000304614F00DFF074668BB4B46182B28BF60
:102FC0001823C4F83001A36204F10C05A26A31464B
:102FD000284614F01AFF0022A66AA3191A7337B103
:102FE000D4F83021791C04F12C0014F00EFF0022DB
:102FF000D4F83031234483F82C202EB129464046A2
:1030000000F08AFCC4F83401D4E901120A48BDE892
:10301000F84307F069BC831B023DED1A182B1A46D2
:10302000A8BF1822B5F5807F28BF4FF48075A26233
:10303000C4F83051C8E700BF21B8010830B50446D4
:103040000D46084B9DB00093074A084B642103A826
:1030500015F048FE03AA29462046FFF73BFF1DB0A6
:1030600030BD00BF2AB3010811B8010835B301080B
:103070002DE9F0431646642203F10C048FB0074695
:10308000884620461849ADF8042015F0C4FE70B9F2
:10309000336B23B1154A322101A815F023FE01AA92
:1030A00041463846FFF716FF0FB0BDE8F0832046D3
:1030B0000F4915F0B0FE0446A0B9736B002BEED09B
:1030C0000125DFF83490736B01A81B5DC5F1320157
:1030D00028444A46013415F005FE102C05F102057E
:1030E000F1D1DCE7034ADBE72DB8010832B801086B
:1030F00036B801083EB801081FDA01080160002156
:103100000273C0E901117047F8B5054617460E462F
:1031100039B332B32049182003F0A6FF044608B3A0
:10312000C0E9006700261D4B00F108074361C0E9B4
:10313000026606618021384603F0C3FED4E900121E
:10314000384603F0FDFE1449082003F08DFF90B1CE
:103150006B68C0E9004603B96860AB6803B15860AA
:10316000A860F8BD0E4807F049FB01213046BDE8D4
:10317000F84003F089BF0B4807F040FB0A4A40F2D1
:1031800055110A4807F03AFB0121206803F07CFF43
:1031900018212046EBE700BF4EEC010880818283B6
:1031A0007EDA010899B80108B5B80108ECB8010841
:1031B00070B54468054604B3266806F1080003F0BC
:1031C00089FED6E903239A42C4B216D16B681BB9B3
:1031D0006A210B48FFF790F96868082143686B6023
:1031E00003F052FF6B6803B9AB600121306803F054
:1031F0004BFF1821304603F047FF204670BD00BF4B
:103200007EBA01087FB50546FFF723FA15F015FED3
:103210000446861C2846FFF71EFA013803281DD8ED
:10322000DFE800F00206080F0734601C04B070BD30
:103230000D34FAE72846FFF755FA15F0FEFD34186D
:10324000F3E701A82946FFF716FADDE9014301A8D3
:103250001B1B06EB4304FDF74FFFE6E70B34E4E7E7
:103260002DE9F04786B08146884614461D46FFF793
:103270004FFE68B12046FFF7C5FF4049074603F0FF
:10328000FFFE0646C9F8000028B93D4807F0B6FA27
:1032900006B0BDE8F0872046FFF7DDF901380328C6
:1032A00064D8DFE800F00214253D2046FFF7D1F98D
:1032B00081462046FFF7D1F9324B334A002814BF2C
:1032C00018461046CDE900902B46304A0AE02046C9
:1032D000FFF7BFF981462046FFF7F7F92B46CDE906
:1032E00000902B4A3946304615F0FCFC05463AE082
:1032F000612D20460DD1FFF7ACF905462046FFF7BA
:10330000F1F92B46234A00903946304615F0EAFC85
:10331000ECE7FFF79EF981462046FFF7E3F9D1E796
:103320002046FFF796F92B4600901B4A3946304657
:1033300015F0D8FCDFF868902146054603A8FFF792
:103340009AF9DDE9034AA2450AD0AF4214F8013BDD
:1033500006D9791B70194A4615F0C4FC0235F2E70C
:1033600003A8FDF7C9FEC8F8005091E72046FFF713
:1033700070F92B460090094AC6E700BF4EEC0108E1
:103380007EDA0108E9B60108EEB601084DB8010879
:1033900055B801085EB8010865B801086BB80108A6
:1033A0001FDA01082DE9F0430E4607469046D1B0DA
:1033B0004FF49C72002102A81D46589C14F049FD50
:1033C00031463B46424602A8FFF7E2FD3678622EC0
:1033D00000F0F98029D83F2E54D008D82E2E5BD08B
:1033E0009DF808107D4807F009FA7D4A58E0532EF1
:1033F00000F0A180612EF3D10DF1340979484A46DD
:1034000005A907F0FBF94F98002800F0D580FFF7D9
:1034100022F9032800F0AF802846734A2146FFF7BF
:1034200059FD724807F0EAF933E0722E48D00ED801
:10343000642E3AD0672ED3D105A96D4807F0DEF986
:1034400033464F9A21462846FFF70AFF21E0732EA4
:1034500051D0772EC4D1674807F0D0F903990029DD
:1034600000F0BA80644815F0D6FC0646002840F00B
:10347000B380624807F0C2F93146384600F038FFA1
:103480005F4AA4E05F4807F0B9F921462846FFF7F4
:10349000D5FD51B0BDE8F0835B4807F0AFF95B4A5A
:1034A00021462846FFF716FDF3E70399584807F031
:1034B000A5F902AB3A4621462846FFF7D9FDE8E7D1
:1034C00005A9544807F09AF90399534815F0A3FC4D
:1034D00020B9384600F03AF9504AE1E74F993846AA
:1034E000FFF708FD08B14E4ADAE74F9808B1FFF739
:1034F00039FB7223A5E705A94A480DAA07F07EF912
:103500004F993846FFF7F6FC0028ECD14F9810B1E0
:103510000DA9FFF797FC73234F9A21462846FFF722
:103520009FFE2168404807F069F92868216807F084
:10353000CBF93E4876E705A93D480DAA07F05EF9AC
:103540004F993846FFF7D6FC0028CCD14F9810B1E0
:103550000DA9FFF777FC2146284673234F9AFFF702
:103560007FFE0121384600F0C3FE324807F046F9DD
:1035700001F026F98DE74F98FFF7B4F815F05DFCE0
:1035800008F1010606442C49304603F079FD074650
:1035900090B14F98FFF7A6F8284A03463146CDF878
:1035A0000090384615F09EFB39464F98FFF74AFCCD
:1035B0000121384603F068FD61234F9A21462846D1
:1035C000FFF7BAFCADE71E4807F018F91D4A21467F
:1035D0002846FFF77FFCC8E701214EE75DBA0108E6
:1035E0007FBA0108AFB90108C8B90108D4B9010808
:1035F00020B9010810BA010838BA01083EBA01081A
:103600005BBA0108FAB8010804B901080EB901084B
:1036100011B9010831B9010831A8010844B90108FC
:1036200047B9010861B901087AB901087DBA0108F2
:103630008BB9010890BA01084EEC0108E6B90108FF
:10364000EBB901080EBA01082DE9F0410C4680469D
:103650000D4815461E46069F07F0D0F804B14DB937
:103660000A4807F0CBF839463046BDE8F041084A31
:10367000FFF730BC069733462A4621464046BDE850
:10368000F041FFF78FBE00BFBCBA0108D1BA0108F4
:10369000E4BA01087FB504460D4600680C49164699
:1036A00000F000FB78B100F0D1FC03AB0093324690
:1036B000294602ABFFF7C8FFDDE902122046FFF7FB
:1036C00023FD04B070BD034807F098F8F9E700BF88
:1036D00056B901087AB8010810B10C2103F0D4BC26
:1036E000704710B1012103F0CFBC704730B51346CD
:1036F0000D460446AC4207D01BB194E8070083E8AE
:1037000007000C330C34F5E7184630BD10B50446FD
:1037100038B1FCF71BFD2046BDE81040282103F01E
:10372000B3BC10BD70B50446406AFFF7D5FFD4E9BD
:103730000656AE4204D02846FCF708FD2835F8E7C7
:10374000A06908B1FFF7E2FF204670BDF8B5054655
:1037500000242826074FD5E906031B1ADB107B43FC
:103760009C4205D206FB0400FFF7FCF90134F2E7A6
:10377000F8BD00BFCDCCCCCCF8B50446224807F04C
:103780003DF8224807F03AF8D4E90631994218D0BA
:10379000C91A1F4EC91071431E4807F02FF80025A3
:1037A0002827D4E906031B1ADB1073439D4205D278
:1037B00007FB0500FEF7A2FF0135F2E7164807F008
:1037C0001DF8D4E90931154EC91A891071431448FE
:1037D00007F014F800250C27D4E909031B1A9B10E5
:1037E00073439D4205D207FB050000F0FBFF013546
:1037F000F2E70C4807F002F80B4806F0FFFFBDE8BF
:10380000F8400A4806F0FABFB9BB01086AB20108DD
:10381000CDCCCCCCC3BB0108D5BB0108ABAAAAAAAE
:103820000EBC01087DBA01081EBC01086BB001087E
:103830002DE9F043002487B006466846CDE90044F0
:1038400002940CF0D5FB68460CF06AFC4FF0280897
:103850002F4F304DD6E906239B1ADB107B439C4249
:103860004ED208FB04F302EB0309D35C002B43D1D7
:103870004846FEF7EEFE014668460CF043FC48461B
:10388000FEF7E9FE042837D8DFE800F03803101A05
:1038900024004846FEF7E1FE014668460CF0E8FBCE
:1038A00050BBC2212846FEF727FE25E04846FEF71A
:1038B0000CFF014668460CF0C1FBE8B9C621F1E7F0
:1038C0004846FEF70FFF014668460CF01BFC98B90E
:1038D000CA21E7E7494603A8FEF7CDFEDDE903125A
:1038E0006846521A0CF0E6FB18B9CF212846FEF7BD
:1038F00003FE0398FFF7F5FE0134ABE7D321D1E7D0
:1039000068460CF035FC029807B0BDE8F08300BFB4
:10391000CDCCCCCC7EBA01082DE9F04305460E464D
:1039200000244FF028081A4F8DB0D5E906239B1AC2
:10393000DB107B439C4224D208FB04293146182229
:10394000684615F094FA4846FEF783FE18220146B1
:103950000DEB020015F08BFA684607F0BDF86846DB
:1039600007F0CCF806A807F0B7F806A807F0C6F8E5
:10397000182268460DEB020115F067FA18B1013400
:10398000D3E74FF0000948460DB0BDE8F08300BF13
:10399000CDCCCCCC2DE9F04F06460F4600244FF09D
:1039A0000C09DFF86C808DB0D6E909535B1B9B10C6
:1039B00008FB03F39C4224D218223946684615F0CE
:1039C00056FA182209FB04FB0DEB020055F80B1008
:1039D00015F04DFA684607F07FF8684607F08EF854
:1039E00006A807F079F806A807F088F818226846B4
:1039F0000DEB020105EB0B0A15F027FA18B10134A3
:103A0000D2E74FF0000A50460DB0BDE8F08F00BF7E
:103A1000ABAAAAAA10B51446FFF77EFF20B1214633
:103A2000BDE81040FFF70EBA10BD0000F8B50C4617
:103A3000064640F201120021224814F00AFA4FF41F
:103A4000807221461F4814F0E0F91E491E4806F016
:103A5000D5FE1E491B4815F039FA1C4905460020C1
:103A600015F034FA294607463046FFF755FFA0B94E
:103A700029463046FFF78EFF044600B3016814481C
:103A800006F0BCFEA3683846984701242046F8BDDE
:103A90003946104806F0B2FEF8E73A462946304665
:103AA000FFF7B8FF04460028F2D00B4806F0A6FE48
:103AB0000A4806F0A3FE3046FFF75EFEE6E7294619
:103AC0000748E7E7D80A002037BC010869B80108B1
:103AD0003DBC010866BC010852BC01087DBA010862
:103AE0007FBC010810B54FF48072044606490430CB
:103AF0000CF0C2FB002805DD2046BDE8104002495D
:103B0000FFF794BF10BD00BFD809002038B5144698
:103B10001D46FFF701FF28B12A462146BDE838407F
:103B2000FFF738B938BD10B51446FFF7F5FE20B1E0
:103B30002146BDE81040FFF78DB810BD10B5144602
:103B4000FFF7EAFE10B12146FEF798FF002010BDF6
:103B500038B514461D46FFF7DFFE28B12A46214638
:103B6000BDE83840FFF786B938BD00002DE9F047C1
:103B700000248CB0074603A8CDE9034405940CF05B
:103B800037FA214603A800940CF04EFB01460028AA
:103B900034D0214603A80CF0D0FA40F2E7330446B3
:103BA000009300263546DFF8F890009BB34273D9A6
:103BB000214603A80CF0F3FA824600286CD11823A2
:103BC00021460DEB030203A80CF07AFA04442146C7
:103BD00003A80CF0F2FA8046B0B10CAA214642F8D4
:103BE00028AD03A80CF00AFA029A044406A9384644
:103BF000FFF799FF00B101350136D6E76A4603A801
:103C00000CF0A2FA0446CCE7214603A80CF01FFBF7
:103C100070B10CAA02F8288D214603A80CF018FAFE
:103C20009DF80820044406A93846FFF787FFE1E71E
:103C3000214603A80CF0DCFA804668B102AB01AA69
:103C4000214603A80CF04DFADDE90123044406A93E
:103C50003846FFF75BFFCDE7214603A80CF0BAFA20
:103C600090B10CAB43F8288D01AA214603A8CDF8EA
:103C700004800CF00EFA9DF808300444019A06A95D
:103C80003846FFF765FFB5E7039B4846195D01F02D
:103C9000E00106F0B3FDAFE728460CB0BDE8F087C1
:103CA00048BB010808B5FFF737FE18B1BDE808406A
:103CB000FEF7D3BC08BD10B5044608461146FFF711
:103CC0002BFE014620B9C4E90000A060204610BDCB
:103CD0002046FEF7D0FCF9E708B5FFF71DFE18B146
:103CE000BDE80840FEF7F1BC08BD08B5FFF714FEBB
:103CF00018B1BDE80840FEF7F5BC08BD037810B563
:103D0000044643B1044806F079FD0021204600F046
:103D1000EFFA0023237010BD33BB01082DE9F041F9
:103D20000E469DF81840174698469DF81C50FFF720
:103D3000D3FF844205DCA84203DC88F80000BDE81C
:103D4000F081012322463B70314606902B46BDE8A8
:103D5000F041014806F052BD0BBB01082DE9F041CE
:103D60000E46BDF8184017469846BDF81C50FFF7A0
:103D7000B3FF844205DCA84203DCA8F80000BDE8DC
:103D8000F081012322463B70314606902B46BDE868
:103D9000F041014806F032BD0BBB010873B51C466B
:103DA0000E461546FFF7A1FF002302AA42F8043D84
:103DB0002060069906F008FB019B33B1226831466A
:103DC000034806F01BFD01232B7002B070BD00BF3D
:103DD000A2BC0108002370B5D1E90025AD1A044644
:103DE000C0E9003383600E46284601D006F0A2FDEC
:103DF000C4E900000544A560D6E9005302462946FF
:103E00008B4205D00AB10E78167001310132F7E706
:103E10005B1B18446060204670BD38B504460D46F3
:103E20000B78103000F8103C4B68103140F80C3C17
:103E300051F8083C40F8083C51F8043C40F8043C78
:103E4000FFF7C8FF05F11C0104F11C00FFF7C2FFDA
:103E5000204638BD2DE9F843D0E90054641B914653
:103E6000A2101F4C06465443B4F5A04F0F4602D192
:103E70001C4803F0C9F8002C14BF22460122A418E4
:103E8000A1EB050526D2B4F5A04F23D82CB30C2006
:103E9000604306F04FFD804618EB05031CBF99E810
:103EA000070083E80700424639463068FFF71EFCEA
:103EB000716800F10C023846FFF718FC05463068BF
:103EC000FFF70AFC0C2303FB0484C6E90085B460F9
:103ED000BDE8F8834FF4A044D9E7A046DCE700BF73
:103EE000ABAAAAAAA7B601082DE9F043054685B0FA
:103EF00008460C4617461E4614F09FFF172803D9A4
:103F000082212D48FEF7F8FACDE90147D5E9097875
:103F100003962A4AA8EB0706B41054430134B4F5BB
:103F2000A04F02D9264803F06FF8EB6ADB1B9B1009
:103F300053439C4215D94FF00C0909FB04F91CB1FD
:103F4000484606F0F7FC0446224641463846FFF74D
:103F5000CDFB686AFFF7C0FB26446C624C44AE623E
:103F6000EC62EA6AD5E9090314491B1A9B10121A7C
:103F70004B4392104A430133934206D9114806F04D
:103F80003DFC8C210C48FEF7B7FAD5E90A32934282
:103F90000AD023B104AA12E9070083E807000C3312
:103FA000AB6205B0BDE8F08301AA194605F1240013
:103FB000FFF750FFF5E700BF7EBA0108ABAAAAAA37
:103FC0006CB60108F0BA010838B50025034604466E
:103FD00003F8045B29461846142213F03AFF0A4AF4
:103FE000C4E906556261C4E90855C4E90A55C4E943
:103FF0000C5580210CF039F92046044B044A054940
:10400000FFF772FF204638BD5809002051400008D4
:10401000C5BC0108D1BC010810B5084C2368DB07FA
:1040200009D40748FFF7D0FF0123064A0649044890
:10403000236012F0C7F9024810BD00BF54090020E8
:10404000DC0B00200000002025370008FFF7E4BF4C
:1040500008B5FFF7E1FFBDE80840FFF78DBB002280
:10406000C0E90022826010B50C6804600A604268F2
:104070004C6844604A6082688C6884608A6010BDC5
:1040800070B50E4605461446B54217D09CB12B7844
:1040900005F1100123706B6804F110006360AB68D8
:1040A000A360EB68E360FFF7DAFF05F11C0104F1A0
:1040B0001C00FFF7D4FF28342835E5E7204670BD03
:1040C0002DE9F843D0E90064A41BE310234C054616
:1040D0005C43B4F5A04F0F46914602D1204802F050
:1040E00093FF002C14BF23460123E418A1EB06061E
:1040F00023D2B4F5A04F20D814B32820604306F093
:1041000019FC804618EB060002D04946FFF785FEF1
:10411000394642462868FFF7B3FF696800F1280274
:104120003846FFF7ADFFD5E900690746B14509D02C
:104130003046FCF70BF82836F8E74FF4A044DCE7EC
:10414000A046DFE7286808B1FFF7E0FA282303FB61
:104150000484C5E90087AC60BDE8F883CDCCCCCC45
:10416000A7B601082DE9F047D0E9065704460E46E8
:10417000DFF80C818AB0AF421BD029466846FFF7B2
:104180004CFE6846FEF765FA81463046FEF761FA56
:104190000146484606F0E1FC30B13046FEF759FAD8
:1041A0000146404606F02AFB6846FBF7CFFF28355C
:1041B000E1E7D4E906892E4AA9EB0807FD1055432B
:1041C0000135B5F5A04F02D92A4802F01DFF236A38
:1041D000A3EB0803DB1053439D4220D94FF0280A7C
:1041E0000AFB05FA1DB1504606F0A4FB05464946F8
:1041F00040462A46FFF744FFD4E90689C14505D069
:104200004046FBF7A3FF08F12808F7E7A06908B1CB
:10421000FFF77CFA2F44A5615544E7612562226AC5
:10422000D4E9060312491B1ADB10121A4B43D210B1
:104230004A430133934206D90F4806F0DFFA77214B
:104240000E48FEF759F9D4E90703984209D010B196
:104250003146FFF7E2FDE3692833E3610AB0BDE8C8
:10426000F0870146324604F11800FFF729FFF5E711
:10427000CDCCCCCC6CB601089ABB01087EBA010843
:1042800068BB0108002313B502A941F8043D094B9E
:104290000422D3E90140084B20445B689847044658
:1042A00028B1064806F0AAFA204602B010BD04481C
:1042B000F8E700BF2C0C0020180C0020DCBE010821
:1042C000F0BE010808B5084806F098FAFFF7A4FE0A
:1042D000FFF73CFA054806F091FAFFF79DFEBDE8AE
:1042E0000840FFF749BA00BF0DBF010825BF01080C
:1042F00073B505464FF416700C4606F01BFB0646D8
:1043000030B9214806F07AFA22212048FEF7F4F865
:104310004FF416720021304613F09BFD31462846BB
:104320004FF41672FFF784FA194D014601902CB331
:10433000184806F063FAD5E901431C44164DEB68B2
:104340001BB101992046083198476B680422104937
:104350002046984704226B680DEB0201A01898478D
:104360006B68019A314604F1080098470B4806F043
:1043700045FA304606F0C8FA02B070BD084806F0AB
:104380003DFA6C68DAE700BFB0D401087EBA0108D4
:104390002C0C0020CEBD0108180C002008BE01081E
:1043A000EDBD01082DE9F74FFFF736FE2F4F06460A
:1043B0002F4806F023FAB846DFF8D090DFF8D0A0F7
:1043C00009F0BEFC2B4D38602B68AB462A4C002B05
:1043D00037D003F56A436033984232D223782BB941
:1043E000264806F00BFA264806F008FA0123304664
:1043F0002370FFF777FB41F2883352464FF0FF31CD
:1044000000200AF071F9019009F09AFC019BC8F8AC
:10441000000023B9237813B13046FFF763FBDAF8C5
:104420000030DA0744BFD8F800202A609B07C7D5C0
:104430000023CBF80030D9F80830002BBED09847C5
:10444000BCE723786BB100213046FFF751FF0D48E0
:1044500006F0D4F90C4806F0D1F9D9F8083003B1C8
:104460009847002323702B60C5E700BF440C002051
:104470004CBE0108400C0020380C002061BE010831
:1044800084BE0108A7BE0108B9BE0108180C0020AF
:104490003C0C002010B5FFF7BFFD04460021FFF7DC
:1044A00027FF2046FFF768F9BDE8104003480023C6
:1044B0000122022100680AF061B900BF140C00203B
:1044C00010B5FFF7A9FD04460021FFF711FF2046B4
:1044D000BDE81040FFF750B92DE9F743194E0746E4
:1044E000884675680AB1B3681D440024DFF86090FF
:1044F00002A941F8084D0422D9F80030284698470F
:10450000326800998A4204D00F4806F077F92046B5
:1045100014E00422D9F800300DEB0201A8189847E6
:1045200001990A4806F06AF9019A4245EFD8D9F88C
:104530000030394605F108009847019803B0BDE8FE
:10454000F08300BF2C0C002017BE010832BE01080A
:10455000180C002084B0F0B585B00AAC84E80F00D8
:104560000B9B23B940F229117F48FDF7C5FF0A9B39
:1045700023B94FF495717C48FDF7BEFF7B4C0AAD23
:104580000FCD0FC42B682546794C0FAA07CA45F8F2
:10459000103984E8070012B94FF48063A3602368E0
:1045A00023B940F235117048FDF7A6FF23680133A7
:1045B00004D140F237116C48FDF79EFFFFF72CFD48
:1045C00006466C4B6C4A6D49FFF78EFC6C4B6D4A8E
:1045D0006D493046FFF788FC6C4B6D4A6D4930469B
:1045E000FFF782FC4FF4167006F0A4F9074680B975
:1045F000694806F003F9694806F000F93046FFF70C
:10460000A5F800233370FFF73DFE654806F0F6F885
:104610002CE04FF41672002113F01BFCD4E90103C7
:104620002D68042203A91844A847002861D02268F5
:10463000039B9A425DD15B4806F0E0F801224FF4FB
:1046400016713846FFF748FF0446574806F0D6F87B
:10465000FFF718FE002C48D001233370224639465C
:104660003046FFF783FA384606F04EF933783BBB05
:104670004FF4167006F05EF9044630B9464806F06D
:10468000BDF87F213848FDF737FF4FF4167200213F
:10469000204613F0DEFB00224FF416712046FFF790
:1046A0001BFF074690BB06F02FF9204606F02CF9B9
:1046B0003E4806F0A3F8FFF7AFFC0021FFF718FE15
:1046C0003B4BFA22019301233A4900933A480023D5
:1046D00009F0F4F820B94FF4A8712348FDF70CFF56
:1046E00005B0BDE8F04004B07047344806F086F8E5
:1046F000347000224FF416713846FFF7EDFE044681
:104700000028ABD1384606F0FFF874E74FF4167076
:1047100006F010F9054630B91F4806F06FF88E21F3
:104720001148FDF7E9FE4FF416720021284613F0F8
:1047300090FB4FF4167229463046FFF779F808B916
:104740002846B0E78742FBD10023E95CE25C914256
:10475000F6D101339F42F8D1284606F0D5F820461D
:1047600006F0D2F8ACE700BF7EBA0108180C0020B2
:104770002C0C0020C1440008D5BC0108E1BC010894
:10478000C5420008E6BC010801BD010895440008C7
:1047900009BD010821BD0108B0D4010888BD010888
:1047A00025BF010826BD01084ABD0108ACBD0108AE
:1047B000140C0020C3BD0108A54300085FBD01081B
:1047C00010B5064C226922B94FF4AA710448FDF7CE
:1047D00093FE2369BDE81040184700BF180C002065
:1047E0007EBA010810B504460168074806F006F8CD
:1047F000616831B10B7823B10448BDE8104005F081
:10480000FDBF0348F9E700BF3DBF01082AB7010813
:104810007DBA010810B50446C06908B106F074F805
:10482000206908B106F070F8606808B106F06CF80D
:10483000204610BD10B50446006808F05BFF204616
:1048400010BD00001FB50B46546801780294127821
:1048500001925A68009242681B68024805F0CEFF38
:1048600004B010BD42BF0108CB210148FDF744BE92
:104870007EBA0108FE2307B502A901F8043D054BE5
:104880001868002300681A4608F024FC03B05DF89D
:1048900004FB00BF540C0020D0B51F467423C0E9B0
:1048A00000310023044683600820164602F0CAFB4C
:1048B000C0E90067A0602046D0BD00002DE9D043CC
:1048C000DDE9066799467223C0E90031002396426C
:1048D000836077EB09030446904603DA2B210748EF
:1048E000FDF70AFE102002F0ADFBC0E90089C0E927
:1048F0000267A0602046BDE8D08300BF7EBA0108F1
:10490000036837B5632B04460D4601D0FFF7ACFFB3
:10491000002302AA42F8043DA168284605F054FD90
:10492000019B1BB138210248FDF7E6FD03B030BD05
:104930007EBA010870B563230025C0E90031044642
:1049400085601A20164602F07DFB1A22294613F0D4
:1049500080FA3146A0602046FFF7D2FF204670BDA6
:1049600081647047C16470472DE9F843D0E9017351
:10497000884600254FF00C09DB1B0A4E9B105E4356
:10498000ECB2B4420BD209FB04724146506814F0F9
:1049900042FA01350028F3D12046BDE8F8834FF0F4
:1049A000FF30FAE7ABAAAAAA2DE9F843D0E90473CD
:1049B000884600254FF00C09DB1B0A4E9B105E4316
:1049C000ECB2B4420BD209FB04724146506814F0B9
:1049D00022FA01350028F3D12046BDE8F8834FF0D4
:1049E000FF30FAE7ABAAAAAA2DE9F0410E464968C2
:1049F0000446FFF7B9FFC0B2FF2803D07C21294845
:104A0000FDF77AFDD4E90123274F9B1A9B107B43C6
:104A10007E2B03D97F212348FDF76EFDD4E90112D7
:104A20000C25E068531A9B10121A7B4392107A43AC
:104A30000133934205FB03F80ED84144A160D4E949
:104A4000013496E80700E31A04E9070016489B10B2
:104A500058430138BDE8F081404605F06BFF05463C
:104A600018B969210F48FDF747FDD4E901C30027B4
:104A7000A3EB0C039A100C4B5343002B09DD05EB01
:104A8000070E0CEB070207CA013B8EE807000C3744
:104A9000F3E7604605F038FF65604544C4E9025518
:104AA000CDE700BF7EBA0108ABAAAAAA1FB56E2344
:104AB000CDE90131002301A90393FFF795FF05B06C
:104AC0005DF804FBFF2270B5002380F828204FF02A
:104AD00000424FF0FF31C0E90D23C2636FF07F4207
:104AE000C0E910120522C0E90033C0E91423C0E96F
:104AF00002330022C0E90433C0E90633C0E90833B9
:104B00000363C0E9123383654FF000431E4DC0E9D3
:104B100018232A68044612F0010213D101211B4E0A
:104B200008463260716008F0FBF9306018B9512115
:104B30001748FDF7E1FC0123164A174913482B607B
:104B400011F040FC154B1A680AB9104A1A60144952
:104B50002046FFF7ABFF134B134918702046FFF7B1
:104B6000A5FF124B124918702046FFF79FFF114B0B
:104B7000114918702046FFF799FFFE220F4B18705D
:104B80000F4B20461A7070BD500C0020D80C00202E
:104B90007EBA01080000002035480008540C0020AF
:104BA000AEC001085C0C0020B6C001085A0C002001
:104BB000BEC00108580C0020C3C001085B0C0020D7
:104BC000590C002010B5084C2368DB0709D40748AE
:104BD000FFF778FF0123064A06490448236011F0D5
:104BE000F1FB024810BD00BF4C0C0020700C0020EF
:104BF00000000020154800082DE9F0410E464968E4
:104C00000446FFF7D1FEC0B2FF2803D08721294810
:104C1000FDF772FCD4E90423274F9B1A9B107B43BA
:104C20007E2B03D98A212348FDF766FCD4E90412C0
:104C30000C25A069531A9B10121A7B4392107A43D9
:104C40000133934205FB03F80ED841446161D4E976
:104C5000043496E80700E31A04E9070016489B109D
:104C600058430138BDE8F081404605F063FE054633
:104C700018B969210F48FDF73FFCD4E904C30027A8
:104C8000A3EB0C039A100C4B5343002B09DD05EBEF
:104C9000070E0CEB070207CA013B8EE807000C3732
:104CA000F3E7604605F030FE25614544C4E905554B
:104CB000CDE700BF7EBA0108ABAAAAAA38B5D0E9F1
:104CC00001239B1A074A9B105343CDB29D420446D1
:104CD00003D3A6210448FDF70FFC0C20636800FBFA
:104CE000053038BDABAAAAAA7EBA010838B5CCB245
:104CF000114905460B6813F0010307D10F4A7020D4
:104D00001372012310600E480B605060FF2C10D00E
:104D1000D5E904239B1A0B4A9B1053439C4203D3AF
:104D2000B2210948FDF7E8FB0C23286903FB0400C6
:104D300038BD0248FCE700BF480C0020600C002092
:104D400060BF0108ABAAAAAA7EBA010810B5D0E9D3
:104D50000730C9B2D2B2834209D01C788C4204D148
:104D60005C78944201D1987810BD0333F3E74FF09B
:104D7000FF30F9E72DE9F041D0E904239B1A4F4AAF
:104D80009B1053430D4609780446994203D393215F
:104D90004B48FDF7B1FBD4E901239B1A474A9B100E
:104DA00053436978994203D394214548FDF7A4FB06
:104DB000D4E904239B1A414A9B105343A978994292
:104DC00005D3FE2903D095213D48FDF795FB6A7870
:104DD00029782046FFF7BAFFC3B2FF2B064629D039
:104DE00029782046FFF782FF697807462046FFF7BB
:104DF00065FF314680462046FFF778FF4146024670
:104E00003846FFF71FFD29782046FFF76FFF6978C6
:104E100006462046FFF752FFA97807462046FFF7CF
:104E200065FF394602463046FFF70CFD9C212448B9
:104E3000FDF762FBD4E90723204F9B1A7B437E2BAF
:104E400003D99F211E48FDF757FBD4E90762616A29
:104E5000931B7B43521A57430133BB4203EB430876
:104E60000AD8464426622A88236A23F8032CAA78A3
:104E700003F8012CBDE8F081404605F05BFD0646D5
:104E800018B969210E48FDF737FBD4E90702131A58
:104E90000A4A5A430023002A0ADDC118B1F800C0AB
:104EA000F71826F803C08978013AB9700333F2E79E
:104EB00005F02AFDE66146446662D3E7ABAAAAAADA
:104EC0007EBA0108FF2337B58DF804300A4B0D4632
:104ED0001C6823681BB929210848FDF70DFB2A46E9
:104EE00001A9206808F09AF9012814BF4FF0FF309B
:104EF0009DF8040003B030BD540C00207EBA0108B8
:104F000038B5816800681D46144605F0C5FD0346A6
:104F1000201845EBE37138BD08682DE9F04172288F
:104F20001F461FD074280FD0632820D1886805F051
:104F30000BFB002871F1000304460D460EDADD215B
:104F40000D48FDF7D9FA09E08B68D3E90045B5F1C2
:104F5000004F08BF002C01D0A4187D4120462946EF
:104F6000BDE8F0818868BDE8F041FFF7C9BF0024C3
:104F70004FF00045F2E700BF7EBA01082DE9F0418D
:104F80000F4606460024FFB2FFF7B0FED6E90758E9
:104F9000454511D02B78BB420CD169783046FFF7DC
:104FA0008DFE0368692B05D183681B6803B19847A0
:104FB0000134E4B20335EBE72046BDE8F0812DE98A
:104FC000F34180460F460025FFF790FED8F81C40BD
:104FD000D8F8206003340336FFB2A6421BD0234624
:104FE00033F8032D9B78ADF804208DF8063014F8C3
:104FF000033C9F420DD19DF805104046FFF75EFE31
:105000000368692B05D183685B6803B19847013554
:10501000EDB20334E1E7284602B0BDE8F0810000BC
:10502000836C73B504460D46164623B94FF48E7152
:105030000B48FDF761FACDE9006423462A46094989
:10504000094808F03BFC012807D04FF4917104484F
:1050500002B0BDE87040FDF74FBA02B070BD00BFAE
:105060007EBA010890C00108A956000838B590F82A
:1050700047300446032B0D4604D940F2351106484B
:10508000FDF73AFA94F847305A1C84F847201C443C
:1050900084F8425038BD00BF7EBA010810B590F8C0
:1050A0004730044623B94FF49D710648FDF724FAB2
:1050B00094F84730013BDBB284F847301C4494F845
:1050C000420010BD7EBA0108CBB2FE2B10B50446DB
:1050D0000AD0FFF70BFE03686D2B05D1017A20463D
:1050E000BDE81040FFF702BE10BD00002DE9F843F7
:1050F00004460026114FD4E904239B1A9B107B43DE
:105100005FFA86F8434516D941462046FFF7DCFF93
:10511000D4E90759A9450CD02B78434507D16978C4
:105120002046FFF7CBFDA9782046FFF7CDFF0335DA
:10513000F0E70136DFE7BDE8F88300BFABAAAAAA13
:1051400038B50546002495F84730A34207DD2B19F2
:1051500093F842102846FFF7C9FD0134F3E738BD44
:1051600000232DE9F74FC0E9083388461946D8E9EE
:1051700007594FF000430446C0E90613C0E9001385
:10518000C0E90213C0E90413FF208A469B46D2B24D
:1051900084F8200001924D45D4E9006720D02B7897
:1051A000019A93421AD169784046FFF787FDDDE9FD
:1051B0000C2301464046FFF7AFFE594508BF504556
:1051C0000CD05F4508BF564503D0B04271EB0703D2
:1051D00004DA6B78C4E9000184F820300335DAE79B
:1051E000B7F1004F08BF002E08D0DDE90C23B21A3A
:1051F00067EB030316461F46C4E90467204603B065
:10520000BDE8F08FF8B50D460B4B896906464B4358
:105210004FF47A71B3FBF1F1FFF754FE0446C7B2C5
:10522000B06C03681B689847FF2FC6E90E010CBFDE
:1052300095F820002046F8BD40420F0038B5C36CF9
:1052400004460D461BB9BDE83840FFF7DBBF806C54
:10525000174903685B699847A06C0368DB68984747
:10526000D5E9020105F04AFA0146124805F0C6FAEE
:10527000A06C03689968D5E902238847A06C03688D
:105280001B699847E36C9847A06C0368DB689847F4
:10529000A06C03681B689847C4E90E0100212046F2
:1052A000FFF710FEC0B2FE2808BF95F8200038BDF9
:1052B000754800089BC00108F8B5D1E90667B7F149
:1052C000004F08BF002E05460C4608D11AB1BDE8B4
:1052D000F840FFF797BFBDE8F840FFF7AFBF012EDA
:1052E00077F1000302DA91F82000F8BD92B121466F
:1052F0002846FFF787FF94F82030C0B28342F4D1EC
:10530000D5E90E67D4E90023964277EB0303B8BFD3
:10531000FF20EAE7D0E91423964277EB0303E6DBAC
:10532000FFF78CFFE7E700002DE9F04F8DB0044652
:105330000D46FFF7DBFC03688046702B04D04FF46A
:10534000A0716B48FDF7D8F8A06C03681B689847FC
:105350002A46C4E90C01CDE90001214602A8FFF765
:10536000FFFE29462046FFF709FE9DF82830064635
:10537000FF2B05D120B940F24B115D48FDF7BCF879
:10538000D4E90C0105F0BAF901465A4805F036FA9D
:105390003146594805F032FA9DF82810FF297ED190
:1053A00000224FF00043CDE90623DDE90223CDE9D9
:1053B0000423DDE90623CDE90823A36D13B3984741
:1053C000DDE90223D4E91801B3F1004F08BF002A38
:1053D00009D0DDE9062310F10B0641F100079642E2
:1053E00077EB03030EDAD4E90C23161843EB01071D
:1053F000CDE90801CDE9046705F096F901463F487B
:1054000005F0FCF94FF0000A4FF0004BDFF8F89080
:1054100098F8082002A92046FFF74EFFA36D064624
:1054200003B19847F3B2FF2B5AD1DDE90223D4E947
:105430000E01161A63EB010739463046CDE9042305
:10544000CDE90667CDE9086705F06EF901464846E3
:1054500005F0D4F9A36D002BDAD0DDE90223D4E9FD
:1054600018015B4508BF524509D0DDE9062310F15C
:105470000B0641F10007964277EB0303C8DAD4E943
:105480000E23161843EB0107CDE90801CDE90467A7
:1054900005F04AF90146194805F0B0F9B8E7204689
:1054A000FFF70CFCD0E90067DDE9020105F026F901
:1054B0003A4603463146124805F0A0F9D4E90C23D8
:1054C000DDE90201801A61EB03010F460646CDE9D2
:1054D000066705F029F901460A4805F08FF964E7E7
:1054E00029462046FFF76BFD30460DB0BDE8F08F32
:1054F0007EBA01086EBF01088DBF0108EABF01082E
:10550000A8BF0108CCBF010802C0010870B504465D
:105510000D46FFF7EBFB03686D2B11D0702B09D004
:10552000612B14D1836894F8411094F84000BDE8D1
:105530007040184729462046BDE87040FFF7F4BE8A
:10554000034840F22F11FCF7D7FF4FF0FF3070BD3A
:105550007EBA01082DE9F04790F828300446FF2B69
:1055600004D14FF4E5714A48FCF7C6FF94F82810BF
:105570002046FFF7BBFB42680178464805F03EF93C
:1055800094F82830DFF81C8184F8463094F84610EF
:105590002046FFF7ABFB036805466D2B204694F8C9
:1055A00046100BD1FFF762FD297A204684F8461099
:1055B000FFF79CFB2046FFF7C3FDE7E7FFF7A6FFD9
:1055C000C3B2FF2B06460BD140F2DF113048FCF787
:1055D00093FF40F2DF11304B304A314812F0F8F9B6
:1055E000024694F846102046FFF7B0FBC5B2FF2DE7
:1055F00009D140F2E5112648FCF77EFF264B274AE9
:1056000040F2E511E9E794F84610FE2D204621D13D
:10561000FFF744FD074601462046FFF767FB324689
:1056200039462046FFF792FBC5B2FF2D0DD131461A
:105630002046FFF743FB40F2F1111548FCF75CFFF1
:10564000154B164A40F2F111C7E72046FFF778FDE7
:105650003946DAE7FFF74AFB314607462046FFF7AF
:105660002DFB294681462046FFF740FB82464046F7
:1056700005F0C4F8524649463846FFF7E3F894F877
:10568000463084F8416084F8403084F846507DE725
:105690007EBA01082AC00108EEB60108CBC0010895
:1056A00048C0010880C0010808B505F00DFAFFF7F1
:1056B00089FAFFF74FFFD0B51F461646FFF7FEFAEF
:1056C00003688468742B01D0FFF7CEF8C4E9006743
:1056D000D0BD0000836C10B5044623B94FF4277188
:1056E0000248FCF709FFA06C10BD00BF7EBA01089C
:1056F000FF23054A1370054A1370054A1370054AC3
:105700001370054A137070475C0C00205A0C00207F
:10571000580C00205B0C0020590C0020014B18781D
:10572000704700BF580C002010B50446006807F011
:10573000E1FF204610BD00002DE9F3480BF0B8FA58
:105740004FF6FF71344A13888B421CBF013313801C
:10575000FFF738FAFFF7BEFF03681B6898472F4B27
:1057600083465A788C46D2B92D4A1289BAB12D4C4B
:1057700030CCB5F1004F08BF002C0ED0844275EB41
:105780000C010CDABBEB0406274C6CEB0507544309
:10579000E517A64277EB050201DB01225A700022D1
:1057A000ADF804208DF806205A782AB101228DF830
:1057B00004201C4AC2E900BC1A781C4B92B1012299
:1057C0008DF805201A701A4A1A491B48019B127855
:1057D000097800680BF0FAFAD8B1184B187802B0C3
:1057E000BDE8F0881A700E4B9B89002BEBD04AF66F
:1057F000C0025A43124CD31730CCBBEB04006CEB05
:105800000501904271EB0303A4BF01238DF805301D
:10581000D9E70C4BE2E700BF240D0020000D00206B
:105820000C0D0020B800002080510100090D00205F
:10583000030D0020020D0020FC0C0020580C00205D
:10584000A80000205A0C0020104B1B8913B9104BE4
:10585000187870470F4BD3E90023B3F1004F08BF0E
:10586000002AF4D10C4A13780133DBB2012B1370F8
:10587000EDD80023094A1370094A1370094A1360CE
:10588000094A137001235370084BE1E70C0D002007
:10589000580C0020B0000020380D0020030D00201F
:1058A000020D0020FC0C0020000D00205B0C0020ED
:1058B0001FB57023CDE90131002301A98DF80C300B
:1058C000FFF79AF905B05DF804FB00002DE9F04FF1
:1058D0004A4B85B01A780446002A40F08B80012795
:1058E00047491F70FFF7E2F8464B474918702046BA
:1058F000FFF7DCF8DFF868A144498AF80000204689
:10590000FFF7D4F8DFF85C910A22002389F8000041
:105910003F4901A8FEF7C0FF01A92046FFF764F840
:105920003C4E3D4930702046FFF7C0F83B4B3C49A8
:1059300018702046FFF7BAF83A4B3B4918702046DA
:10594000FFF7B4F8394B3A4918702046FFF7AEF824
:10595000384B394A187039492046FBF76BFADFF8A3
:1059600008B1374A8BF8000036492046FBF762FA47
:10597000354905462046FFF79BFF70230193334BC3
:10598000804601A9204602938DF80C70FFF734F988
:1059900007462F4A2B4612789BF800102046FAF74C
:1059A000F1FD43469AF8002029462046FAF7EAFD21
:1059B0003B4699F8002029462046FAF7E3FD2B469E
:1059C000327841462046FAF7DDFD2B4632783946DB
:1059D0002046FAF7D7FD1F4A2B4612782946204663
:1059E000FAF7D0FD1C4B1D4A1B7812782946204639
:1059F000FAF7C8FD05B0BDE8F08F00BF390D0020F3
:105A000043C10108040D00204DC1010858C101081F
:105A100064C10108E90C002071C10108220D0020B9
:105A20007FC10108210D00208BC10108260D002037
:105A300098C10108270D002039570008A6C10108A8
:105A400075680008B0C10108C4C10108D7C10108C8
:105A5000580C00205B0C0020590C00205C0C00202E
:105A6000080D0020E80C0020060D002008B50BF002
:105A7000FDF818B1BDE808400BF01AB908BD08B52B
:105A80000BF0F4F818B9BDE808400BF0CBB808BD2E
:105A900030B5044685B00D46FFF718FF6D22064B62
:105AA00001A91B782046CDE901258DF80C30FFF7C0
:105AB000A3F805B030BD00BF060D00202DE9F84F5A
:105AC000424B434D1A68044612F0010F01BFFF22FA
:105AD0002A7001221A602B78FF2B73D1FFF7F6FE94
:105AE0003C4A3D492046FBF7A5F93C4A28703C4911
:105AF0002046FBF79FF93B4F3B4A38703B49204615
:105B0000FBF798F93A4E3B4930702046FFF7C0FF4B
:105B1000394982462046FFF7CBFE38498346204666
:105B2000FFF7C6FE8146364A3B7812782978204630
:105B3000FAF728FD334ADFF8E080337812782978C5
:105B40002046FAF71FFD337898F800203978204670
:105B5000FAF718FD2B7898F8002031782046FAF7EC
:105B600011FD294A5B46127839782046FAF70AFD7A
:105B700026493B780A7820465946FAF703FD244A1D
:105B80004B46127839782046FAF7FCFC1F493B78DF
:105B90000A7820464946FAF7F5FC1A4A5346127825
:105BA00031782046FAF7EEFC337898F80020514619
:105BB0002046FAF7E7FC174A2B781278317820460E
:105BC000FAF7E0FC2878BDE8F88F00BFE40C00206D
:105BD0003B0D0020CD62000842C20108D95E0008DA
:105BE0004CC20108050D00204958000856C20108A2
:105BF000070D002060C201086CC201087AC20108CA
:105C0000040D00205B0C0020080D0020E90C002092
:105C10005A0C0020580C00205C0C002038B50446BB
:105C20000D46FFF753FE034A29462046FBF702F9CB
:105C300038BD00BFD5600008344B2DE9F04F5A89BC
:105C40000023044689B0CDE90023039100230022FC
:105C50002F4905A8FEF732FE05A92046FEF7C4FE2F
:105C60002C4982462046FFF723FE2B4983462046D7
:105C7000FFF7D4FF294A804629492046FBF7DAF886
:105C8000284A054628492046FBF7D4F80646274F00
:105C9000DFF8A8903B7899F8002029462046FAF7CB
:105CA00071FC234A5B46294620461278FAF76AFCC3
:105CB000204A4346294620461278FAF763FC3346C9
:105CC000524659462046FAF75DFC33465246414655
:105CD0002046FAF757FC184A3B784146204612788E
:105CE000FAF750FC3B7899F8002031462046FAF745
:105CF00049FC6D230593039B05A9204606938DF867
:105D00001C50FEF779FF09B0BDE8F08F0C0D0020A4
:105D100089C2010896C20108A6C20108D963000819
:105D2000B7C201081D570008C6C20108590C00205F
:105D3000260D0020270D0020220D0020580C0020E9
:105D40002DE9F04F044687B008460E4615469A46A0
:105D500013F073F800F106090746484601F08EF982
:105D60004946334607F107092F4A804612F0BAFF29
:105D7000484601F083F90837494633462B4A8346A3
:105D800012F0B0FF384601F079F933463946284A17
:105D9000814612F0A7FF274A41462046FBF74AF802
:105DA000594680462046FFF783FD494683462046F4
:105DB000FFF734FF8146204A5B4612784146204671
:105DC000FAF7E0FB1D4A4B46127841462046FAF7A7
:105DD000D9FB1B4F1B4A3B78127849462046013DB0
:105DE000FAF7D0FB05EB0A030193019B9D420ED00D
:105DF00015F801AF3B78524659462046FAF7C2FBE8
:105E00003B78524649462046FAF7BCFBEDE76D2346
:105E100003A92046CDE903368DF81480FEF7ECFE89
:105E200007B0BDE8F08F00BF27C201082FC20108EC
:105E300038C20108FD630008260D0020270D002050
:105E4000590C0020220D00202DE970484FF000452C
:105E50000024164E83468C46D6E90001A94208BFAD
:105E6000A04205D010EB0B0241EB0C03C6E9002366
:105E70000F4ED6E90001A94208BFA04205D010EBA1
:105E80000B0241EB0C03C6E900230A4BD3E90045A2
:105E9000B5F1004F08BF002C05D01BEB04004CEB04
:105EA0000501C3E90001BDE8708800BFB000002013
:105EB000B8000020A800002070B50D460446FEF78B
:105EC00081FE044922462B46BDE870400978FFF761
:105ED000F2BB00BFE90C0020F8B5454D2B682F46FA
:105EE00001332B600AF0E4FE0AF01CFF44F6206048
:105EF0000AF0F4FE41780646042908D03D4804F033
:105F00007DFC304604F000FD0120002147E00478CC
:105F1000466804F0F9FC012C4AD12B68042B0CD9FB
:105F2000FEF794F8037843B1334B9B6803B198476D
:105F300040F29B113148FCF7DFFA3B681E22013B1F
:105F4000DBB21E2B28BF1E23A3F12005C3F12004C2
:105F500002FA05F122FA04F4002521434FF4E1444A
:105F600002FA03F08D4208BF84421CD3002908BF07
:105F7000B0F5616F04460D4615D2B0F5167F71F18C
:105F8000000313DA3C2871F10003ACBF11460A216B
:105F9000002004F081FD0346201845EBE371FFF774
:105FA0008BFF174B0BE04FF41671F1E73C21EFE745
:105FB000032C06D130460021FFF77EFF114B1878E5
:105FC000F8BD74B92C600AF02DFEFEF7FBFDFFF75B
:105FD00081FB03681B6898470B4BC3E900010B4B1F
:105FE000EDE70B48214604F009FC0A208DE700BFCD
:105FF000340D0020F0C001083C0D00207EBA0108DD
:106000005A0C0020080D0020A80000205C0C002085
:1060100011C10108054B1870054B1A700022054B81
:106020001960054B1A705A70704700BF030D0020AD
:10603000020D0020FC0C0020000D002002790168F8
:106040004079FFF7E7BF00000122014B1A7070474B
:10605000200D002008B50AF073FFC0B2DE2828BF6B
:10606000DE2008BD002337B54FF47A7401930B4B43
:1060700060431D68B0FBF4F42B681BB92921084864
:10608000FCF73AFA224601A9286807F0C7F8012868
:1060900014BF0020019803B030BD00BFEC0C0020FD
:1060A0007EBA01084FF47A7337B5002403FB00F27F
:1060B000074802A9056841F8044DB2FBF3F22868CD
:1060C00007F0EEF9012814BF2046019803B030BD57
:1060D000EC0C00202DE9F04F99B0FEF773FD90F81D
:1060E0004630044603930026FFF7C0FC4FF000093A
:1060F000214DDFF89080A06C0EAF03681B689847B5
:106100009DF80C20CDE9000121460EA8FFF728F8E4
:106110000FCFDDE912AB0DF1100CACE80F000FCF83
:10612000ACE80F003B688CF80030DDE90E23B3F1DA
:10613000004F08BF002A03D0D04579EB0B0313DAD8
:10614000AA46B34601274FF47A73AAFB030103FB67
:106150000B11FFF7A7FF48B10122084B5A72084BF9
:10616000187819B0BDE8F08F0027ECE7002FC2D1F6
:106170009DF83000F5E700BF80510100F00C0020D1
:10618000220D00208551010010B500200021FFF7ED
:1061900089FF10B1084B187810BD084C2368984748
:1061A00020B9074B1B780BB9064BF4E7637A0BB1A8
:1061B000054BF0E7054BEEE7220D0020F00C002028
:1061C000280D0020580C00205C0C00205B0C0020E7
:1061D000022818BF00200AF0ABBF00002DE9FF41E4
:1061E0002E4B05461F78002F55D1012204AE06F82C
:1061F000017D1A700AF0DEF907230C22284CCDE944
:10620000003228493246231D2846FDF787FD0E231C
:1062100063710D2324492846A3714FF47A782761CE
:10622000FDF740FD04F10803607032461F4928461F
:10623000CDE90078FDF792FD42F210733246CDE9C8
:1062400000731B4904F10A032846FDF787FD19492D
:106250002846FDF727FD04F10C03A07032461649CD
:106260002846CDE90078FDF779FD14492846FDF769
:1062700019FD9DF80F30E07053B1114804F0BEFADB
:10628000104B1B6803B1984760210F48FCF734F9A5
:106290002069FFF79DFF04B0BDE8F0813A0D0020B2
:1062A0000C0D0020EBC10108EEC10108F2C101088C
:1062B000FBC1010856B9010804C201080FC2010858
:1062C00014C201083C0D00207EBA010870B5294BAC
:1062D000C0B21B78984206D1FDF7B8FEFDF70EFD5F
:1062E000254B187870BD254CFDF7B0FEFFF776FF03
:1062F00094F905000CF0BEFC0AF036FE20790CF093
:1063000087FC0AF027FE1E4DA0790AF035FE607862
:106310000AF008FF2A6812F0010213D10421194E75
:1063200008463260716006F0FBFD306018B95121FB
:106330001548FCF7E1F80123144A154911482B6070
:1063400010F040F8134B1A680AB90E4A1A60FEF7AB
:1063500039FCFFF7BFF903681B68984701220E4B11
:10636000C3E900010D4B5A72E3780BB10C4BB8E74F
:106370000C4BB6E7070D00205C0C00200C0D002034
:10638000E00C00202C0D00207EBA01080000002047
:1063900029570008EC0C0020A8000020F00C002079
:1063A000040D00205B0C0020034B93F82F30022BD0
:1063B0000CBF0220002070474801002008B5FFF7FD
:1063C000F3FF02280CBF024B024B187808BD00BF38
:1063D000270D0020260D0020054B5B8913B9054BC6
:1063E00018787047044B5B7A002BF8D1FFF7E6BFB3
:1063F0000C0D0020580C0020F00C0020FFF7DEBF31
:1064000001232DE9F348404C6372404B1B785BB18C
:106410000AF004FB40B93E4BDB6803B1984740F2F9
:106420003F313C48FCF768F800200021FFF73AFEB6
:1064300010B1394B187813E02368984798B10AF0E7
:106440008DFF012871F1000306460F4637DBFEF78A
:10645000B9FB32463B46217AFFF72DF9FFF7AEFF35
:1064600002B0BDE8F0882D4B1B78002BE7D10AF075
:10647000D5FA0028E3D12A4DAB89E3B1FEF7A2FBA0
:10648000FFF728F903681B689847AB89254A264D12
:106490005A43D5E90067861B61EB0707D317B24261
:1064A000BB4108DA1A4B5B6803B198474FF45B7144
:1064B0001848FCF721F8002363721C4BBAE72368E5
:1064C000984770B1002364680093ADF80430FFF77B
:1064D000C1FD01466846A0476846FFF7AFFD144B73
:1064E000A8E70E4B1B784BB1124B1B88022BE4D84C
:1064F000002211461046FFF78DFDF0E70AF08EFAF4
:106500000028F1D1B7E700BFF00C0020200D0020DB
:106510003C0D00207EBA0108220D0020280D00202D
:106520000C0D002080510100A8000020580C002014
:10653000210D0020240D00202DE9F04F0446574D79
:1065400087B0C5E90023019100230A22544903A81A
:10655000FEF7A2F903A92046FEF746FA514A814602
:10656000287251492046FAF765FC504A05465049C1
:106570002046FAF75FFC4F4907462046FFF788FAA6
:106580004D498DF802002046FFF792F94B498DF8EE
:1065900003002046FFF742FB494982462046FFF7A9
:1065A0004BFB8346474EDFF83881337898F800205C
:1065B00039462046F9F7E6FF434A33783946204604
:1065C0001278F9F7DFFF414A5B46394620461278D8
:1065D000F9F7D8FF3E492B460A7820463946F9F7A5
:1065E000D1FF394A2B46594620461278F9F7CAFF9F
:1065F000337898F8002059462046F9F7C3FF3378DE
:1066000098F8002029462046F9F7BCFF2E4A337837
:10661000294620461278F9F7B5FF2E4A9DF8023038
:10662000294620461278F9F7ADFF29492B460A780A
:1066300020469DF80210F9F7A5FF274A9DF8033080
:10664000294620461278F9F79DFF2B464A469DF8C9
:1066500003102046F9F796FF204A53462946204664
:106660001278F9F78FFF2B464A4651462046F9F734
:1066700089FF337898F8002051462046F9F782FFC9
:106680006D230393019B03A9204604938DF8147096
:10669000FEF7B2FA07B0BDE8F08F00BFF00C0020A3
:1066A000D5C2010801640008E5C20108896100083B
:1066B000F3C2010800C301084DC1010858C1010817
:1066C0000CC30108590C0020580C00205B0C002062
:1066D0005C0C0020210D0020260D0020270D00203D
:1066E000220D002010B50FC8014C84E80F0010BD2A
:1066F0003C0D0020F8B51D4600234171BDF818106F
:1067000004460360C180174602B115B923712046C3
:10671000F8BD0749284600F0B3FC064610B92071C1
:106720002660F4E72A46394611F06FFB2571F7E73A
:106730004EEC010810B50446006808B100F0A2FC58
:10674000204610BD2DE9FF4142F210700AF0C6FA52
:106750000546002875D00778032F03D14068002133
:10676000FFF7AAFB384ED5F8A040336823B940F2B2
:10677000C9113648FBF7C0FE002C56D00022344B1E
:106780001A80D4E91C23134318D0324BD3F800806D
:1067900007F0D6FA01463048C047FEF713FAFEF775
:1067A00099FF03685968D4E91C238847D4E91C235E
:1067B0002A49C1E900232A49C1E90023FEF702FA68
:1067C000FEF788FF03681B689847264B264AC3E9F3
:1067D0000001237AC3F3C0031370637F2BB3237FBD
:1067E0001BB32249082000F03FFC804630B162898B
:1067F000237F617F0092A26EFFF77CFFCDF80C80B3
:10680000B8F1000F11D0002330681A4603A90068C0
:1068100006F0AAFB012808D0039C34B12046FFF7FC
:1068200089FF0821204600F02FFC2B7A13B10022AB
:106830000F4B1A7028460BF0DDFF384604B0BDE858
:10684000F0810127F9E700BFEC0C00207EBA0108B7
:10685000240D00204801002036C10108B0000020AE
:10686000B8000020A8000020280D00204EEC0108F0
:10687000090D0020002310B5114C84F834300AF0C3
:10688000F5F908B10AF014FAFFF75CFF012809D9FD
:1068900003280AD00B484FF43171FBF72DFE4FF05F
:1068A000FF3001E0084B187810BDFFF77DFD02288E
:1068B00009BF0123054B84F83430054BF3E700BFD3
:1068C000480100207EBA01085C0C0020080D002061
:1068D000E80C0020FF2300210D4A13700D4A1370AD
:1068E0000D4A13700D4A13700D4A13700D4A137040
:1068F0000D4A13700D4A13700D4A13700D4A137030
:106900000D4A13700D4AC2E900111372704700BF9F
:10691000060D0020050D0020070D0020220D00208F
:10692000210D0020270D0020260D0020040D002041
:10693000080D0020E80C0020E90C0020F00C0020DD
:1069400010B1012100F0A0BB704710B50446006BE8
:10695000FFF7F6FF606A10B1042100F095FBA06913
:1069600010B1042100F090FB204610BD7FB500243B
:106970000E4601A82146CDE9014403940EF00AFE1B
:10698000051E04DA29460F4803F038FF0EE001A97E
:1069900030460EF069FC08B1F36953B929460A483C
:1069A00003F02CFF28460EF0CBFD0024204604B057
:1069B00070BD28460EF0C4FD04460028F6D12946D5
:1069C0000248E1E7F4C401081BC5010851C50108EC
:1069D000F8B506460F460024094D39463046FFF704
:1069E000C5FF50B90134E4B20F2CF6D90EF088FB84
:1069F00031212846FBF780FDEFE70120F8BD00BFFD
:106A00007EBA01082DE970430646406988B00368E4
:106A10000C461B6898471C228046894601A8002125
:106A200011F017FAE3886079ADF818300FF092FB97
:106A3000B8F1010F8DF81D0079F100032079A8BF8E
:106A4000CDF8088003F076FF054628B32279216847
:106A500011F0DBF960790FF085FB41288DF81E00FD
:106A600005D042281BD0114803F0C8FE11E021795F
:106A700028460EF01DF904460246294606F1180084
:106A80000DF0E8FC80B1002301AA214628460EF053
:106A900031FC284603F038FF08B0BDE87083217947
:106AA00028460EF020F9E6E70148DDE7B9C4010801
:106AB000D7C4010882B073B50D46164600211022D6
:106AC0000446079311F0C5F900216561217428225D
:106AD00004F118000E4D11F0BCF904F140030BAAAB
:106AE00007CA83E807002A781AB968210948FBF722
:106AF00003FD00232B700A9B3046009307AB0ECB9F
:106B00000EF01AFB204602B0BDE8704002B070479C
:106B1000C00000207EBA010882B070B5144C86B067
:106B20000E460AA981E80C0023680546DB0716D447
:106B300003AB0EAA07CA83E807000BAB93E8070074
:106B40000A9B8DE80700324629460A48FFF7B2FF44
:106B50000123094A0949074823600FF033FC05481F
:106B6000074B186006B0BDE8704002B0704700BF28
:106B70004C0D0020540D0020000000204B6900083F
:106B8000500D002010B5044C22681AB97521034835
:106B9000FBF7B2FC206810BD500D00207EBA010842
:106BA0002DE9F84F037C04468A461BB97A21324806
:106BB000FBF7A2FC606903681B689847BAF1020FF3
:106BC000804689460CD10027632226882B4D56EA41
:106BD000070310D12946BDE8F84F294803F00EBE3F
:106BE000BAF1010F04D1668800277322254DEEE724
:106BF0002D22254DEEE7236C504698473046394606
:106C000003F092FD29460246204803F0F7FD18EBF9
:106C1000060A1F4E49EB070B606903681B6898471B
:106C2000504571EB0B03074688461CDABAEB0700A8
:106C30006BEB080103F078FD29460246304603F06D
:106C4000DDFD636C4FF47A70984707460028E3D067
:106C500001462046FFF7D6FE386803F055FE384659
:106C600003F052FED8E7A36C98472946BDE8F84FD9
:106C7000084803F0C3BD00BF7EBA01087CC5010807
:106C800085C5010882C5010847EF0108BFC5010895
:106C9000FBC5010827C601082DE9FF41002748F67A
:106CA000A04805460C4604AE06F8017D0B46324668
:106CB000CDE900781049FDF751F8A31C324628466B
:106CC000CDE900780D49FDF749F80D492846FDF753
:106CD0000CF80C4960602846FDF707F80A49A060E7
:106CE0002846FDF702F8E0609DF80F0080F00100F3
:106CF00004B0BDE8F08100BF17C3010823C3010839
:106D00002FC3010837C3010841C3010870B5054608
:106D10000C460FC985E80F0005F11806616830467A
:106D20000DF01AFEA16830460DF090FEE168304685
:106D30000DF002FF01232B7470BD00004FF4967319
:106D400030B504468DB0254A00930221244B02A899
:106D5000F9F798FA02A92046FDF704FA02A8F9F714
:106D6000F5F900231F4A009302211F4B02A8F9F7EF
:106D700089FA1E4D02A92046FDF7F4F902A8F9F799
:106D8000E5F91B4B1B4A0095032102A8F9F752FABB
:106D900002A92046FDF7E6F902A8F9F7D7F9164B44
:106DA000164A0095032102A8F9F744FA02A92046E1
:106DB000FDF7D8F902A8F9F7C9F9114B114A009566
:106DC000032102A8F9F736FA02A92046FDF7CAF90D
:106DD00002A8F9F7BBF90DB030BD00BF17C3010819
:106DE0004BC3010823C301088BC301087EBA010805
:106DF000CBC301082FC3010811C4010837C3010820
:106E000061C4010841C30108034A02600022027103
:106E10000274C0E90222704754C6010838B50479EB
:106E200000F1080500EB84040834AC4205D054F8A6
:106E3000040D03685B699847F7E738BD70B50646EF
:106E4000002400F108053379A34206DD55F8040B50
:106E5000013403681B699847F5E770BD012A70B5D6
:106E600005460E46144603D815211248FBF744FB8D
:106E7000D5E9021088421BD2C0B92B78091A3046D6
:106E8000013C8C4222BF0C466A7813432A7C43EAB9
:106E9000820300F8013BEB6869682246194410F050
:106EA000B4FFEB68601C2344EB6070BD0023E5E792
:106EB0000020FAE77EBA01080023C0E90112C3608E
:106EC00070474B1C017343738B1C03318373C17375
:106ED000704700002DE9F041074688461E461546DA
:106EE0001AB952211548FBF707FBD7E90143A34222
:106EF00021D2E41ADEB1A3B9A5420ED33B7B337095
:106F0000BB68396822461944404610F07EFFBB68D2
:106F10002344BB602046BDE8F0817B7B33702C4668
:106F2000EEE7A54201D3FB7BE9E7BB7BF6E7AC428A
:106F300028BF2C46E4E70024ECE700BF7EBA010836
:106F40000023C0E900128360704710B5044608466C
:106F5000C4E900120021A160217310F07AFF2046DD
:106F600010BD000038B51546D0E901230446581974
:106F7000904202D9257B55B1D51A20682A4618447B
:106F800010F043FFA3681D44A560012503E017210D
:106F90000248FBF7B1FA284638BD00BF7EBA0108A7
:106FA00007B502AB03F8011D01221946FFF7DAFF0E
:106FB00003B05DF804FB006870478068704713B544
:106FC000044689B201A803F02EFD022201A9204641
:106FD000FFF7C8FF02B010BD13B50446684603F0C2
:106FE0000FFD052269462046FFF7BCFF02B010BD29
:106FF00013B5044601A803F016FD022201A920469C
:10700000FFF7B0FF02B010BD08B50146044803F019
:10701000F5FBBDE808400C210248FBF76DBA00BF44
:1070200068C601087EBA010808B5044803F0E6FB0B
:10703000BDE808401E210248FBF75EBAADC6010854
:107040007EBA010810B503F075FC044630B9044857
:1070500003F0D4FB27210348FBF74EFA204610BD6E
:107060009BC601087EBA010803F064BC10B902484F
:1070700003F0C4BB03F048BC86C60108FFF7E2BFBB
:1070800003F058BCFFF7F2BFFFF7F0BF002103E0A9
:107090000A4B5B584350043109480A4B42189A4244
:1070A000F6D3094A02E0002342F8043B074B9A4218
:1070B000F9D300F00DF8F9F7E3FF7047ACF10108E0
:1070C00000000020D4050020D8050020501A002020
:1070D000314B82B01A6842F480721A6099682F4A64
:1070E0000A409A601A6822F0885222F001121A604F
:1070F0001A6822F480221A609A6822F47D029A604B
:107100000022DA6001921B6813F4007318BF012398
:107110000193019B012B37D14FF48051204B1A680A
:10712000A3F5806322F00102C3F80024D3F8002401
:1071300022F00202C3F80024D3F8002422F0040253
:10714000C3F800245A6A42F080525A62154A11600C
:107150005168C906FCD49A689A609A689A609A68DD
:107160009A605A6822F460425A605A6842F4404277
:107170005A609A6822F003029A609A689A60064AF6
:10718000936813F00C0FFBD14FF00062064B9A602E
:10719000064ADA6002B07047003802400CC0FF882F
:1071A000003C02400070004000ED00E00003FA05E2
:1071B00070B5064688B02E4801F094FB2D4B1A6836
:1071C0000092009A91073CD501214FF4007001F024
:1071D000E3FD012001F0D6FB274A536843F4003356
:1071E0005360A2F5374253681B07FCD500240125E4
:1071F00002A801F0B1FB02A91D488DF80D400694CC
:107200008DF81C508DF80C4001F080FB2A460623B7
:107210003146174801F0C2FB2946154801F0A8FB8A
:107220000221134801F04CFC114801F03BFC134DC6
:1072300001940F4C0221204601F03CFC58B108B0EB
:1072400070BD1A6842F001021A60009A9207BBD41E
:107250001A680092F9E7019B01330193019BB3F592
:10726000805FE7DB38212846FBF746F9E2E700BFFD
:107270000024014000380240002701407EBA010886
:1072800008B5002001F07EFB0021074801F070FBEB
:1072900000214FF4007001F07FFD044A136823F0D1
:1072A0000103136008BD00BF002401400038024004
:1072B00013B5072301220146114801F06FFB02219B
:1072C0000F4801F0FDFB0E4801F0ECFB00230D4CD4
:1072D000019302210A4801F0EDFB28B1084802B0F1
:1072E000BDE8104001F0E3BB019B01330193019B1A
:1072F000B3F5805FEDDB4C212046FBF7FDF8E8E7B6
:10730000002401407EBA010870B506460825FFF743
:107310004FFF00243046FFF7CBFF013D0444F9D175
:10732000FFF7AEFFC4F3CF0070BD00000000000007
:1073300008B51120FFF7E8FF0FF024FF01460848C9
:1073400010F02CF80FF006FB03A3D3E900230FF095
:1073500059FB0FF011FE08BD2FDD24068195F33F88
:1073600000F07F450F4A536A43F0805353620E4B3F
:107370001A465968C906FCD41B68022823F4C05376
:1073800006D143F4C05313605368DB06FCD4704746
:10739000012802D143F48053F5E70028F3D143F4E8
:1073A0000063F0E7003802400070004010B50C4B5D
:1073B0005A68D206FCD41C6814F4C05F0BD114F4D4
:1073C00080500AD114F4006404D106482A21FBF746
:1073D00093F8204610BD0220FCE70120FAE700BF29
:1073E000007000407EBA010838B50546012001F062
:1073F00077FB022D01BF154A136843F001031360A8
:10740000134B1A6842F480321A601A689203FCD552
:1074100042F690529A6099689142FCD19A6842F083
:1074200002029A600A4B9C6814F00804FBD14FF4E6
:1074300080321A60074B084A28461A60FFF792FF0D
:107440002046BDE8384001F03FBB00BF003C024091
:1074500000380240C400002000093D0038B5054650
:10746000012001F03DFB022D01BF144A136843F0D7
:1074700001031360124B1A6842F480721A601A6892
:107480009205FCD55A6822F4604242F440425A60A8
:1074900000229A600A4B9C6814F00C04FBD14FF454
:1074A00080721A60074B084A28461A60FFF75AFF95
:1074B0002046BDE8384001F007BB00BF003C024059
:1074C00000380240C4000020D0FE3F000C4B5A6B35
:1074D000900513D45A6A42F080525A62094A1168E0
:1074E00041F480711160596B41F480715963596B9B
:1074F0008905FCD5136823F480731360704700BFBF
:107500000038024000700040054B5A6B910706D4CA
:107510005A6B42F001025A635A6B9207FCD57047CE
:1075200000380240094B5A6A42F020025A629A69B6
:1075300042F020029A619A6922F020029A610022A8
:10754000A3F509331A801A855A6270470038024041
:10755000002349F6FE7282B00193019B934201DD44
:1075600002B07047019B01330193F6E7002340F618
:10757000FE7282B00193019B934201DD02B070471D
:10758000019B01330193F6E7002382B00193019B35
:10759000B3F5CC7F01DD02B07047019B0133F5E705
:1075A000D0B1012801D1FFF7EFBF0C4B00211A68C1
:1075B0004FF47A73B2FBF3F2094B013A92B21A8597
:1075C00001220138D8629A82596219821A801A8A75
:1075D000D207FCD500221A80704700BFC4000020EB
:1075E0000014004000F1774303F57803B3F5804FB2
:1075F0002DE9F04106460C4617462DD202F1F7332D
:1076000003F608030344B3F5804F25D2FFF7CEFEFF
:10761000804610B10020FFF7A5FE01F079FA0125A0
:107620002744361BA7420AD101F082FAB8F1000FB5
:1076300002D04046FFF796FE2846BDE8F08141F6AD
:10764000027001F07DFA301914F8011B01F0D4FA30
:10765000042818BF0025E5E70025EDE710B50C4626
:1076600000F1774101F57801B1F5804F0DD202F1BB
:10767000F73303F608030344B3F5804F05D2014600
:10768000204610F0C2FB012010BD0020FCE70000E6
:1076900008B5114B984215D003F58063984213D07A
:1076A00003F58063984211D003F5806398420FD0B0
:1076B00003F5006398420DD0084B094A142109488C
:1076C00010F086F9002008BD0120FCE70220FAE74F
:1076D0000320F8E70520F6E70000024020C7010874
:1076E000DAC6010839C701080F2808B505D9094BC2
:1076F000094A3B21094810F06BF9012303FA00F015
:10770000C043074A51680140516013681840106037
:1077100008BD00BF78C70108E4C6010839C70108E1
:10772000000401400F292DE9F84F82460D4693468B
:107730001F4605D95A4B5B4A54215B4810F048F963
:107740004FF0010909FA05F900F0B8F86FEA0903EA
:10775000564E032D7268564C02EA0302726032687C
:1077600003EA0203534A3360136A43F001031362CE
:107770002ED80F22A3684FEA850802FA08F223EAFE
:107780000203A3605046FFF783FFA36800FA08F0E6
:107790001843A0601BF0020F18BFB368464A1CBF15
:1077A00043EA0903B3601BF0040F1EBFF36843EA0A
:1077B0000903F360336843EA090333603B01DBB23A
:1077C000002D45D182F8063340231360BDE8F88FC1
:1077D000072D13D80F22A5F10408E3684FEA8808A3
:1077E00002FA08F223EA0203E3605046FFF750FF73
:1077F000E36800FA08F01843E060CBE70B2D13D8DC
:107800000F22A5F1080823694FEA880802FA08F256
:1078100023EA020323615046FFF73AFF236900FA87
:1078200008F018432061B5E70F22A5F10C08636941
:107830004FEA880802FA08F223EA0203636150461D
:10784000FFF726FF636900FA08F018436061A1E7BB
:10785000012D03D182F807338023B6E7022D04D12E
:1078600082F808334FF48073AFE7032D04D182F818
:1078700009334FF40073A8E7042D04D182F80A33CA
:107880004FF48063A1E7092D04D882F817334FF431
:1078900000039AE782F828334FF48073536095E72A
:1078A00084C70108FFC6010839C701080004014068
:1078B000000001400038024000E100E0144B984213
:1078C00005D1144AD36943F00103D3617047124BC9
:1078D000984204D10F4AD36943F00203F5E70F4BF6
:1078E000984204D10B4AD36943F00403EDE70C4BF3
:1078F000984204D1074AD36943F00803E5E7094BEE
:107900009842E3D1034AD36943F02003DDE700BF87
:10791000000002400038024000040240000802401B
:10792000000C0240001402400323490010B5846893
:107930008B4024EA030484600124022A04FA01F43F
:1079400007D0032A0DD0012A07D18368234383601F
:1079500003E083688A401A43826083681C43846022
:1079600010BD82681343F2E70F29F8B504460F46AD
:1079700015461E4603D94B211948FAF7BDFD20468E
:10798000FFF79CFF03237A009340DB4321681940F3
:1079900021600121D4F800C001FA02F04CEA000C89
:1079A000B940C4F800C009B266B1A688314389B2B3
:1079B000A180E168012D03EA0103E36006D0022DF6
:1079C00008D0F8BDA68826EA0101F1E7E368034381
:1079D000E360F6E7E36805FA02F21A43E260F0E7D3
:1079E0007EBA01080F2970B505460C46164603D924
:1079F0006B210E48FAF780FD2846FFF75FFF03234F
:107A000061008B40DB43EA68012E02EA0302EA6070
:107A100005D0022E03D02A6813402B6070BDEA689F
:107A200006FA01F11143E960F5E700BF7EBA0108EB
:107A30000F2938B50446154605D987211B4B1C4A2A
:107A40001C480FF0C5FF0F2A03D91B4B184A882189
:107A5000F6E7FFF733FF07294FF00F0318D8006A46
:107A60008A00934020EA03032362236A05FA02F2A4
:107A70001A4322620322236849008A4023EA020350
:107A800023600223226803FA01F11143216038BD0B
:107A9000A1F10802406A9200934020EA0303636266
:107AA000636A95401D436562E4E700BF78C701083B
:107AB00090C70108C1C70108AEC70108012303FA36
:107AC00001F189B201837047012303FA01F189B200
:107AD00041837047012303FA01F189B20AB101839E
:107AE000704741837047008A084100F001007047E9
:107AF00010B5084C23681BB9012005F0D9FA2060A5
:107B000023682BB9BDE8104036210348FAF7F4BCCE
:107B100010BD00BFA00D00207EBA010810B50B4CAF
:107B200022681AB93C210A48FAF7E6FC206842F2BA
:107B3000107105F005FC01280CBF0124002403D0BE
:107B400040210348FAF7D8FC204610BDA00D0020C4
:107B50007EBA010810B5074C22681AB951210648AF
:107B6000FAF7CAFC002320681A46BDE810401946FF
:107B700005F0FAB9A00D00207EBA010810B5044640
:107B8000FFF7B6FFFFF7CAFF21461022034801F0B6
:107B900003FE0446FFF7DEFF204610BD0054004000
:107BA00010B5FFF7A5FFFFF7B9FF01F0ADFD0446E3
:107BB000FFF7D0FF204610BD08B513460A46014620
:107BC000034801F0E1F9003018BF012008BD00BFF3
:107BD0000054004008B513460A460146034801F028
:107BE000D3FA003018BF012008BD00BF0054004088
:107BF00008B513460A460146034801F0A1FB0030D0
:107C000018BF012008BD00BF0054004008B513464E
:107C10000A460146034801F023FC003018BF01204A
:107C200008BD00BF0054004008B513460A4601468F
:107C3000034801F06DFC003018BF012008BD00BFF3
:107C4000005400400123064A83405169194205D07F
:107C50005361044B53F8203003B11847704700BFFD
:107C600000040140A40D00200F2838B504460D463D
:107C700003D926210348FAF73FFC034B43F824506D
:107C800038BD00BF7EBA0108A40D00200020FFF718
:107C9000D9BF0120FFF7D6BF0220FFF7D3BF0320D3
:107CA000FFF7D0BF0420FFF7CDBF08B50920FFF7CD
:107CB000C9FF0820FFF7C6FF0720FFF7C3FF062014
:107CC000FFF7C0FFBDE808400520FFF7BBBF08B5C0
:107CD0000F20FFF7B7FF0E20FFF7B4FF0D20FFF7CF
:107CE000B1FF0C20FFF7AEFF0B20FFF7ABFFBDE8A5
:107CF00008400A20FFF7A6BFFEE7FEE7FEE7FEE723
:107D0000FEE7FEE7FEE7FEE7FEE7FEE7FEE7FEE74B
:107D1000FEE7FEE7FEE7FEE7FEE7FEE7FEE7FEE73B
:107D2000FEE7FEE7FEE7FEE7FEE7FEE7FEE7FEE72B
:107D3000FEE7FEE7FEE7FEE7FEE7FEE7FEE7FEE71B
:107D4000FEE7FEE7FEE7FEE70A23B0FBF3F203FBE4
:107D5000120040EA0210C0B270470000CA22024B73
:107D60005A6253225A62704700280040014B186043
:107D7000704700BFE40D00204FF400320F4B10B5E8
:107D80000F4C5A61E368DB0503D430210D48FAF744
:107D9000B3FBFFF7E3FF4FF40072A36823F48853AB
:107DA000A360094BC3F88420FF236362074B1B6861
:107DB00013B1BDE81040184710BD00BF00040140DA
:107DC000002800407EBA010800E100E0E40D002038
:107DD0002DE9F04F9846374B85B01B788246914687
:107DE0009DF838709DF83C602BB9334B334A8C2199
:107DF00033480FF0EDFD431E1E2B59D80C2957D8E0
:107E0000A2F5FA63632B53D8B8F1170F50D83B2F64
:107E10004ED83B2E4CD802F13000C0B2FFF794FF91
:107E200083460846FFF790FF04465046FFF78CFF55
:107E300040F400554046FFF787FF45EA0B4545EA09
:107E4000042504463846FFF77FFF000240EA044459
:107E50003046FFF779FF20431A4CFFF77FFFE368B6
:107E600043F08003E360E3685B06FCD56560206057
:107E7000E36823F08003E360124BDA689206FCD5D6
:107E8000FF2204A85A6200F80C6D8DF807A08DF847
:107E90000810ADF809908DF806808DF8057002F095
:107EA000EAFB094BC3E90001012005B0BDE8F08FF2
:107EB0000020FAE7E80D002031C8010825C80108B4
:107EC0003AC8010800280040F00D002037B50578B9
:107ED000C4788378B0F80520017901954078009046
:107EE0002046FFF775FF03B030BD000038B52B4BBF
:107EF00004461B781BB9E4212948FAF7FDFA294A00
:107F0000D36823F02003D360D3689B06FCD51368A5
:107F10005268C2F30741080900EB800001F00F012D
:107F200001EB4001C9B201F5FA61A4F80510C2F3F2
:107F30000721C1F300108500284401F00F0101EB77
:107F40004001D2B22171C2F3011101EB810102F0B3
:107F50000F0202EB4102E270C3F30742C2F30111C8
:107F600001EB810102F00F0202EB4102A270C3F3A8
:107F70000722C2F3021101EB810102F00F0202EBB2
:107F80004102DBB26270C3F3021202EB820203F021
:107F90000F0303EB4203237038BD00BFE80D002040
:107FA0007EBA0108002800401FB501A8FFF79EFF18
:107FB00001A802F060FB05B05DF804FB08B5FFF70F
:107FC00085FA1B4A136843F480731360FFF7C6FEFB
:107FD000184A536B23F4403343F482035363164B24
:107FE000DA6842F08002DA60DA685106FCD5FF22D6
:107FF0001A611A6942F4FE021A619A6822F040027C
:108000009A609A6822F44C529A60DA6822F08002F0
:10801000DA60094BDA689206FCD5FF225A62012227
:10802000064B1A70FFF7C0FF054BC3E9000108BDFE
:10803000007000400038024000280040E80D002099
:10804000F00D002008B5094B1B7823B940F21F1131
:108050000748FAF751FAFFF781FE064B9A6822F4B7
:1080600080729A60FF225A6208BD00BFE80D0020AE
:108070007EBA01080028004008B5144B1B7833B9BC
:10808000134B144A40F2271113480FF0A1FCFFF7DD
:1080900065FE124BDA6822F48072DA60104A916849
:1080A00041F400319160116841F400311160F02118
:1080B0000C4A82F829134FF4007151609A6842F417
:1080C00088529A60FF225A6208BD00BFE80D002066
:1080D00031C80108FEC701083AC80108002800405D
:1080E0000004014000E100E0F8B51E46194B1746B8
:1080F0001B7833B9184B194A4FF4A57118480FF083
:1081000067FC184CFFF72AFEA56825F48075A5606A
:10811000E56825F48075E560FFF716FE054608461C
:10812000FFF712FE000440EA05613846FFF70CFE37
:1081300005463046FFF708FE084340EA0520E3689D
:10814000DB07FCD5FF23E0616362BDE8F840FFF781
:1081500093BF00BFE80D002031C8010813C8010813
:108160003AC8010800280040037842788178C07836
:10817000FFF7BABF38B50D46044604F0B3FC1F4AFA
:10818000136823F00103136004F0CCFC25B11C4AF2
:10819000536843F00603536072B6BFF34F8FBFF3CB
:1081A0006F8F184A0120136823F0030343F4007310
:1081B00043F00103136000F09FFC134B1A6942F077
:1081C00004021A6130BF1A6922F004021A610F4BCF
:1081D0000F4A1B6893420AD10220FFF73FF9074A72
:1081E000136843F00103136004B162B638BD094A55
:1081F0009342F4D10220FFF7F7F8F0E710E000E037
:10820000002004E00070004000ED00E0C400002009
:10821000D0FE3F0000093D0062B6704700220E4BC1
:1082200010B51A700D4A0E4C1388204623F04003F7
:108230001B041B0C13800D210222FFF7D3FB2046E9
:1082400002220E21FFF7CEFB2046BDE8104002229D
:108250000F21FFF7C7BB00BFF80D0020003800401A
:108260000004024038B50546274A2848536A0C46A0
:1082700043F4804353620D210522FFF7D9FB052209
:108280000E212248FFF7D4FB05220F211F48FFF7DC
:10829000CFFBC5B101220D211C48FFF745FB012290
:1082A0000E211A48FFF740FB01220F211748FFF764
:1082B0003BFB012C21D144F451740122144B1C804E
:1082C000144B1A7038BD2A460D211048FFF72CFBBD
:1082D0002A460E210D48FFF727FB2A460F210B489F
:1082E000FFF722FB012C05D0022C03D0032C14BF76
:1082F0000024032444F45974DFE7022CDBD0032C60
:108300000CBF03240024D6E70038024000040240DA
:1083100000380040F80D0020064B074A988111787C
:108320001A461889C00701D40029FAD19089C0B231
:10833000704700BF00380040F80D0020284A38B5CB
:10834000136A054643F480531362052225480C4600
:108350001146FFF76DFB052206212248FFF768FB57
:10836000052207211F48FFF763FBC5B10222052143
:108370001C48FFF7D9FA022206211A48FFF7D4FA5F
:10838000022207211748FFF7CFFA012C21D144F42C
:1083900051740122144B1C80144B1A7038BD2A46AC
:1083A00005211048FFF7C0FA2A4606210D48FFF7BD
:1083B000BBFA2A4607210B48FFF7B6FA012C05D075
:1083C000022C03D0032C14BF0024032444F459745A
:1083D000DFE7022CDBD0032C0CBF03240024D6E7FC
:1083E000003802400000024000300140F90D00203A
:1083F00000220E4B10B51A700D4A0E4C1388204601
:1084000023F040031B041B0C138005210222FFF7FD
:10841000E9FA204602220621FFF7E4FA2046BDE8E9
:10842000104002220721FFF7DDBA00BFF90D00203E
:108430000030014000000240064B074A9881117845
:108440001A461889C00701D40029FAD19089C0B210
:10845000704700BF00300140F90D0020054AD36885
:1084600023F4E0631B041B0C43F0BF6343F40033AD
:10847000D360704700ED00E020220021114B10B5C1
:10848000C3F88420104B114C1A6A204642F48042F3
:108490001A625A6942F480425A615A6922F480424F
:1084A0005A610B4A91811A6A092122F480421A62A8
:1084B0000222FFF797FA2046BDE8104002220A2167
:1084C000FFF790BA00E100E00038024000000240EF
:1084D0000038014010B50B4C40F22551204600F009
:1084E0002CFD48B1204600F006FD074BC0B21B68CA
:1084F00033B1BDE810401847A388044ADBB21370BB
:1085000010BD00BF00380140FC0D0020A019002064
:1085100010B504468021084800F009FD0028F9D074
:108520002146054800F0E3FC034C4021204600F0C2
:10853000FEFC0028F9D010BD0038014010B5441EE3
:1085400014F8010F00B910BDFFF7E2FFF8E70000D3
:1085500008B5024800F0CFFCC0B208BD00380140A9
:108560002DE9F0438846012189B08146084614462A
:108570001D4600F005FC01214FF4804000F00CFC8A
:108580004FF4C06702230122002602A93F488DF85C
:108590000C308DF80D308DF80F2002978DF80E609D
:1085A00000F050FB07220921384800F08DFB07221C
:1085B0000A21364800F088FBB8F1450FCDF810903D
:1085C0003CD14FF48063ADF81830072C42D1002322
:1085D000ADF81430052D4ED14FF48053ADF8163060
:1085E0000023ADF81C300C2304A92948ADF81A303B
:1085F00000F022FC274B1A6802B1012240F22551FB
:10860000234800F07CFC0121214800F065FCFFF7C5
:108610009FFF25238DF804309DF840308DF80530FC
:1086200000238DF8063001238DF80730FFF716FF81
:1086300001A800F03BF909B0BDE8F083B8F14F0F95
:1086400002D1ADF81870C0E7072CADF818600DD155
:10865000592107E0082C02D14FF48053B8E7092CC8
:10866000B8D154210C48F9F747FFB3E7082CAED036
:10867000092CAFD1F0E70F2D02D14FF44053ADE7F5
:10868000022D0CBF4FF400530023A7E70000024067
:1086900000380140FC0D00207EBA01080E2307B50A
:1086A000082200934E210123FFF75AFF03B05DF823
:1086B00004FB000070B5134C40F22551204600F039
:1086C0003CFCC0B1104B1D6825B1204600F013FCE6
:1086D000C0B2A84740F226610A4800F02EFC78B1EB
:1086E00040F22661074800F047FC084B1B683BB18D
:1086F000BDE870401847A388054ADBB21370E9E76C
:1087000070BD00BF00440040000E0020040E002099
:10871000A0190020BFF34F8F0449054BCA6802F42B
:10872000E0621343CB60BFF34F8FFEE700ED00E044
:108730000400FA0510B5441EE3B2052B03D9172136
:108740001148F9F7D9FEFEF7DFFE45F255520F4BFF
:108750001A60DA68D207FCD4052C06D8DFE804F0EA
:1087600003090B0D0F1101225A604CF6CC421A601E
:1087700010BD0222F8E70322F6E70422F4E70522FF
:10878000F2E70622F0E700BF7EBA010800300040A1
:1087900038B5224C236853B95F2000F015FB204DFB
:1087A00038B1204B236001232B7000F01DFB2068A3
:1087B00038BD5E2000F008FB18B11B4B236002237C
:1087C000F2E75D2000F000FB18B1184B2360032393
:1087D000EAE75C2000F0F8FA18B1154B2360042397
:1087E000E2E75B2000F0F0FA18B1124B236005239A
:1087F000DAE75A2000F0E8FA18B10F4B236006239D
:10880000D2E7592000F0E0FA18B10C4B236007239F
:10881000CAE70B4B2360FF23C6E700BF0C0E002006
:10882000100E002076C8010886C801089CC80108FF
:10883000B7C80108C6C80108D5C80108EEC80108B4
:108840003DCE010838B5084B084D1A7852B90124BD
:1088500020461C7000F0E0FA287020F0FF0120464E
:1088600000F0CAFA287838BD080E0020090E002052
:1088700010B50446012000F0CFFA20F0FF0121439B
:108880000120BDE8104000F0B7BA08B5FFF7F0FFCF
:10889000FFF740FF08B5012000F0BEFA10F0FF0F0F
:1088A00002D10120FFF7F1FFFFF734FF30B50124BB
:1088B00003780A4D03F01F029440C278590952B15F
:1088C000074A2B44D26842781201D2B283F80023BF
:1088D00045F8214030BD2031FAE700BF00E100E05B
:1088E00000ED00E008B5084B98420BD101214FF490
:1088F000007000F05DFABDE8084000214FF4007000
:1089000000F056BA08BD00BF0024014043680A7950
:1089100023F0407323F4807343EA02230A6810B5FE
:1089200013434360D1E9032313438A6884681343E4
:10893000084A224013434A7943EA420383600A7D8E
:10894000036B013A23F0F873D2B243EA0253036394
:1089500010BD00BFFDF7FFC000234FF04072036061
:10896000037143718360C0E90323012303757047DA
:10897000836819B143F001038360704723F001035A
:10898000FAE70000044B5A6818B142F400025A603A
:10899000704722F40002FAE7002701401D2970B554
:1089A0001BD90725A1F11E06C46D06EB4606B5408E
:1089B00024EA050403FA06F62643C665062A38D8D3
:1089C0001F24013A036C02EB8202944023EA040361
:1089D00001FA02F21A43026470BD13290DD9072669
:1089E000A1F11405C46805EB4505AE4024EA060470
:1089F00003FA05F52543C560E0E709290DD90726E7
:108A0000A1F10A04056904EB4404A64025EA060521
:108A100003FA04F42C430461D0E70726446901EB10
:108A20004105AE4024EA060403FA05F626434661F2
:108A3000C4E70C2A0CD81F24073AC36B02EB82024E
:108A4000944023EA040301FA02F21A43C263C3E723
:108A5000122A0CD81F240D3A836B02EB8202944039
:108A600023EA040301FA02F21A438263B4E7182AE4
:108A70000CD81F24133A436B02EB8202944023EA82
:108A8000040301FA02F21A434263A5E71F24193ACC
:108A9000036B02EB8202944023EA040391401943E2
:108AA000016399E7836843F0804383607047806D7A
:108AB00080B270470368194214BF0120002070473C
:108AC000C943016070470000044B1A6818B142F0B6
:108AD00002021A60704722F00202FAE7003C0240EC
:108AE000044B1A6818B142F004021A60704722F071
:108AF0000402FAE7003C0240044B1A6818B142F045
:108B000008021A60704722F00802FAE7003C0240AF
:108B1000044B5A68D20741BF034ADA60034ADA605D
:108B2000704700BF003C0240EFCDAB890504030253
:108B3000024A536843F0010353607047003C02400F
:108B4000014B9861704700BF003C0240084B9A6996
:108B5000D10709D49A69D20508D49B6913F4F05F50
:108B600014BF032004207047012070470220704783
:108B7000003C0240042313B504468DF80730FFF78C
:108B8000E5FF8DF807009DF80730012B0AD11CB9CD
:108B900005238DF8073007E0FFF7D8FF013C8DF87B
:108BA0000700F0E7002CF3D09DF8070002B010BDDD
:108BB00010B504464FF40040FFF7DCFF042804BF63
:108BC0000023236010BD000038B504464FF4004078
:108BD0000D46FFF7CFFF04280BD1064A4FF40040A3
:108BE000536823F4807353602560BDE83840FFF775
:108BF000C1BF38BD003C024038B504464FF40040C8
:108C00000D46FFF7B7FF04281BD135B125704FF48F
:108C10000040BDE83840FFF7ADBFFF2324F0030557
:108C200004F003042968E40003FA04F421EA0404CC
:108C30002846FFF7BDFF21462846BDE83840FFF72C
:108C4000C3BF38BD2DE9F0430022012703250E687C
:108C500007FA02F333EA060431D14FEA420C05FA6F
:108C60000CF4E44391F804E0D0F800900EFA0CF80C
:108C700004EA09090EF1FF3E48EA0908BEF1010FB6
:108C8000C0F8008011D8D0F808E004EA0E0E4C7944
:108C900004FA0CF444EA0E048460848824EA030491
:108CA0008B7993409BB223438380C36805FA0CF40D
:108CB00023EA0404CB7903FA0CF32343C3600132A3
:108CC000102AC5D1BDE8F08310B50F2401F00703C9
:108CD000C90800EB8100016A9B009C4021EA040165
:108CE0000162016A9A400A43026210BD204B10B52E
:108CF0009A6802F00C020C2A30D8DFE802F02F2F1D
:108D00002F2F072F2F2F072F2F2F2000194B184AF7
:108D1000036093681849C3F30313CC5C0368E34012
:108D200043609468C4F302240C5D23FA04F4846065
:108D30009268C2F3C2228A5CD340C36010BD9968B6
:108D40000E4CC1F383419A68615C9B68094BC2F386
:108D500081524B430132B3FBF2F3D8E74FF40042A8
:108D60005B68C3F34233013302FA03F3CFE700BF7A
:108D7000003802400024F400C8000020D800002081
:108D8000044BDA6911B11043D861704722EA000040
:108D9000FAE700BF00380240044B1A6A11B11043D1
:108DA0001862704722EA0000FAE700BF003802406C
:108DB000044B5A6911B110435861704722EA000010
:108DC000FAE700BF003802404309012B054B00F0D1
:108DD0001F000CBF1B685B6B23FA00F000F0010062
:108DE000704700BF00380240024A536B43F0807363
:108DF0005363704700380240002382B00193054B53
:108E00000193019B03EB80000190019B196002B06C
:108E1000704700BF50280040002382B00193054BEB
:108E20000193019B03EB80000190019B186802B045
:108E3000704700BF5028004030B50D460446028AF6
:108E4000EB8892B222F440521A43898902828389C4
:108E5000288923F4B052AB8822F00C0203436889BE
:108E600085B003431343A381A38A68469BB223F4CE
:108E700040730B43A382FFF739FFDDE90231154A46
:108E8000944218BF19461923A2894B43296810043C
:108E90004CBF49008900B3FBF1F16425B1FBF5F348
:108EA000A2891801120405FB13130BD5DA00323224
:108EB000B2FBF5F202F0070242EA00039BB2238103
:108EC00005B030BD1B013233B3FBF5F303F00F03E4
:108ED0000343F3E700380140838919B143F4005399
:108EE0008381704723F400531B041B0CF8E7C1F384
:108EF0000801818070478088C0F30800704701F046
:108F00001F0310B5C1F342140121012C01FA03F132
:108F100005D10C3003683AB11943016010BD022C31
:108F20000CBF10301430F5E723EA0101F5E70388A0
:108F3000194214BF0120002070470123C1F34212DF
:108F400010B5012A01F01F0403FA04F30DD1828940
:108F50001340028892B26BB10123090A03FA01F1AE
:108F60000A4214BF1846002010BD022A0CBF028A14
:108F7000828AEDE71846F7E70B0A01219940C943B9
:108F800089B20180704700002DE9F3411F4600239C
:108F900004460D46019316461AB9012002B0BDE8F9
:108FA000F08140F6FF7301934FF40031204600F04A
:108FB0004CFD002852D10121204600F016FD4FF251
:108FC000FF71204600F02AFD0121204600F0F7FC49
:108FD00040F6FF73DFF8AC8101934146204600F074
:108FE00029FD002841D039460122204600F008FD25
:108FF00040F6FF735F4F01933946204600F025FD90
:10900000002838D0012E42D10021204600F0EDFC8E
:1090100003F068FD31462046238B00F0DBFC03F0B3
:1090200081FD40F6FF73544E01933146204600F017
:109030000CFD30B3204600F0EEFC287040F6FF73C4
:109040004E4D01932946204600F0FFFC0028A4D095
:10905000019B5A1E0192002BF4D104E0019B5A1E81
:109060000192002BA0D1002098E7019B5A1E01928B
:10907000002BB2D1F7E7019B5A1E0192002BBBD106
:10908000F1E7019B5A1E0192002BCED1EBE7022E95
:1090900025D103F027FD4FF40061204600F0BEFC0F
:1090A0000021204600F0A1FC238B03F03BFD40F69D
:1090B000FF73334E01933146204600F0C6FC40B1A9
:1090C0000121204600F086FC238A2B70238A6B70D6
:1090D000B4E7019B5A1E0192002BECD1C3E740F686
:1090E000FF77033E238BDFF898802E44B54201972B
:1090F00028D1234E3146204600F0A7FC70B3002152
:10910000204600F072FC204600F085FC40F6FF731C
:109110001B4E287001933146204600F096FC18B390
:109120000121204600F056FC204600F074FC6870D7
:10913000204600F070FCA87080E7019B5A1E019247
:10914000002B90D04146204600F07FFC0028F4D050
:10915000204600F060FC05F8010BC7E7019B5A1E92
:109160000192002BC6D17EE7019B5A1E0192002B73
:10917000D1D178E70200001040000010100000106C
:1091800004000010010003002DE9F3411E460023F6
:10919000019340F6FF7304460D4617460193002ADB
:1091A00000F081804FF40031204600F04EFC002892
:1091B00042D10121204600F002FC40F6FF73DFF8A7
:1091C0007C8101934146204600F034FC00283CD0CD
:1091D00031460022204600F013FC40F6FF73534E48
:1091E00001933146204600F025FC002833D0297831
:1091F00020466E1C00F00DFC3D4440F6FF77DFF882
:109200003081AE42019731D1494D2946204600F0C8
:109210001CFC002836D02046012100F0DBFB40F684
:10922000FF73444D444C01932946204600F00DFC49
:1092300000282DD1012005E0019B5A1E0192002B30
:10924000B0D1002002B0BDE8F081019B5A1E01920E
:10925000002BB7D1F5E7019B5A1E0192002BC0D11C
:10926000EFE7019B5A1E0192002BEAD041462046AF
:1092700000F0EBFB0028F4D016F8011B204600F0AC
:10928000C8FBBEE7019B5A1E0192002BBDD1D8E757
:10929000019B5A1E0192002BC6D1D2E7019B5A1E98
:1092A0000192002BCDD04FF40031204600F0CDFBD1
:1092B0000028F3D10121204600F081FB40F6FF7326
:1092C0001E4D01932946204600F0B4FB10B3002246
:1092D0003146204600F094FB40F6FF73134D019396
:1092E0002946204600F0A6FBD0B12046012100F01F
:1092F00071FB40F6FF730F4D0F4C0193294620463A
:1093000000F0A3FB002895D0019B5A1E0192002B70
:10931000F4D196E7019B5A1E0192002BD2D190E71F
:10932000019B5A1E0192002BDAD18AE782000700C6
:109330000400001010000010005400400100030061
:109340002DE9F3411E46002304460D4601931746BE
:109350001AB9012002B0BDE8F08140F6FF73019315
:109360004FF40031204600F070FB002837D1012176
:10937000204600F024FB40F6FF73DFF8E080019305
:109380004146204600F056FB002842D031460022DC
:10939000204600F035FB40F6FF732C4E019331461A
:1093A000204600F047FB002839D0297820466E1C63
:1093B00000F02FFB3D4440F6FF77DFF89480AE428B
:1093C000019737D1224D2946204600F03EFB002868
:1093D000BFD1019B5A1E0192002BF4D104E0019BE6
:1093E0005A1E0192002BBBD12046012100F0F2FA57
:1093F00040F6FF73174D184C01932946204600F0A4
:1094000024FB20B1019B5A1E0192002BF5D10020B4
:10941000A0E7019B5A1E0192002BB1D1E4E7019B0A
:109420005A1E0192002BBAD1DEE7019B5A1E01920F
:10943000002BD9D04146204600F007FB0028F4D08D
:1094400016F8011B204600F0E4FAB8E78200070096
:109450000400001010000010005400400100030040
:1094600000232DE9F3410D464FF400310446174621
:10947000019300F0EAFA18B9002002B0BDE8F081CB
:109480000FB90120F9E7297820466E1C00F0C1FAD7
:109490003D4440F6FF77DFF86C80AE4201971FD164
:1094A000184D2946204600F0D0FA28B32046012165
:1094B00000F090FA40F6FF73134D144C01932946C7
:1094C000204600F0C2FA0028DBD0019B5A1E019210
:1094D000002BF4D1D0E7019B5A1E0192002BCBD078
:1094E0004146204600F0B1FA0028F4D016F8011BDE
:1094F000204600F08EFAD0E7019B5A1E0192002B05
:10950000CFD1B9E704000010100000100054004053
:109510002DE9F3411F46002304460D4601931646EC
:109520001AB9012002B0BDE8F0814FF4003100F01B
:109530008CFA08B90020F5E70121204600F055FA21
:109540004FF2FF71204600F069FA0121204600F039
:1095500036FA40F6FF73DFF8AC81019341462046AE
:1095600000F068FA00283AD039460122204600F07F
:1095700047FA40F6FF735F4F01933946204600F0EB
:1095800064FA002831D0012E3BD10021204600F0A2
:109590002CFA03F0A7FA31462046238B00F01AFA82
:1095A00003F0C0FA40F6FF73534E01933146204654
:1095B00000F04BFAF8B1204600F02DFA287040F682
:1095C000FF734E4D01932946204600F03EFA0028D5
:1095D000A7D0019B5A1E0192002BF4D1AAE7019B50
:1095E0005A1E0192002BB9D1A4E7019B5A1E019289
:1095F000002BC2D19EE7019B5A1E0192002BD5D1B0
:1096000098E7022E29D14FF40061204600F006FAB7
:1096100003F068FA00212046238B00F0E6F903F0FE
:1096200081FA40F6FF73364E01933146204600F032
:109630000CFA60B103F056FA0121204600F0CAF995
:10964000238A2B70238A6B7003F06CFAB7E7019BB7
:109650005A1E0192002BE8D16CE740F6FF77033EDB
:10966000238BDFF89C802E44B542019729D1244EEC
:109670003146204600F0E9F978B30021204600F099
:10968000B4F9204600F0C7F940F6FF731C4E28706D
:1096900001933146204600F0D8F920B3012120463D
:1096A00000F098F9204600F0B6F96870204600F006
:1096B000B2F9A87083E7019B5A1E0192002B3FF478
:1096C00039AF4146204600F0C0F90028F3D02046CB
:1096D00000F0A1F905F8010BC6E7019B5A1E0192A3
:1096E000002BC5D126E7019B5A1E0192002BD0D139
:1096F00020E700BF02000010400000101000001022
:10970000040000100100030038B5204B08219A69BD
:109710001F4842F400129A619A6922F400129A6179
:109720005A6A22F400125A62FEF7C8F9012308218E
:109730001A461748FEF718F9092115480122FEF7C5
:1097400051F909211248FEF7CEF9D8B1012038BDF0
:1097500008212846FEF7B2F9FDF716FF0821284632
:10976000FEF7B2F9FDF710FF013CF1D109210848DD
:10977000FEF7B9F920B940F27D110648F8F7BCFEB2
:109780002046E4E73324024DEEE700BF00380240F4
:10979000000402407EBA01082DE9FF41444B054612
:1097A00098420E4617467CD103F5F2335A6A0821D7
:1097B00042F400125A629A693E4842F400129A61D9
:1097C0009A6922F400129A61FEF778F901230821C0
:1097D0001A463848FEF7C8F8092136480122FEF734
:1097E00001F909213348FEF77EF9002855D00123FD
:1097F00008211A462F48FEF7B7F8042208212D4801
:10980000FEF716F9012309211A462A48FEF7ACF89B
:10981000042209212748FEF70BF9274B9A6942F4E5
:1098200000129A619A6922F400129A61684600F067
:10983000ADF8224B694601934FF48063ADF80A30CE
:109840004FF480432846ADF80C30ADF80870009610
:1098500000F038F82846012100F0A6F8012019E0B0
:1098600008214046FEF72AF9FDF78EFE0821404602
:10987000FEF72AF9FDF788FE013CF1D109210D48D8
:10988000FEF731F90028B2D10D4840F2A511F8F7E2
:1098900033FE204604B0BDE8F0813324DFF81480A5
:1098A000EAE74FF4DA710648F8F726FEBEE700BF94
:1098B0000054004000040240003802400000FFBF96
:1098C0007EBA01087FB50446868868460D46FFF7D4
:1098D0000DFA029A2B4926F03F06B2FBF1F136044D
:1098E000360C88B20643A6802388274E23F0010356
:1098F0001B041B0C23802B68B3421ED85B00B2FBF9
:10990000F3F39BB2042B38BF0423013080B22084D0
:10991000A3832388AA8843F00103238023886989CD
:1099200023F481630A4323F00203134323802A892B
:10993000AB891343238104B070BD4BF6FF70EE88F2
:1099400086421BBF1920434303EB4303B2FBF3F3EF
:109950000BBFB2FBF3F39BB29BB243F48043C3F360
:109960000B020AB943F001034FF496724A434FF4D5
:109970007A7192FBF1F2013292B243F400432284F5
:10998000C6E700BF40420F00A086010041F28832C6
:10999000044BC0E90023002383604FF4804383819C
:1099A000704700BF0000FFBF038819B143F00103F7
:1099B0000380704723F001031B041B0CF8E70388A6
:1099C00019B143F480730380704723F480731B0440
:1099D0001B0CF8E7038819B143F400730380704748
:1099E00023F400731B041B0CF8E7038819B143F43C
:1099F00080630380704723F480631B041B0CF8E72B
:109A000022B141F0010189B20182704701F0FE01EB
:109A1000F9E701827047008AC0B270470388B1F548
:109A2000006F1BBF23F400631B0443F400631B0C93
:109A300003807047838A008B43EA004321F07F4014
:109A40001840431A584258417047002382B000938F
:109A500001930B0F01900093009B21F07F4153B1C4
:109A6000019B14330193019B1B680B4214BF01201F
:109A7000002002B07047019B090C1833F2E7F8B5DB
:109A80000E46054680B14F1C384600F053FF044691
:109A900040B13A4600210EF0DCF932462946204614
:109AA0000EF0B3F92046F8BD0446FBE738B50D4685
:109AB000044628B10FF0C1F923462044834201D166
:109AC000002038BD13F8012BAA42F7D10120F8E796
:109AD00037B504460D460DF0A7FF002201A902602C
:109AE00020460FF0D7FA04460DF09EFF0368222BA4
:109AF00008D0019B1B782BB9002C03DB20462B6080
:109B000003B030BD012300202B60F9E72DE9F04FB1
:109B100005464FF0010B002687B0CDE9031206F190
:109B20000903122B8CBF0320022000F003FF0090DA
:109B3000E8B1324636490FF009F9039B53F82690F5
:109B4000EDB90024009800F0DFFEBBF1000F02D158
:109B5000284600F0D9FE84B1049B0136B342254665
:109B60004FF0000BDBD1204607B0BDE8F08FBBF112
:109B7000000F02D1284600F0C7FE0024F3E7254B72
:109B80004FF00008B9F1000F08BF994648460FF0A2
:109B900054F9019000980FF050F902902846494678
:109BA0000FF07AF9B8B928460FF047F9DDE901233B
:109BB00001309B1A08FB030000F0BCFE044600289D
:109BC000BFD003462F4618F1FF3809D23946184650
:109BD0000FF02BF9B6E7019B08F101081844DEE706
:109BE0004946384605930FF057F9059BA0EB070A45
:109BF0005246394618460FF03AF9009950440FF092
:109C000014F9019A029B9244C3185744DBE700BF42
:109C100074AB01087EBA010830B580B10346021F5B
:109C200000F1180452F8045F8D4208D0A242F9D125
:109C30001C301A4614680433013401D1116030BD60
:109C40008342F6D1FBE770B5044680B1064600EBCF
:109C50008105AE4204D12046BDE8704000F054BEFC
:109C600056F8040B0028F4D000F04EFEF1E770BD6A
:109C70002DE9F74F89460092002838D00027C45DAF
:109C80008CBB05468346264600EB070AD34538D1F0
:109C900004B10136002E6FD00137384600F04AFE7D
:109CA0008346002866D03A4600210EF0D2F8B00074
:109CB00000F040FE0446002860D04FF00008414606
:109CC000AA4532D131B15846FFF7D9FE002855D008
:109CD00044F82800584600F017FE009B1E602046FE
:109CE00003B0BDE8F08F0137B7F5807FC7D10024FE
:109CF0002646204600243146FFF7A5FF009B1C6046
:109D0000EDE79BF800304B4505D10CB1002401363E
:109D10000BF1010BBAE70EF02BF89BF8003018445A
:109D200043781B0758BF0134F2E72B784B4513D11A
:109D300081B15846FFF7A3FE00B308F1010344F8D0
:109D4000280000213A46584601930EF082F8019B04
:109D5000002198460135B3E701910EF009F82B7800
:109D600001991844407810F0080F04BF0BF8013037
:109D70000131EFE70446BCE73446B0E7584600F04F
:109D8000C3FDB6E72DE9F7430025064608208846BF
:109D900091461F46009500F0CDFD0446002868D08E
:109DA000C0E9005530460FF048F801280FD133784C
:109DB0002A2B0CD109F1FF33C4F8008063602268BC
:109DC0004A4502D263684B4543D32B4B0EE02D210D
:109DD0003046FFF76BFE0546C0B902A941F8040DF5
:109DE0003046FFF775FE019B63B1244B3B60009941
:109DF0002846FFF728FF002C37D0204600F084FDCE
:109E0000002432E0C4E900001D46D8E76A462D214F
:109E10003046FFF72DFF009B0546013B012B01D982
:109E2000174BE3E7002302AE46F8043D31460068D5
:109E3000FFF74EFE2060019B0BB1124BD6E7314677
:109E40006868FFF745FE6060019B002BB7D00E4BA2
:109E5000CCE7424501D3434501D20C4BC6E70099FC
:109E60002846FFF7F0FE00233B60204603B0BDE824
:109E7000F0830546BBE700BFD4C901084EC90108FD
:109E80006DC9010896C90108B5C90108F4C90108DE
:109E900038B590B1451E15F8014F0CB9204638BDB4
:109EA0000DF066FF23462044427802F00302022AA6
:109EB00008BFA4F120032B70EDE70120EFE708B500
:109EC00020B34A1C22D0062920D8DFE801F0040D77
:109ED000101316191C00002303600EF09DF80840B3
:109EE000431C5842584108BD00234360F5E7002356
:109EF0008360F2E700238361EFE70123C360ECE7AF
:109F000000230361E9E700234361E6E70120EAE774
:109F100070B506460D1F01F1180455F8041F4B1CBF
:109F200003D1A542F9D1002070BD3046FFF7C7FF2D
:109F30000028F6D0F8E708234A4291FBF3F302F039
:109F4000070201F0070158BF51420122DBB2C9B23A
:109F500002FA01F1C25C1143C154704708234A421E
:109F600091FBF3F302F0070201F0070158BF5142E1
:109F70000122DBB2C9B28A40C15C21EA0201C154AC
:109F80007047082391FBF3F3DBB2C05C4B4203F054
:109F9000070301F0070158BF5942C9B2084100F058
:109FA000010070472DE9F047089E8A4690461D46FD
:109FB000DDF82890074610B11446A24507D875B9B8
:109FC000012200240B9B1A602046BDE8F087214641
:109FD0003846FFF7D6FF002861D10134EDE7099B31
:109FE000023B042B04D8DFE803F0282C2C3034008B
:109FF0006B6801336B6028460EF00EF8013108BF24
:10A00000B0F1FF3FDCD031462846FFF758FF00286B
:10A01000D6D12FB3044621463846FFF7B2FF0028B9
:10A0200041D10134A245F6D10446013E042E19D88F
:10A03000DFE806F02B2D2F313300AB680133AB6026
:10A04000D9E7EB680133EB60D5E72B6901332B616E
:10A05000D1E76B6901336B61CDE7002DE5D1AFE747
:10A060003C46E2E72C6028460DF0D6FF013108BFE0
:10A07000B0F1FF3FA4D0B9F1000FA1D04946284666
:10A08000FFF746FF00289FD09AE76C60EBE7AC60D3
:10A09000E9E7AC61E7E7EC60E5E72C61E3E7A045C1
:10A0A000DBD1444690E7A045BFD1FAE700232DE974
:10A0B000F04F06468BB01C200C469046099300F0EA
:10A0C00039FC0546002800F0E4801C2000F032FC3A
:10A0D0000746002800F0DD804FF0FF31021F2B1FE4
:10A0E00005F1180043F8041F984242F8041FF9D103
:10A0F00000230121D4F800A00DF12409CDE900319D
:10A10000CDE902793C21234652463046FFF74AFF0B
:10A11000099900296ED1824502D12846FFF77CFDBE
:10A1200002234FF0010AD4F804B0CDE900A3CDE931
:10A13000025923465A463C2106F10800FFF732FF38
:10A14000099B002B56D183454CD151462846FFF739
:10A1500063FD03234FF0020AD4F808B0CDE900A351
:10A16000CDE9025923465A46182106F11000FFF79F
:10A1700019FF099B002B3DD1834546D15146284606
:10A18000FFF74AFD40F26F1BA3690593E368049350
:10A1900006F114030693DDF810A006F113030793EC
:10A1A00051460698FFF7EDFE28B105990798FFF78D
:10A1B000E8FE002836D1BBF1010B33D0E36820461E
:10A1C0000133E3600DF028FF013108BFB0F1FF3F1C
:10A1D00024D0A36929462046D4F80CA00593FFF7A4
:10A1E00097FEDDE7424621463046FFF75FFF0990C4
:10A1F0000028AED0284600F087FB17B1384600F0A3
:10A2000083FB09980BB0BDE8F08F424621463046EB
:10A21000FFF74CFF09900028ECD1B3E701234FF082
:10A22000000A0993099B002BE4D1049B534520D1DC
:10A2300004212846FFF7F0FC05230622D4F810A0DD
:10A24000CDE90032CDE90259234652460C2106F1F0
:10A250001800FFF7A7FE099B002BCBD18245C9D080
:10A260006369A3EB0803042B0CD94FF0FF33099368
:10A27000C0E7424621463046FFF718FF0990002804
:10A28000B8D1D9E7424621463046FFF70FFF099083
:10A29000B0E74FF0FF330993002DB2D00027A9E7B4
:10A2A0002DE9F04F002487B0924606AA894642F86D
:10A2B0000C4D2C219846109DFFF7DAFC074688B913
:10A2C0003E4B2B6003993846FFF7BDFC07B0BDE855
:10A2D000F08FD0F800B072685A451CD2304600F0BA
:10A2E00013FB0134039BA342ECD957F824602F21C0
:10A2F0003046FFF7DBFBA8B92B46304642465146B5
:10A30000FFF740FD2B680646002BE2D00028D9D08D
:10A3100000F0FAFAD6E759464846FFF70CFE0BF173
:10A32000010BD8E700232F21304604AA0493FFF73E
:10A330009FFC049906464B1E012B04D9204B2B6031
:10A34000FFF781FCBEE742462B4651460068FFF707
:10A3500019FD2A6883462AB108B100F0D5FA04999C
:10A360003046EDE72D213068FFF7A0FB18B908F162
:10A37000FF32CBF80420002306A941F8043D7068A1
:10A38000FFF7A6FB059A00901AB10E4A58462A60BC
:10A39000E3E7DBF80020DBF80410914205D23046F9
:10A3A0000499FFF750FC584699E711464846019238
:10A3B000FFF7C1FDDDE900321A44ECE719CA0108D4
:10A3C0002BCA010850CA01082DE9FF4100230E469F
:10A3D0000393144602B902AC236048B90546564BB4
:10A3E000236003992846FFF72EFC04B0BDE8F081F6
:10A3F00003AA2021FFF73CFC039B0546062B02D055
:10A400004E4B2360EDE71A22002130460DF021FD6E
:10A41000009400223C2331462868FFF741FF226860
:10A42000002ADED100943C2306F108016868FFF79A
:10A4300037FF2268002AD4D10094182306F11001B6
:10A44000A868FFF72DFF2368002BCAD16869FFF7C2
:10A450001FFD07223A496869FFF758FB80460EF056
:10A46000ECFC012806F1130706D198F800303F2BC9
:10A4700004BF2A2388F800300022082339464046CA
:10A480000094FFF70DFF404600F03EFA2268002AD4
:10A49000A7D107213846FFF774FD30B11146384681
:10A4A000FFF749FD0721FFF759FDEF6806F1140892
:10A4B00038460EF0C2FC012804D13B783F2B04BF84
:10A4C0002A233B7020230022414638460094FFF7A0
:10A4D000E7FE00214046FFF741FD2368002B80D1B5
:10A4E0002F693846FFF7D4FC00287FF47AAF38464E
:10A4F0000D221449FFF70AFB074600283FF471AF0D
:10A50000183600940D2301223146FFF7C9FE384664
:10A5100000F0FAF9012421463046FFF732FD30B150
:10A52000611E3046FFF707FD2146FFF717FD013496
:10A530000D2CF0D155E700BFF8C8010810C901087B
:10A54000E400002000010020F0B58DB0CDE900232B
:10A55000054628B94FF0FF304FF0FF310DB0F0BD88
:10A560002422002103A80DF074FC03A968460DF015
:10A570004FFB04460028EDD00DF04EFD4A1C08BFED
:10A58000B0F1FF3F06460F46E4D0626921462846F7
:10A59000FFF78CFD0028DDD120460DF03DFD4B1C62
:10A5A00008BFB0F1FF3FD5D08F4208BF864203D02D
:10A5B00020460DF031FDD1E72368204601332360AA
:10A5C0000DF02AFD013108BFB0F1FF3FC2D0626932
:10A5D00021462846FFF76AFD0028E9D0BAE770B5A2
:10A5E0003C258AB0DDE90E64019496FBF5F405FB89
:10A5F00014640294182493FBF4F505FB1433CDE99D
:10A600000330481E0C2190FBF1F301FB13010023E2
:10A61000CDE907339DF84030A2F26C7201A8059194
:10A62000069209930DF0F8FC0AB070BDF7B5044628
:10A6300002A860E902230DF0D9FA0269037A551CD9
:10A64000426990F804C0077B02F26C71067EC26911
:10A650000068A3700033207018BF01232046013228
:10A6600084F801C0E7702571A4F80510E671227224
:10A67000637203B0F0BD30B5457A85B0C478837895
:10A68000B0F8052001790295057801954078009091
:10A690002046FFF7A4FF05B030BD904271EB0303E5
:10A6A000B4BF012000207047032210B5104986B0C6
:10A6B0000B78013393FBF2F202EB42029B1A0D4A34
:10A6C0000B7052F823400278B0F8053004924278BB
:10A6D0001A21039282780292C2780192027920466E
:10A6E0000092054A0EF0FEFA204606B010BD00BFEB
:10A6F0005F0E0020FCCA0108BFCA0108B1F1004F7B
:10A7000008BF00281FB502460B4608D001A8FFF776
:10A710008DFF01A8FFF7C8FF05B05DF804FB0148F5
:10A72000FAE700BFF1CA01082DE9FF4703220D46F1
:10A730002B4900280B78044603F1010393FBF2F246
:10A7400002EB4202A3EB0203264A0B7052F823608D
:10A7500075F100033EDA4FF0010A444265EB45050E
:10A76000214A0023204629460CF070FF1E4A074666
:10A770000023204629460CF069FF104619464FF485
:10A78000616200230CF062FF4FF461628046002397
:10A79000204629460CF05AFF104619463C22002359
:10A7A0000CF054FF3C2281460023204629460CF041
:10A7B0004DFFCDF80080CDE901923B46BAF1000F84
:10A7C0000BD00A4A1A2130460EF08CFA304604B0FB
:10A7D000BDE8F0874FF0000AC2E7054AF2E700BF84
:10A7E0005F0E0020FCCA010880510100DDCA01088B
:10A7F000DECA01080FB404B0704700000FB437B5CB
:10A800001B4C256855B903222946012002F088FB1C
:10A810002B462A462946206002F0A6FB154D2A68E1
:10A82000013A03321ED86421206802F089FD80229B
:10A83000002111480DF00DFB07AB069A80210E4850
:10A8400001930EF097FE7F2803DD0C490C480EF0B3
:10A85000ECFA2B6808489847002320681A461946E6
:10A8600002F082FB03B0BDE8304004B0704700BF87
:10A87000E80E0020600E0020680E00203EE901086E
:10A88000E30E00200FB410B50D4CA2B02268013ABF
:10A89000033210D825AB249A802102A801930EF030
:10A8A00069FE7F2804DD07490DF183000EF0BDFA33
:10A8B000236802A8984722B0BDE8104004B0704752
:10A8C000640E00203EE9010870B50446054E4518A7
:10A8D000AC4200D170BD14F8011B3046FFF78EFF6B
:10A8E000F6E700BF08CB010838B50C461546FFF760
:10A8F00085FF20462946FFF7E7FFBDE838400148BD
:10A90000FFF77CBF7DBA010810B5044670B102F0B4
:10A910003DFA204602F028FA02F0E4F8BDE81040C3
:10A92000034A93880133938002F0FCB810BD00BF46
:10A93000A219002070B5234C8AB022680546013266
:10A94000226000283BD0632A1F4E0BDD03F0B8FDC8
:10A950000523002201A903F0F5FC03F0F1F900231F
:10A960003060236003F0ECF9336803F57A739842A2
:10A9700004D903F0E5F9002330602360134A144C36
:10A9800013781BB9236063600123137002F0FEF992
:10A99000284602F0E7F9064668B12A4600210DF084
:10A9A00058FA02F09FF823880133238002F0BAF8A6
:10A9B00030460AB070BD638801336380F8E706460D
:10A9C000F6E700BFF00E0020F40E0020EC0E002091
:10A9D000A2190020006800BA7047008840BA80B20F
:10A9E000704700687047837842781B04007843EA18
:10A9F000022318437047FFF7F4BFB0F90000704717
:10AA00000370130E4370130C8370130AC37002712A
:10AA1000052070470B0E03700B0C43700B0A8370FC
:10AA2000C170042070470B0A037041700220704708
:10AA30000B0A017043700B0C090E8370C170042067
:10AA40007047A0F14103052B02D83738C0B27047D8
:10AA5000A0F16103052B01D85738F7E73038C0B2B1
:10AA60000A2828BFFF2070470022013910B5014491
:10AA7000441E8C4204D014F8010F08B1002A01DAF8
:10AA8000104610BDFFF7DDFF0F2802D840EA021282
:10AA9000EFE74FF0FF32F3E738B505460C460EF00E
:10AAA0003FF8611B013190FBF1F303FB11002844D7
:10AAB00038BD000010B504460EF00EF8014B1C60C6
:10AAC00010BD00BF34010020024B1868013018602F
:10AAD0000EF002B83401002038B5451E15F8014FBC
:10AAE00004B938BD0DF044F923462044427802F001
:10AAF0000302012A08BF20332B70EFE72DE9F04154
:10AB000006460EF09AF930B3002734180DF030F9EC
:10AB100014F8013C354618444378621E19070DD4D9
:10AB20002F463B78A4EB050801355BB908F101021B
:10AB300039463046BDE8F0410DF072B904F8017CA9
:10AB40001446E3E70DF014F915F8013C1844437876
:10AB50001B07E5D4EAE7BDE8F08108B50EF05BF924
:10AB6000B0FA80F0400908BD0078013070470FB49A
:10AB700004B070472DE9FF470F46002104AC254E75
:10AB800044F8041D8046924630682246994602F0F9
:10AB900019FD0128039B31D13BB14FF080521E4B70
:10ABA0001A60BFF34F8FBFF36F8FB7F5C87F88BFB1
:10ABB0004FF4C87741463A4618480DF026F9184D2B
:10ABC000164B21463068AF802B60A5F806A085F8AB
:10ABD000089002F0D9FA039B3BB14FF080520E4B24
:10ABE0001A60BFF34F8FBFF36F8F0E48009400239E
:10ABF00001220421006803F031FE039B3BB14FF0BA
:10AC00008052054B1A60BFF34F8FBFF36F8F04B0B4
:10AC1000BDE8F087FC10002004ED00E0600F00208C
:10AC2000540F0020081100200348002301220221B4
:10AC3000006803F0A3BD00BF081100201FB503F09A
:10AC400085F80D4B04AA1860002342F8043D0092D9
:10AC500001220A481146006803F000FE039B3BB145
:10AC60004FF08052064B1A60BFF34F8FBFF36F8FC8
:10AC700005B05DF804FB00BF04110020081100209E
:10AC800004ED00E01FB5002304AA42F8043D0A4881
:10AC9000009280210122006803F0E0FD039B3BB19C
:10ACA0004FF08052054B1A60BFF34F8FBFF36F8F89
:10ACB00005B05DF804FB00BF0811002004ED00E0C2
:10ACC0001FB5104B1C680346A8B1002304AA42F824
:10ACD000043D009208210122204603F0BFFD039BA2
:10ACE0003BB14FF08052084B1A60BFF34F8FBFF358
:10ACF0006F8F04B010BD01220821204603F03EFDF5
:10AD0000F7E700BF0811002004ED00E01FB50023A5
:10AD100004AA42F8043D0A4800921021012200686A
:10AD200003F09CFD039B3BB14FF08052054B1A6032
:10AD3000BFF34F8FBFF36F8F05B05DF804FB00BF0B
:10AD40000811002004ED00E01FB500230C4904AAFF
:10AD500042F8043D08700B4800924021012200682F
:10AD600003F07CFD039B3BB14FF08052064B1A6011
:10AD7000BFF34F8FBFF36F8F05B05DF804FB00BFCB
:10AD8000440F00200811002004ED00E00048704747
:10AD90003C0F0020114810B5002303224FF48071AE
:10ADA000006803F0EBFC4FF080520D4B1A60BFF3CC
:10ADB0004F8FBFF36F8F0B4C206802F04FFC40B1F8
:10ADC000BDE81040002308481A461946006802F002
:10ADD000CBB8012003F00CF9EEE700BF081100200A
:10ADE00004ED00E000110020F8100020F8B5104B31
:10ADF0000146186802F0A4FA0446B8B14FF0805634
:10AE00000C4F0D4D002303224FF40071386803F0FE
:10AE1000B5FC2E60BFF34F8FBFF36F8F386802F021
:10AE2000FBFE2E60BFF34F8FBFF36F8F2046F8BD40
:10AE3000F81000200811002004ED00E0014B18601C
:10AE4000704700BFF010002070B5044678B1037859
:10AE5000032B0CD1436853B10025054E1868F269E5
:10AE600090476068F369056098476560257070BD1C
:10AE7000180F002010B50C480C4C00230522214669
:10AE8000006802F071F8012807D100236360084BC5
:10AE90001B683BB1BDE8104018472046BDE8104094
:10AEA000FFF7D2BF10BD00BFF4100020480F0020F4
:10AEB000F01000201FB5064C002201A9206802F006
:10AEC000ADF908B904B010BD01A8FFF7BDFFF3E765
:10AED000F4100020014B1868704700BFF4100020E8
:10AEE00010B50446064B010AA3F84A00202000F0E2
:10AEF00051FBE1B22120BDE8104000F04BBB00BF88
:10AF0000C419002008B5FFF7EBFF0122014B83F8BD
:10AF1000522008BDC4190020002238B50B4B05464D
:10AF20001D2083F84E100C4683F84C2000F08CFB5B
:10AF300020F0060040EA4401C9B21D2000F02AFBBF
:10AF40002946BDE83840232000F024BBC419002066
:10AF500013B5164C0120A3689847002341F6FE72F2
:10AF60000093009B934218DDA368022098470023BA
:10AF700041F6FE720193019B934212DD0C4BB52109
:10AF80001C6C4020A047A0214120A04700210120A7
:10AF9000234602B0BDE810401847009B01330093E0
:10AFA000DFE7019B01330193E5E700BF180F0020A5
:10AFB00018CB0108094B07B51B6CC2213B209847F1
:10AFC000002341F6FE720193019B934202DD03B020
:10AFD0005DF804FB019B01330193F5E718CB0108F1
:10AFE0002DE98748814B8248824E0360824B834C17
:10AFF0008360834BDFF834924360824BDFF830B2DA
:10B00000C360814B0361814B8361814BC3613368B2
:10B010009847002320681A46194601F0A5FF7D4B8A
:10B020001879F0B94FF0FF33194601AA03F05CFB21
:10B030000028F4D0019BD8051AD500F069FA002049
:10B0400000F0BCFDF36A9847FFF734FF0023D9F8FE
:10B0500000001A46194601F087FF002003F046F869
:10B06000DDE741F2883301AA4FF0FF310020DDE730
:10B0700099050DD500F04CFAFFF79CFFF36A98474D
:10B08000FFF718FF6421D9F8000002F059F9C6E76C
:10B09000D9F8000002F0E2FA0128C0D0DBF8003055
:10B0A00023B94FF4B6715C48F7F726FA019B1A06EC
:10B0B00004D50722594B1A70FFF7DCFE019B5B0792
:10B0C0004DD50021206802F03BF9012847D1DFF877
:10B0D00064A10C20DAF818309847054668B9034691
:10B0E00002460146206801F03FFF002897D140F258
:10B0F00081114948F7F700FA91E7DFF83C81DAF867
:10B100001830B8F804009847074678B9DAF81C30C8
:10B11000284698473B463A463946206801F024FFC6
:10B1200000287FF47CAF40F28911E2E708F10403C4
:10B1300003CB2F606860A9603846D8F80010B8F8D3
:10B1400004200CF062FE0322344B1A705D60FFF79E
:10B1500091FE002320681A46194601F005FF019B65
:10B16000DF0709D501222D4B1A7000225A602C4AA4
:10B1700012689A60FFF77EFE019BDD0606D5052268
:10B18000264B1A7000225A60FFF774FE019B1807C5
:10B1900006D50422214B1A7000225A60FFF76AFE7E
:10B1A000019B990706D502221C4B1A7000225A6097
:10B1B000FFF760FE019B9A0606D50622174B1A7010
:10B1C000184A5A60FFF756FE019B5B067FF527AFD2
:10B1D000154B1A78114B32B108221A7000225A60AE
:10B1E000FFF748FE1BE70922F7E700BF3DAC000868
:10B1F000F80E002018CB010875AB0008FC100020E9
:10B2000029AC0008C1AC00080DAD000849AD00082C
:10B2100085AC00083C0F00207EBA0108480F0020D2
:10B2200004110020450F0020440F002000110020D1
:10B23000F4100020180F0020540F0020044B10B50C
:10B240005B6998470446FFF783FE204610BD00BFA8
:10B2500018CB0108F0B5674C054626460F46182264
:10B26000002185B064480CF0F4FD0FCD0FC695E8C1
:10B270000F0086E80F0097E8030063695F4D013B0C
:10B28000033388BF5E4B85E8030088BF6361636852
:10B29000013B033304D94FF431715A48F7F72CF9C5
:10B2A0002368013B033304D94FF432715548F7F753
:10B2B00023F9A368013B033304D94FF43371514898
:10B2C000F7F71AF9E368013B033304D94FF43471FB
:10B2D0004C48F7F711F92369013B033304D94FF4C4
:10B2E00035714848F7F708F9E369013B033304D99E
:10B2F0004FF436714348F7F7FFF8A369013B033376
:10B3000004D94FF437713F48F7F7F6F83E4B0FCBAF
:10B310008DE80F0094E80F0000F0D0F823689847FC
:10B32000FFF716FE394B42205B6C9847222807D066
:10B3300040F2EE213348F7F7DFF8002005B0F0BD0A
:10B3400003220021012001F0EBFD314B18600120A8
:10B3500001F0AEFE2F4B186020B94FF43E71294822
:10B36000F7F7CAF803220021012001F0D9FD2A4C89
:10B37000206020B94FF43F712248F7F7BDF8002351
:10B3800020681A46194601F0EFFD20B940F2FD2170
:10B390001C48F7F7B1F84FF0FF31206801F0D0FFFB
:10B3A00000220C21032001F0BBFD1C4B186010B9DA
:10B3B00040F20331BEE71A4B1A4A1A602B680BB9E8
:10B3C00004232B60184B1C680CB10120B6E70193D5
:10B3D0002B68FA22009315490123154802F06EFAF2
:10B3E0000128F2D0074840F21531F7F785F82046DA
:10B3F000A4E700BF180F0020AC1900203C0F00206C
:10B400006FAB00087EBA0108280F002018CB010896
:10B41000FC100020F810002000110020F410002083
:10B42000380F002069AB0008081100200ECB01087E
:10B43000E1AF0008014B83F828007047C4190020D1
:10B44000014B1860704700BF380F002070B5084CE2
:10B45000054622680E4622B940F225310548F7F725
:10B460004BF8236831462846BDE87040184700BFB6
:10B47000380F00207EBA010800F03AB8012070476A
:10B4800008B5FFF783FC4379002B0CBF8020002018
:10B4900008BD0000002310B5074951F83340DA0019
:10B4A000844203D80A449468844203D80133152B9C
:10B4B000F3D1FEE7107910BD88CB010884B030B518
:10B4C00003AC84E80F00064C03AD0FCD0FC495E824
:10B4D0000F0084E80F00BDE8304004B0704700BFA3
:10B4E00038140020014B1878704700BFC4190020A1
:10B4F000C82307B50093002304481A4603210068B7
:10B5000003F0DEFA03B05DF804FB00BF1011002069
:10B5100013B5104C0120A368984700230093009BAB
:10B52000B3F5CC7F0FDDA36800209847002342F6D7
:10B53000FE720193019B934208DD0220A36802B0D2
:10B54000BDE810401847009B0133E7E7019B01333A
:10B550000193EFE7381400202DE9F04107460C4C29
:10B560000D46E368002016469847236947F080009F
:10B570009847013D2E44B54204D1E3680120BDE85F
:10B58000F0411847236915F8010F9847F3E700BF0A
:10B590003814002007B502AB03F8011D012219463B
:10B5A000FFF7DAFF03B05DF804FB000000000000C5
:10B5B000134A10B55060134A904219D00BF0A8F905
:10B5C0000DA3D3E900230BF047FB0BF0B5FC0446B9
:10B5D000C4F307410620FFF7DDFFC4F3072107206E
:10B5E000FFF7D8FFE1B20820BDE81040FFF7D2BF57
:10B5F000054CEDE7AFF300800000000080844E4072
:10B60000C4190020F01FCB33CD3CD9002DE9F04107
:10B6100007460C4C0D46E368002016469847236900
:10B6200007F07F009847013D2E44B54204D1E368FE
:10B630000120BDE8F041184723690020984705F82C
:10B64000010FF2E73814002007B501220DF10701C0
:10B65000FFF7DCFF9DF8070003B05DF804FB000076
:10B6600001282DE9F84F0D4603D0022854D00020C0
:10B670004BE06D4E2720B48BFFF7E6FFA4B220F01D
:10B68000F800013420440BF043F9B37F0022002B73
:10B690003DD1664B0BF000F8804630208946FFF71D
:10B6A000D3FF30F0F9030CBF0023604B002240466B
:10B6B00049460AF0F1FF8046284689460BF038F9E2
:10B6C00002460B46404649460AF0E6FF96F820300F
:10B6D0000022F3B900230AF0DFFF0022544B0BF0E5
:10B6E00091F9B669044630460D460BF011F9024651
:10B6F0000B46204629460BF0AFFA00224D4B0BF0CB
:10B7000081F90AF075FF0BF017FCBDE8F88F0023F4
:10B71000C0E74FF08043DEE7434C226C022A79D821
:10B72000454B03EBC203D3E900670120636C9840EB
:10B730000BF0FEF802460B46304639460BF08CFA09
:10B7400002460B46002039490BF086FA06460F46A2
:10B75000B4F84A000BF0ECF80022384B0AF09CFFDA
:10B7600032463B460BF04EF98B46616C824694F8AC
:10B770004E0094F84C308900002BC1F11C0101EB04
:10B78000001114BF1420002001EBC501081A0BF0B2
:10B79000BFF88046606C94F848308946002B14BF8F
:10B7A00002230023C3EB80000BF0B2F802460B46E5
:10B7B000404649460BF050FA0AF00EFE8046894694
:10B7C00094F8490004300BF0B3F842464B460BF0B6
:10B7D00019F90022002304460D460BF0A3FBE0B14B
:10B7E0000022134B204629460AF056FF32463B46BC
:10B7F0000BF008F952465B460AF04EFF00220D4B53
:10B800000BF000F906A3D3E900230AF045FF0AF084
:10B810006BFE78E70026002787E700200449E5E76C
:10B820002B8716D9CEF7EF3FC41900200000F03F58
:10B830000000204000408F4070CB01080000114004
:10B84000012808B504D002280AD04FF0FF3006E0E6
:10B850001120FFF7F9FEC0F34700404200B208BDD7
:10B860001B20FFF7F1FE8B38F8E700000B4B10B5FB
:10B870005B68044660B9022098470120FFF7E4FEA8
:10B8800000F0F80121430120BDE81040FFF782BE1F
:10B8900003280CBF01200020EEE700BF3814002071
:10B8A00013B5C82400230B4800941A4603210068EE
:10B8B00003F006F90023084800941A4603210068A3
:10B8C00003F0FEF80020FFF7D1FF0022034B1A70AF
:10B8D00002B010BD1011002034140020C419002043
:10B8E00013B5C82400230B4800941A4603210068AE
:10B8F00003F0E6F80023084800941A460321006884
:10B9000003F0DEF80120FFF7B1FF0022034B1A70AD
:10B9100002B010BD1011002034140020C419002002
:10B9200073B55D4C06466378DBB2012B03D0022B66
:10B9300065D0002538E0402094F82250FFF784FEBF
:10B940000C214020FFF726FE4120FFF77DFE60F02E
:10B950000E01C9B24120FFF71DFE3520FFF774FE2E
:10B9600000F0C00141F020013520FFF713FE352023
:10B97000FFF76AFE00F03F00112184F83A003F20F3
:10B98000FFF708FE00230D2084F82C3084F82D30BA
:10B990002387E386FFF758FE00F04001EDB241F047
:10B9A0002E010D20FFF7F6FD4FF4C87200213B4831
:10B9B0000CF04FFA01232370394B18684FF0FF3316
:10B9C000002E5BD04FF47A7101FB06F20093B2FBBC
:10B9D000F1F20023042103F073F86378012B52D1B4
:10B9E0000520FFF743FF0D20FFF72EFE40F020015A
:10B9F0000D20C9B202B0BDE87040FFF7CBBD94F88E
:10BA0000513033201BB3FFF71FFE40F04101C9B294
:10BA10003320FFF7BFFD19213B20FFF7BBFD94F852
:10BA2000525094F84F30EDB2E3B11D211120FFF7D1
:10BA3000B1FD4020FFF708FE00F033014020FFF782
:10BA4000A9FD00210F20FFF7A5FD0021A9E7FFF7C1
:10BA5000FBFD00F0BE0141F001013320FFF79AFD2C
:10BA60001D21D9E70F211120FFF794FD4020FFF79A
:10BA7000EBFD00F03C0141F00101DFE700933246AD
:10BA800033460321A7E72DB1052002B0BDE8704081
:10BA9000FFF7ECBE0620F8E7C419002014110020BF
:10BAA0001011002037B54FF47A72642350432B4DA8
:10BAB000B0FBF2F2009304210023286803F000F8A1
:10BAC0000022274B274C1A706378DBB2012B14D06D
:10BAD000022B26D0022323702C6802F031F90523B3
:10BAE0000246009301210023204602F0E9FF0320D3
:10BAF00003B0BDE83040FFF7B9BE14214020FFF786
:10BB000049FDB0214120FFF745FD8F213520FFF78A
:10BB100041FD3520FFF798FD00F03F0084F83A0022
:10BB2000D8E794F84F3073B1F5211120FFF732FDBB
:10BB30004020FFF789FD00F0330141F04001402033
:10BB4000FFF728FDC6E7F7211120FFF723FD40206E
:10BB5000FFF77AFD00F03F01EFE700BF341400204B
:10BB600058140020C419002010B5124C6378DBB2C1
:10BB7000012B04D0022B09D040F2134101E04FF415
:10BB80007F71BDE810400C48F6F7B6BCFA211120D1
:10BB9000FFF700FD4020FFF757FD00F0FC014020BB
:10BBA000FFF7F8FC032307202370BDE81040FFF7E0
:10BBB0005DBE00BFC41900207EBA010808B51A4B4B
:10BBC0005A7882422ED058705B780020022B13D016
:10BBD000FFF74CFE0120FFF737FD00F07F01012049
:10BBE000FFF7D8FC00214020FFF7D4FC3021412092
:10BBF000BDE80840FFF7CEBCFFF738FE0120FFF795
:10BC000023FD60F07F01C9B20120FFF7C3FC0021D2
:10BC10004020FFF7BFFC00214120FFF7BBFC432180
:10BC20003120E5E708BD00BFC41900201D4B13B546
:10BC3000186000231C4C1A4600944FF47A711B487C
:10BC400002F01CFF1A4B186020B94FF48671194896
:10BC5000F6F752FC002300941A464FF47A71164806
:10BC600002F00CFF154B186020B94FF48771114892
:10BC7000F6F742FCFFF74CFC0020FFF79FFF002087
:10BC8000FFF7F4FD4FF4C87200210D480CF0E1F805
:10BC9000002201210B4B83F8282083F829101A7009
:10BCA00002B010BD0C1100206DC2000838CC010894
:10BCB000341400207EBA01083BCC0108101100208A
:10BCC00014110020C419002073B50E461446054611
:10BCD000FFF774FF3046FFF76BFC0520FFF7C6FD4A
:10BCE00000230193019BB3F5CC7F0BDD2846FFF7C2
:10BCF000A7FD0546FFF7D4FDA542CCBF00200120DB
:10BD000002B070BD019B0133EBE773B50024022044
:10BD1000FFF754FFFF211120FFF73CFC0520FFF740
:10BD2000A5FD254626460196019BB3F5CC7F0DDD8A
:10BD30002C20FFF789FC00F00100A0400134202CEA
:10BD400045EA0005EFD1284602B070BD019B0133E2
:10BD50000193E9E7000000002DE9F04F824687B02B
:10BD60000093109B0D4601939DF85C309DF8581090
:10BD7000029393469DF864309DF8602003930492EB
:10BD8000BDF84460BDF848409DF84C709DF8508067
:10BD90009DF854900591FFF711FFDDE90332BAF1E8
:10BDA000010F06D0BAF1020F059968D007B0BDE8BF
:10BDB000F08F7F4C019925615846C4F818B0616135
:10BDC000A77784F81F8084F8209084F8212084F8D5
:10BDD0002230A6830AF09CFD02460B4672A1D1E9EF
:10BDE00000010AF039FF0BF0A7F81FFA80FB4FEAB9
:10BDF0001B210220FFF7CEFB5FFA8BF10320FFF738
:10BE0000C9FB2846FFF746FB01461220FFF7C2FB9D
:10BE10000198FFF73FFB01461320FFF7BBFB310AF8
:10BE20002520FFF7B7FBF1B22620FFF7B3FBE27F37
:10BE30002346DAB9A27FCAB184F829A0414632204C
:10BE4000FFF7A8FB3020FFF7FFFB002F14BF0021F6
:10BE5000802100F06F0040EA0919302041EA090111
:10BE6000C9B207B0BDE8F04FFFF794BB00224FF412
:10BE7000D271504883F82920F6F73EFBDEE74C48A4
:10BE80009DF800C00564C0F844B080F849C0A0F82F
:10BE90004A6080F84C7080F84D8080F84E9080F8B1
:10BEA0004F109DF80810BBF10C0F80F8501082461F
:10BEB00080F8512080F8523072D8BBF1050F60D95C
:10BEC00025B9ABF10B03012B5DD804E0012D5AD14C
:10BED000BBF10C0F57D101238AF848301D20FFF722
:10BEE000B3FB9AF84810009B41EA490141EA8701F7
:10BEF00041EAC30141EA8511C9B21D20FFF74AFB9F
:10BF00001E20FFF7A1FBC4F3012100F00C00014348
:10BF100041EA0B11C9B21E20FFF73CFBE1B21F2022
:10BF2000FFF738FB310A2020FFF734FBF1B2212064
:10BF3000FFF730FB1FB141462220FFF72BFB9AF899
:10BF40004F306BB14B20FFF77FFB60F07F01C9B230
:10BF50004B20FFF71FFB9AF850102420FFF71AFB25
:10BF6000BBF1060F4FF031000FD1FFF76DFB00F072
:10BF7000F80141F005013120FFF70CFB0C213720BF
:10BF80006FE74FF0060B0023A6E7FFF75DFB00F01D
:10BF9000F80141F003013120FFF7FCFA0A21EEE736
:10BFA0004FF00C0B012D8FE70000000080847E41D4
:10BFB000C41900207EBA01082DE9F04F89B01E4651
:10BFC0009DF84C300C4602939DF85C30019205932D
:10BFD0009DF86030009006939DF86430129D0393A5
:10BFE0001A9BBDF8507004939DF854809DF85890AA
:10BFF000FFF7E4FD0920FFF727FB82465A20FFF7F1
:10C0000023FB0AF07F01DFF860A28346DAF8040020
:10C010000791FFF735FA07990843C0B2030600F00D
:10C02000F00C2ED5112CCBBF4BF007020BF0F80211
:10C030005FFA82FB42F0040B0BF00701072918D1CD
:10C04000142CA8BF1424052CB8BF0524611F4CEA8A
:10C050000101C9B20920FFF79DFA59465A20FFF79E
:10C0600099FA009B012B13D0022B6CD009B0BDE8CC
:10C07000F08F112CA8BF1124022CB8BF0224A11EDE
:10C08000E5E70E2CA8BF0E2444EAE474611CDEE749
:10C09000019B8AF80840CAF80C309DF80C30CAF8A9
:10C0A0001060CAF81850AAF81C708AF81E808AF826
:10C0B00020908AF82130049B0198CAF824300AF0B5
:10C0C00027FC65A3D3E900230AF0C6FD0AF034FF7C
:10C0D00084B2210A0420FFF75DFAE1B20520FFF7E0
:10C0E00059FA28460AF014FC02460B465CA1D1E935
:10C0F00000010AF0B1FD0AF01FFF84B2210A0220FC
:10C10000FFF748FAE1B20320FFF744FA390A252085
:10C11000FFF740FAF9B22620FFF73CFA3020FFF78C
:10C1200093FAB8F1000F0CBF8021002100F06F00DE
:10C1300040EA0919302041EA0901C9B209B0BDE855
:10C14000F04FFFF727BA484A9DF8083082F83C4084
:10C150001664556482F849309DF81430A2F84A708C
:10C1600082F84C8082F84F309DF818300C2D82F800
:10C1700050309DF80C3082F84E9082F85130049B7C
:10C180001446536562D8052D52D926B9A5F10B0284
:10C19000012A4ED803E0012E4BD10C2D49D10122AA
:10C1A00084F8482094F84F206AB14B20FFF74CFAEE
:10C1B00060F07F01C9B24B20FFF7ECF994F8501002
:10C1C0002420FFF7E7F91D20FFF73EFA9AF8481000
:10C1D000029B41EA490141EA880141EAC30141EA7F
:10C1E0008611C9B21D20FFF7D5F91E20FFF72CFAE2
:10C1F00000F00F0141EA0511C9B21E20FFF7CAF98C
:10C20000390A2020FFF7C6F92120F9B2FFF7C2F959
:10C21000062D4FF031000ED1FFF716FA00F0F801AD
:10C2200041F005013120FFF7B5F90C21372085E7F2
:10C2300006250022B4E7FFF707FA00F0F80141F005
:10C2400003013120FFF7A6F90A21EFE70C25012EA3
:10C250009FE700BFAFF300800000000080844E40E5
:10C260000000000080847E41C419002010B5254CD8
:10C270002378DBB2012B02D0022B34D010BD6378BF
:10C28000012B29D100230B213E2084F82C3084F887
:10C290002D302387E386FFF77DF910213F20FFF73C
:10C2A00079F994F8223003F0FF029BB10D20FFF7DB
:10C2B000CBF940F02001C9B20D20FFF76BF9124B0A
:10C2C0001B68002BDAD0DB68002BD7D0BDE810400C
:10C2D000002018472270F2E794F85230002BEED07D
:10C2E000FFF7FEFAEBE7002301222370074B1A70D9
:10C2F000054B1B68002BC1D05B68002BBED0BDE88E
:10C3000010401847C41900200C11002058140020B8
:10C3100007B50022154B8DF8072083F82C2083F8F1
:10C320002D201A87DA8683F82E2093F8223023B93D
:10C3300003B05DF804EBFFF7B3BA3F20FFF784F9D1
:10C340008DF807009DF80730DB0603D510213F204C
:10C35000FFF720F90D20FFF777F940F040010D209D
:10C36000C9B203B05DF804EBFFF714B9C41900209B
:10C370002DE9F04107460D4C0D46E36800201646B6
:10C380009847236907F07F009847013D2E44B54246
:10C3900004D1E3680120BDE8F0411847236900207B
:10C3A0009847C04305F8010FF1E700BF381400209B
:10C3B0000A4601460020FFF7CFB80000F7B5554CFC
:10C3C000064663780D46DBB2012B04D0022B34D035
:10C3D000002528461AE0002323878BB2E386A37F3B
:10C3E00013B13220FFF7D6F86B1E3F2B1BD884F811
:10C3F0003B500025304694F83B10FFF7D9FF94F8E6
:10C400003B30228F13449BB22387606AFFF74AFBBD
:10C410006378012B7BD1002D79D03F4E3F4D33788F
:10C42000002B4DD073E02A4631463C480BF0EDFC22
:10C430003C23012584F83B30DCE794F8513033206D
:10C440002BB3FFF701F900F0BE013320FFF7A2F88C
:10C4500019213B20FFF79EF82946222084F85C50E2
:10C46000FFF798F800210E20FFF794F800210D2027
:10C47000FFF790F80120FFF7E7F830F0F80711D048
:10C4800029463046FFF794FF0025606DBEE7FFF7B1
:10C49000DBF800F0BE0141F001013320FFF77AF82C
:10C4A0001D21D6E7FFF71CFA0197019BB3F5CC7F5E
:10C4B000E6DC019B01330193F7E7012001F098FDD1
:10C4C0003F20FFF7C1F88306F7D4E38E218F94F85D
:10C4D0003B205B1A9342208F0BDD94F83B102844DD
:10C4E000FFF766FF94F83B30228F13449BB22387FB
:10C4F00095E7E18E238F2844C91AC9B2FFF758FF88
:10C50000E18E228F238F0B449B1A9BB2238703B0AB
:10C51000F0BD00BFC41900205814002014110020E1
:10C520000A4601460020FFF771B80A46014600207E
:10C53000FFF71EBF38B505460C46FFF73FFB012D40
:10C5400002D0022D0AD038BD064B9B7F002BFAD1BA
:10C5500021463220BDE83840FFF71CB82146232091
:10C56000F8E700BFC419002001230022F0B5684E8F
:10C5700085B0684D33608DF80B202B780392DBB2C9
:10C58000012B2C4606D0022B00F0A0800023336044
:10C5900005B0F0BD6B78DBB2012B34D0022BF5D1A6
:10C5A00040211220FEF7F6FF1220FFF74DF88DF81C
:10C5B0000B009DF80B30584F13F0200F29D020218D
:10C5C0001220FEF7E7FF95F8523003F0FF0203B99F
:10C5D0002A7000225148009203AB0821006802F043
:10C5E0006FFA039B3BB14FF080524D4B1A60BFF383
:10C5F0004F8FBFF36F8F3B68002BC7D01B69002B99
:10C60000C4D09847C2E740F21F514648F5F774FF7F
:10C61000BCE71920FFF718F840B285F8580095F8E4
:10C62000583095F858501B0642BF6DB26D42C5F3A5
:10C6300085054FF01A004CBF6D42AD08FFF704F8B6
:10C64000002D40F30B13B8BF40198B389BB2034445
:10C650001BB2A4F85A301320FEF7F6FF84F85C00F2
:10C660001020FEF7F1FF01460D20FEF793FF94F82E
:10C670005C102D48FFF754FF94F8523003F0FF028E
:10C680008BB926482270009203AB0821006802F0A3
:10C6900017FA039B3BB14FF08052214B1A60BFF356
:10C6A0004F8FBFF36F8F3B68002B3FF46FAF9D68D8
:10C6B000002D3FF46BAF94F85C10B4F85A2094F856
:10C6C000583012B25BB21848A8475FE7134800928F
:10C6D00003AB0821006802F0F3F9039B3BB14FF074
:10C6E00080520F4B1A60BFF34F8FBFF36F8F637889
:10C6F000022B03D108211220FEF74CFF00232370E8
:10C70000054B1B68002B3FF441AF1B6877E700BF68
:10C71000AC190020C41900200C11002010110020B9
:10C7200004ED00E07EBA010814110020012300226C
:10C730002DE9F0435F4D85B05F496B608DF80B20AC
:10C740000B780392DBB2012B2F460C4605D0022B4F
:10C7500000F0AD8000237B6031E04B78DBB2012B31
:10C7600022D0022BF6D15548009203AB0821006875
:10C7700002F0A6F9039B3BB14FF08052504B1A6078
:10C78000BFF34F8FBFF36F8F80211220FEF702FFA0
:10C79000002323704B4B1B68002BDBD0DB68002B86
:10C7A000D8D001209847D5E73F20FEF74DFF8DF800
:10C7B0000B009DF80B3013F0200303D16B6005B024
:10C7C000BDE8F0839DF80B30DB0605D53E48FEF74B
:10C7D00059F8FFF79DFDBDE794F8293023B940F2E1
:10C7E000D3513A48F5F788FE94F82830022B2DD122
:10C7F000238F374894F83A101844FFF796FE238F9A
:10C800009BB2002B40D094F83A30228F13449BB255
:10C810002387238FE28E9A429CD8E28E2C492D48A2
:10C820000BF0F3FA94F82E50E48EFFF771FD254BD0
:10C830006DB21B68A4B2002B8CD09E68002E89D0EC
:10C8400000232A4621462348B04783E7224D002093
:10C85000EB6898472B69002098474FF00008DFF8F5
:10C86000709094F83A30434503DCEB680120984718
:10C87000C5E72B690020268F9847B6B24E4406F8CC
:10C88000080008F10108ECE794F82D30002BA0D047
:10C8900094F83A100E48FEF7D9FDE086E38EB3F522
:10C8A000C87F96D2E38E9BB2002B92D0ABE74B7839
:10C8B00050E700BFAC190020C4190020101100205F
:10C8C00004ED00E00C1100203ECC01087EBA010806
:10C8D00014110020A41200203814002038B50123C0
:10C8E0001B4D1C4CAB602378DBB2012B04D0022B18
:10C8F0002AD00023AB6038BD6178C9B2012916D0B7
:10C900000229F6D194F84F30002BF2D01220FEF716
:10C9100041FE114B1B68002BEBD05C69002CE8D06A
:10C920001C20FEF791FE00F03F00A047E1E7002346
:10C930001120238784F82D10FEF786FE4008404220
:10C9400040B284F82E00D4E76178C9B2D8E700BFBE
:10C95000AC190020C41900200C110020F8B50126E4
:10C96000204C214BE6605A78022A05D11B78DBB2B5
:10C97000B34204D0032B14D00023E360F8BD12208F
:10C98000FEF762FEC306F7D510211220FEF702FE65
:10C99000164B1B68002BEFD0DB69002BECD09847BF
:10C9A000EAE71220FEF750FE10F001070F4D0CD001
:10C9B00005211220FEF7EEFD2B68002BDCD09B69D1
:10C9C000002BD9D030469847D6E704211220FEF735
:10C9D000E1FD2B68002BCFD09B69002BCCD03846D3
:10C9E000F1E700BFAC190020C41900200C11002091
:10C9F000012210B5094C2261094A5178012909D157
:10CA00001378DBB2012B05D102213E2082F82C30B5
:10CA1000FEF7C0FD0023236110BD00BFAC1900204C
:10CA2000C41900200122034B5A61034A52780022A4
:10CA30005A617047AC190020C419002006480068EC
:10CA4000006880F3088862B661B6BFF34F8FBFF30A
:10CA50006F8F00DF00BF000008ED00E0002307B586
:10CA600001930B4B1B68013303D0CA210948F5F72A
:10CA700043FD4FF0500383F31188BFF36F8FBFF373
:10CA80004F8F019B002BFCD003B05DF804FB00BF6F
:10CA9000380100207EBA01084FF0807340F8043C52
:10CAA000054B21F0010140F8081C40F80C3C40F80F
:10CAB000202C4038704700BF5DCA0008000000000D
:10CAC000074B19680868B0E8F00F80F30988BFF3D6
:10CAD0006F8F4FF0000080F311884EF00D0E7047FD
:10CAE000641400204FF0500383F31188BFF36F8F5D
:10CAF000BFF34F8F084A13680133012B136009D12C
:10CB0000064B1B6813F0FF0F04D040F27511044868
:10CB1000F5F7F2BC704700BF3801002004ED00E0DB
:10CB20007EBA010810B5074C236823B94FF4BE71D3
:10CB30000548F5F7E1FC2368013B23600BB983F35B
:10CB4000118810BD380100207EBA010800000000E5
:10CB5000EFF30980BFF36F8F0D4B1A6820E9F00FD8
:10CB600010602DE908404FF0500080F3118801F06B
:10CB700065FA4FF0000080F31188BDE8084019689D
:10CB80000868B0E8F00F80F30988BFF36F8F704733
:10CB90006414002008B54FF0500383F31188BFF3ED
:10CBA0006F8FBFF34F8F01F0DFF818B14FF0805255
:10CBB000024B1A60002383F3118808BD04ED00E0E6
:10CBC0000022054B05491A600A6041F26701044AD8
:10CBD000116007221A60704710E000E018E000E0E2
:10CBE00014E000E013B5264B264C1A78D2B201921D
:10CBF000FF221A701B78244ADBB28DF803309DF8AF
:10CC0000033003F0500313700723002223609DF8C4
:10CC10000310581E090629D402B123602368032B90
:10CC200004D04FF49B711948F5F766FC2368144A49
:10CC30001B0203F4E06323600024019BDBB213704A
:10CC4000134B1A6842F470021A601A6842F070427C
:10CC50001A60FFF7B5FF0F4B1C60FFF7EFFE01F006
:10CC6000EDF9FFF7FBFE204602B010BD9DF8033042
:10CC700001225B00DBB28DF803300346C7E700BF3B
:10CC800000E400E05C140020591400207EBA010882
:10CC900020ED00E03801002008B5EFF305830F2BED
:10CCA0000AD90D4A9B5C0D4A12789A4204D940F287
:10CCB000A5210B48F5F720FC0A4B0B4A1B681268AC
:10CCC00003F4E063934206D9BDE8084040F2B52181
:10CCD0000348F5F711BC08BDF0E300E0591400204B
:10CCE0007EBA01080CED00E05C14002070B50D4622
:10CCF000064601F01DF80D4B0D491C6862198A4269
:10CD000007D90C23336001F0BFF84FF0FF34204601
:10CD100070BD1A60074A13685B1B1360064A1368EC
:10CD20002B44136001F0B0F8F1E700BF3C01002094
:10CD3000506A0020400100206014002008B5EFF385
:10CD400005831BB1C2210348F5F7D6FBBDE80840B7
:10CD500000F0EEBF7EBA010801F096B800F0E8BF1F
:10CD600001F092B80BF012B80BF018B800B58BB008
:10CD700068460BF00BFB034B08981B6818440BB07C
:10CD80005DF804FB4001002000207047704710B59B
:10CD90000446FFF7A7FEA46BFFF7C4FEB4FA84F0C5
:10CDA000400910BD70B51546026C0446866B42B949
:10CDB00005689DB9806801F0EBFBA5600136A663AC
:10CDC00070BD6DB940680BF020F86368226C1344A5
:10CDD000A2686360934201D3236863600020EDE79B
:10CDE000C0680BF012F8236CE2685B4221681A44B9
:10CDF0008A42E2603EBFA2689B18E360022DEDD13B
:10CE00000EB1013EEAE73046D8E703461A6C10B48B
:10CE1000084662B1D9689C681144A142D96028BF14
:10CE2000196810BC28BFD960D9680AF0EEBF10BCE1
:10CE3000704770B50446FFF755FE94F8455004F16D
:10CE400024066DB2002D14DCFF2384F84530FFF773
:10CE500069FEFFF747FE94F8445004F110066DB2E6
:10CE6000002D12DCFF2384F84430BDE87040FFF74A
:10CE700059BE636A002BE7D0304601F0DBF908B1F8
:10CE800001F05AFA013D6DB2DCE72369002BE9D0CD
:10CE9000304601F0CFF908B101F04EFA013D6DB214
:10CEA000DEE7000038B50D46044620B940F2031114
:10CEB0001948F5F721FBFFF715FED4E90F314B4375
:10CEC0002268D0185B1A1344A060E3600020FF239F
:10CED000A063626084F8443084F8453095B92369D2
:10CEE00063B104F1100001F0A5F938B14FF08052A0
:10CEF0000A4B1A60BFF34F8FBFF36F8FFFF712FE1D
:10CF0000012038BD04F1100001F01AFF04F12400E3
:10CF100001F016FFF2E700BF7EBA010804ED00E061
:10CF2000F8B50D461746064620B94FF4BB710D48BB
:10CF3000F5F7E2FA05FB06F05030FFF713FF044661
:10CF400048B155B92060C4E90F6501212046FFF7BB
:10CF5000A9FF84F84C702046F8BD00F1500303602F
:10CF6000F1E700BF7EBA01082DE9FF47884601922C
:10CF70001E46044620B940F2F1214B48F5F7BCFAB1
:10CF8000B8F1000F06D1236C23B140F2F2214648DC
:10CF9000F5F7B2FA022E07D1E36B012B04D040F271
:10CFA000F3214148F5F7A8FA01F090FA30B9019B56
:10CFB00023B140F2F6213C48F5F79EFA0027B94626
:10CFC000DFF8E8A0FFF78EFDA26BE36B9A4201D376
:10CFD000022E19D1324641462046FFF7E3FE636A2E
:10CFE0001BB104F1240001F025F938B14FF0805253
:10CFF0002E4B1A60BFF34F8FBFF36F8FFFF792FD79
:10D00000012004B0BDE8F087019D1DB9FFF78AFD3E
:10D010000020F6E717B902A801F04CF9FFF782FDEE
:10D0200000F086FEFFF75EFD94F84430FF2B08BF4A
:10D0300084F8449094F84530FF2B08BF84F845905D
:10D04000FFF770FD01A902A801F040F928BBFFF726
:10D0500049FDA26BE36B9A420ED1FFF763FD019984
:10D0600004F1100001F0ACF82046FFF7E2FE00F0FA
:10D070000BFF48B10127A5E7FFF754FD2046FFF756
:10D08000D8FE00F001FFF5E74FF08053CAF80030FA
:10D09000BFF34F8FBFF36F8FECE72046FFF7C9FE5A
:10D0A00000F0F2FEB4E700BF7EBA010804ED00E034
:10D0B00010B5024600210120FFF732FF044638B1C7
:10D0C000002383600360C3601A461946FFF74CFFD4
:10D0D000204610BD2DE9F843894690461F46044678
:10D0E00020B940F2C3312748F5F706FAB9F1000F2D
:10D0F00006D1236C23B14FF471712248F5F7FCF986
:10D10000022F07D1E36B012B04D040F2C5311D483B
:10D11000F5F7F2F9FFF7C0FDEFF311864FF050037A
:10D1200083F31188BFF36F8FBFF34F8FA26BE36B55
:10D130009A4201D3022F22D194F845503A466DB25B
:10D1400049462046FFF72EFE6B1C13D1636A0BB9CC
:10D1500001200BE004F1240001F06CF80028F7D066
:10D16000B8F1000FF4D00120C8F8000086F3118850
:10D17000BDE8F88301356DB284F84550E8E700203A
:10D18000F4E700BF7EBA010870B50D46044620B929
:10D190004FF48C612048F5F7AFF9236C23B140F2CE
:10D1A00064411D48F5F7A8F9236833B9A36823B192
:10D1B00040F269411848F5F79FF9FFF76DFDEFF36D
:10D1C00011864FF0500383F31188BFF36F8FBFF3C5
:10D1D0004F8FA26BE36B93421CD994F84530013218
:10D1E0005BB2A2635A1C10D1636A0BB9012009E03B
:10D1F00004F1240001F01EF80028F7D0002DF5D02E
:10D200000120286086F3118870BD01335BB284F879
:10D210004530EBE70020F5E77EBA01082DE9F04341
:10D2200085B00F460192044620B94FF4A0614248F0
:10D23000F5F762F937B9236C23B140F204513E4847
:10D24000F5F75AF901F042F930B9019B23B140F2E8
:10D2500009513948F5F750F90026B046DFF8DC905F
:10D26000FFF740FCA56BD5B139462046013DFFF7DD
:10D27000CCFDA563236963B104F1100000F0DAFF6F
:10D2800038B14FF080522D4B1A60BFF34F8FBFF370
:10D290006F8FFFF747FC012005B0BDE8F083019DCB
:10D2A0001DB9FFF73FFC0020F6E716B902A801F010
:10D2B00001F8FFF737FC00F03BFDFFF713FC94F893
:10D2C0004430FF2B08BF84F8448094F84530FF2B8E
:10D2D00008BF84F84580FFF725FC01A902A800F0EB
:10D2E000F5FFF0B92046FFF752FDA0B1019904F116
:10D2F000240000F065FF2046FFF79BFD00F0C4FD11
:10D3000038B94FF08053C9F80030BFF34F8FBFF3E7
:10D310006F8F0126A4E72046FFF78BFD00F0B4FDD8
:10D32000F7E72046FFF785FD00F0AEFD2046FFF74A
:10D330002EFD0028EDD0B6E77EBA010804ED00E02E
:10D340002DE9FF410446019120B940F29151524824
:10D35000F5F7D2F8236C23B140F295514E48F5F71A
:10D36000CBF801F0B3F830B9019B23B140F29A51E8
:10D370004948F5F7C1F800252F462E46DFF81C81F5
:10D38000FFF7B0FBA36BE3B1013BA363236813B9C1
:10D3900001F09EF9A060236963B104F1100000F070
:10D3A00049FF38B14FF080523C4B1A60BFF34F8FAA
:10D3B000BFF36F8FFFF7B6FB0125284604B0BDE829
:10D3C000F081019B4BB925B140F2E1513248F5F7AC
:10D3D00093F8FFF7A7FB0025EFE717B902A800F0C5
:10D3E00069FFFFF79FFB00F0A3FCFFF77BFB94F8BE
:10D3F0004430FF2B08BF84F8446094F84530FF2B7D
:10D4000008BF84F84560FFF78DFB01A902A800F072
:10D410005DFF40BB2046FFF7BAFCF0B123683BB983
:10D42000FFF760FBA06801F061F80546FFF77AFBA3
:10D43000019904F1240000F0C3FE2046FFF7F9FC37
:10D4400000F022FD38B94FF08053C8F80030BFF328
:10D450004F8FBFF36F8F012792E72046FFF7E9FC5C
:10D4600000F012FDF7E72046FFF7E3FC00F00CFDAB
:10D470002046FFF78CFC0028EDD0002D9DD0FFF753
:10D4800031FB616A19B1236B1968C1F10501A0680C
:10D4900001F0CAF89DE700BF7EBA010804ED00E084
:10D4A0002DE9F04385B00F460192044620B94FF4B0
:10D4B000CD614248F5F720F837B9236C23B140F22B
:10D4C0006C613E48F5F718F801F000F830B9019B9F
:10D4D00023B140F271613948F5F70EF80026B046E5
:10D4E000DFF8DC90FFF7FEFAA36BD3B13946204694
:10D4F000E568FFF78AFC636AE56063B104F1240024
:10D5000000F098FE38B14FF080522D4B1A60BFF3F7
:10D510004F8FBFF36F8FFFF705FB012005B0BDE80C
:10D52000F083019D1DB9FFF7FDFA0020F6E716B95B
:10D5300002A800F0BFFEFFF7F5FA00F0F9FBFFF7D5
:10D54000D1FA94F84430FF2B08BF84F8448094F853
:10D550004530FF2B08BF84F84580FFF7E3FA01A9A7
:10D5600002A800F0B3FEF0B92046FFF710FCA0B10E
:10D57000019904F1240000F023FE2046FFF759FC36
:10D5800000F082FC38B94FF08053C9F80030BFF387
:10D590004F8FBFF36F8F0126A4E72046FFF749FCAA
:10D5A00000F072FCF7E72046FFF743FC00F06CFC4C
:10D5B0002046FFF7ECFB0028EDD0B6E77EBA010865
:10D5C00004ED00E02DE9F84389469046054620B970
:10D5D00040F2FB612048F4F78FFFB9F1000F06D14C
:10D5E0002B6C23B140F2FC611B48F4F785FFFFF779
:10D5F00053FBEFF311874FF0500383F31188BFF310
:10D600006F8FBFF34F8FAC6B1CB395F844604946E6
:10D6100076B22846FFF7F9FB013C731CAC6313D1CB
:10D620002B690BB901200BE005F1100000F002FEA0
:10D630000028F7D0B8F1000FF4D00120C8F800009E
:10D6400087F31188BDE8F883013676B285F8446027
:10D65000E8E72046F4E700BF7EBA010810B50446AB
:10D6600020B940F28A710548F4F746FFFFF73AFA0D
:10D67000A46BFFF757FA204610BD00BF7EBA010821
:10D6800038B5054620B940F2A4710648F4F734FFD6
:10D69000FFF728FAA86BEC6B241AFFF743FA204631
:10D6A00038BD00BF7EBA0108002330B5064A52F8E3
:10D6B000335002EBC3041DB942F83310606030BD33
:10D6C0000133052BF3D1FAE7241A0020002310B50B
:10D6D000074A02EBC3014C68844204D1002042F89F
:10D6E0003300486010BD0133052BF2D1FAE700BFCB
:10D6F000241A002010B5044620B94FF4F8610548FB
:10D70000F4F7FAFE2046FFF7E1FF2046BDE810409F
:10D71000FFF72ABB7EBA010870B504460D461646CF
:10D72000FFF7E0F994F84430FF2B04BF002384F89E
:10D73000443094F84530FF2B04BF002384F8453073
:10D74000FFF7F0F9A36B2BB93246294604F1240008
:10D7500000F050FD2046BDE87040FFF76ABB0000B6
:10D76000064A13681968064B19B94FF0FF321A6060
:10D7700070471268D268D2685268F8E768140020CF
:10D780001815002010B5044620B940F2F26108488F
:10D79000F4F7B2FE6269074B9A4207D1A06A064BC2
:10D7A000984203D0B0FA80F0400910BD0020FCE799
:10D7B0007EBA01083815002020150020F8B51B4B53
:10D7C0001B4E1C68054630680F46043001F0E9FA2C
:10D7D000334640B901203168164EC96A3268884024
:10D7E00022EA000232606A1C07D137B11968124878
:10D7F0000431BDE8F84001F0B1BA1A686419546008
:10D8000007D30E4A10681968BDE8F840043101F0EA
:10D81000B1BA0B4A10681968043101F0ABFA094B30
:10D820001A68A24288BF1C60F8BD00BF60150020C6
:10D8300064140020E8140020381500206C14002027
:10D84000681400201815002080B5DFF86C80164F92
:10D85000164D174E2B6863B9164B1B68012BF8D970
:10D860004FF08053C8F80030BFF34F8FBFF36F8F76
:10D87000EEE7FFF737F9FB68DC68201D01F091FA4D
:10D880003368013B33602B68013B2B60FFF74AF99B
:10D8900004F154000BF086F9206BFFF765FA20467F
:10D8A000FFF762FAD6E700BF4C150020D81400201D
:10D8B000D41400207014002004ED00E02DE9F84F8E
:10D8C0004FEA820A804650460D4699460B9EFFF766
:10D8D00049FA0746002800F0B780BC20FFF742FA5B
:10D8E0000446002800F0AD80076325B94FF4587155
:10D8F0005C48F4F701FE5246A521206B0AF0A9FA14
:10D90000236BAAF1040A9A442AF0070A6B1E04F159
:10D9100034020F3513F8011F02F8011B197809B101
:10D92000AB42F7D10A9D4FF0000B042D28BF042510
:10D93000271DE562C4E9135B384684F843B001F063
:10D940000AFAC5F1050504F1180001F004FAC4F85B
:10D95000B4B0602259462461A561646284F8B8B00D
:10D9600004F154000AF075FA3F4B4A46A3653F4B59
:10D970004146E3653E4B50462366FFF78DF8206035
:10D9800006B13460FFF7AEF83A4B3B4E1A68DFF849
:10D99000248101321A603268002A58D134601B6831
:10D9A000012B25D1354801F0CBF9354801F0C8F9F4
:10D9B000344801F0C5F9DFF80091334801F0C0F9AF
:10D9C000324D334801F0BCF9484601F0B9F9284618
:10D9D00001F0B6F92F4801F0B3F92F4801F0B0F982
:10D9E0002E4801F0ADF92E4BC3F800902D4B1D6071
:10D9F00001252D4A2D491368086801331360E26A36
:10DA0000636405FA02F3034314200B601B4B394691
:10DA100000FB023001F0A2F9FFF784F8D8F80030DB
:10DA200063B13368DA6AE36A9A4207D24FF08052F0
:10DA30001F4B1A60BFF34F8FBFF36F8F2846BDE8AF
:10DA4000F88F3846FFF790F94FF0FF35F6E7D8F832
:10DA50000030002BCCD13368DA6AE36A9A4298BF6F
:10DA60003460C5E77EBA0108ACEC0108CCEC0108D3
:10DA70008CEC0108D41400206414002070140020E1
:10DA80008414002098140020AC14002000150020FD
:10DA9000C0140020201500204C150020381500204F
:10DAA000681400206C140020E4140020E814002006
:10DAB00004ED00E034150020EC14002070B504469D
:10DAC0002A4DFFF70FF804B92C68261D304601F0E7
:10DAD00068F960B91421E06A254B41435B5833B9BA
:10DAE0000122244982400B6823EA02030B60A36AE7
:10DAF0001BB104F1180001F054F91F4A13680133F7
:10DB000013602B68A34220D131461C4801F026F94E
:10DB10001B4A136801331360FFF704F8194B1B68A5
:10DB200093B12B68A3420FD1174B1B6823B140F26E
:10DB3000B6411648F4F7E0FC4FF08052144B1A60DF
:10DB4000BFF34F8FBFF36F8F70BD124A04F15400C3
:10DB50001368013B13600BF025F8206BFFF704F905
:10DB60002046FFF701F9FFF7FBFDD5E7641400201D
:10DB700070140020E8140020E41400204C1500204C
:10DB8000D814002034150020E01400207EBA0108CB
:10DB900004ED00E0D4140020F8B5054620B940F2A9
:10DBA0004C511748F4F7A8FC164B1B68AB4220D029
:10DBB000FEF798FF144B6C691F68144B1E68FEF744
:10DBC000B1FFBC4217D0B44215D0114B9C4208D1D2
:10DBD000AB6A83B995F8B830012B0CBF0220032043
:10DBE000F8BD0C4B9C4208D0002C0CBF0420012037
:10DBF000F6E70020F4E70220F2E70420F0E700BF98
:10DC00007EBA010864140020681400206C140020FF
:10DC1000381500204C15002070B5044620B940F29C
:10DC20001C711948F4F768FC184D2B68A34229D0E1
:10DC300044B3FEF757FF2046FFF7A4FDF0B1261DC1
:10DC4000304601F0AEF801231149E26A08689340BA
:10DC5000034314200B600F4B314600FB023001F0F0
:10DC60007DF82B68E26ADB6A9A4207D34FF0805254
:10DC7000094B1A60BFF34F8FBFF36F8FBDE8704041
:10DC8000FEF750BF70BD00BF7EBA010864140020CB
:10DC9000E81400207014002004ED00E013B5002407
:10DCA0001A4B009401935022234619491948FFF753
:10DCB00005FE01281DD100F0BBFE012819D14FF04F
:10DCC000500383F31188BFF36F8FBFF34F8F124B55
:10DCD000124A1B68543313604FF0FF32104B1A6026
:10DCE000104B1860104B1C6002B0BDE81040FEF7EE
:10DCF00079BF013007D140F604010C4802B0BDE8FD
:10DD00001040F4F7F9BB02B010BD00BF141500209D
:10DD10004CCC010849D80008641400208803002076
:10DD20001815002034150020601500207EBA010867
:10DD3000024A136801331360704700BFE0140020EB
:10DD4000014B1868704700BF6015002008B5FEF74A
:10DD5000A3FF014B186808BD60150020014B18682F
:10DD6000704700BFD41400202DE9F84F3A4B1B68D0
:10DD7000002B6AD1394B1C6801341C609CB9384DAA
:10DD80002B681B6823B140F662213648F4F7B4FBD8
:10DD9000354B2A68196829601A60344A13680133C0
:10DDA0001360FFF7DDFC324D4FF0000B2B68314F55
:10DDB000A34211D93A68304BD16A14224A439A5887
:10DDC000022A28BF4FF0010B2C4A1268002A0CBF10
:10DDD00058460120BDE8F88FDFF884A0DFF8A49052
:10DDE000DAF8002012681AB94FF0FF322A60E1E732
:10DDF000DAF80020D268D66871688C4201D22960B6
:10DE0000D8E706F10408404600F0CBFFB16A19B12B
:10DE100006F1180000F0C5FF01224FF0140CF06A63
:10DE2000D9F8003002FA00F11943134BC9F8001079
:10DE30000CFB0030414600F091FF3868F16AC26A7D
:10DE4000914228BF4FF0010BCAE70D4A4FF0000B7B
:10DE5000136801331360B7E7E01400206015002059
:10DE6000681400207EBA01086C1400201C150020E4
:10DE70001815002064140020701400206415002080
:10DE8000DC140020E81400202DE9F8432E4C236810
:10DE900023B940F668012D48F4F72EFBFEF722FE69
:10DEA0002368013B236024682CB10024FEF73AFE6E
:10DEB0002046BDE8F883264B1B68002BF5D0254D86
:10DEC000254EDFF8A8801FE0EB680127DC6804F12D
:10DED000040904F1180000F064FF484600F061FFF7
:10DEE0001420E26A316807FA02F30B4300FB028058
:10DEF0004946336000F032FF184BE26A1B68DB6A68
:10DF00009A4201D3164B1F602B68002BDCD10CB159
:10DF1000FFF726FC134D2C6844B10127104EFFF784
:10DF200023FF00B13760013CF9D12C600C4B1B681A
:10DF3000002BBAD04FF080520B4B1A60BFF34F8FBB
:10DF4000BFF36F8F0124B1E7E01400207EBA01080F
:10DF5000D414002020150020E814002064140020B0
:10DF600064150020DC14002004ED00E07014002093
:10DF700038B50C46054620B940F2CA411848F4F7B6
:10DF8000BBFA24B940F2CB411548F4F7B5FA154B6A
:10DF90001B6823B140F2CC411148F4F7ADFAFFF70A
:10DFA000C7FE114B2A68186814192CBF01210021E3
:10DFB00082422C600CD961B9FFF766FF38B94FF087
:10DFC00080520A4B1A60BFF34F8FBFF36F8F38BD7B
:10DFD00009B9A042F0D20021201AFFF7EFFBEBE7CE
:10DFE0007EBA0108E01400206015002004ED00E076
:10DFF00010B5044640B94FF080520D4B1A60BFF384
:10E000004F8FBFF36F8F10BD0A4B1B6823B14FF4C6
:10E01000A4610948F4F770FAFFF78AFE0021204650
:10E02000FFF7CCFBFFF730FF0028E4D0EBE700BFA1
:10E0300004ED00E0E01400207EBA0108244B70B526
:10E040001A68244B12B101221A6070BD224E1A6068
:10E0500033681B6B1A68B2F1A53F0BD15A68B2F155
:10E06000A53F07D19A68B2F1A53F03D1DB68B3F1B0
:10E07000A53F04D0306831683431F4F70DFA174BFE
:10E080001C68B4FA84F41423E4B2C4F11F0463439B
:10E09000134DEB5823B940F688311248F4F72CFAA7
:10E0A000142202FB04F3E9184868083340682B4443
:10E0B000984202FB045408BF4368486008BF4B60A5
:10E0C0006368094ADB683360336854331360BCE724
:10E0D000E01400206415002064140020E8140020DF
:10E0E000701400207EBA01088803002070B5044631
:10E0F0002A4EFEF7F7FC04B93468251D284600F0C7
:10E1000050FE60B91421E06A254B41435B5833B996
:10E110000122244982400B6823EA02030B60A36AB0
:10E120001BB104F1180000F03CFE29461E4800F027
:10E1300015FE94F8B8301D4D012B04BF002384F860
:10E14000B830FEF7EFFC2A682AB1FEF7CBFCFFF7E8
:10E1500007FBFEF7E7FC3368A34211D12B6883B1BC
:10E16000134B1B6823B14FF4D9611248F4F7C4F97B
:10E170004FF08052104B1A60BFF34F8FBFF36F8F79
:10E1800070BD094A11680D4A1268914201D133608D
:10E19000F6E7BDE87040FFF751BF00BF64140020F0
:10E1A00070140020E81400203815002034150020D9
:10E1B000E01400207EBA010804ED00E0D414002031
:10E1C00038B50D46044620B940F69F310748F4F7AC
:10E1D00093F9074B20461968183100F0CBFD28460B
:10E1E000BDE838400121FFF7E9BA00BF7EBA010857
:10E1F0006414002070B50E461446054620B940F65A
:10E20000CA310A48F4F778F9094B284619681831D9
:10E2100000F0A4FD002C214608BF3046BDE8704048
:10E2200018BF4FF0FF30FFF7C9BA00BF7EBA010830
:10E230006414002038B5C368DC6824B940F6FA31AC
:10E240001548F4F759F904F11805284600F0A9FD1E
:10E25000124B1B68E3B9251D284600F0A2FD0123DF
:10E260000F49E26A08689340034314200B60294673
:10E270000C4B00FB023000F071FD0B4BE26A1B6897
:10E28000DB6A9A4285BF0120084B0020186038BD28
:10E2900029460748EFE700BF7EBA0108E0140020D6
:10E2A000E81400207014002064140020641500207D
:10E2B00020150020034B1B680360034B1B68436061
:10E2C000704700BF1C1500206015002070B50C467B
:10E2D000054620B940F665411448F4F70DF924B914
:10E2E00040F666411148F4F707F9FEF7FBFB104BC7
:10E2F0001A682368591C0FD00E482E680068696898
:10E30000864201D091420ED9521A934209D99B1AE2
:10E3100023602846FFF7CEFF0024FEF703FC2046CB
:10E3200070BD002323600124F7E700BF7EBA010817
:10E33000601500201C1500200122014B1A60704757
:10E340006415002070B50C461646054608B91B4AF0
:10E35000156805F134026260EA6A052B22612A6BB6
:10E360002560E2616A6CA260EA6C62614FF00002B3
:10E37000A2611BD011490968A9420BD12273D6B101
:10E38000296B0A46531A12F8010BA528FAD09B08EC
:10E39000238470BD032B2373F1D1FFF7C9FCAB6A53
:10E3A0000BB102232373FFF76FFDE8E72846FFF761
:10E3B000F3FB2073E3E72684EBE700BF641400203F
:10E3C0002DE9F84F0D6881460C4692461DB3002595
:10E3D0004FF0240B4B6801F108075B68BB424B60B0
:10E3E00004BFCB684B604B68D3F80C8063680BFBB1
:10E3F00005915B6801229F42636008BFE36805F1F5
:10E40000010508BF63606368DE6853463046FFF766
:10E4100099FFB045EAD12846BDE8F88F2DE9F843C9
:10E4200005461746FFF784FC1F4B1B688B4238D804
:10E430004FF0000824264446DFF8809009EB0801DD
:10E4400006FB04500122FFF7BBFFA8F1140818F1E6
:10E45000640F0444F2D1154B0222196806FB0450E4
:10E46000FFF7AEFF124B04441968022206FB04506A
:10E47000FFF7A6FF044404220E4906FB0450FFF7F1
:10E480009FFF044406FB045003220B49FFF798FF4B
:10E4900004440FB100233B60FFF7F6FC2046BDE8C3
:10E4A000F8830024F8E700BFD4140020681400208B
:10E4B0006C1400204C15002038150020C0140020DA
:10E4C000014B1868704700BF64140020054B1B689F
:10E4D00033B1054B1B68002B0CBF02200020704796
:10E4E0000120704734150020E01400202DE9F04190
:10E4F0000446002836D0234AC36A11681746C96A01
:10E500008B4237D2142682691F4D002AA8BF3A6871
:10E5100006FB0353A2BFD26AC2F1050282614269BF
:10E520009A4221D100F10408404600F03AFC174B12
:10E5300048B9E06A4643AA592AB901211A688140BC
:10E5400022EA01021A603A681968D26AE26201247A
:10E5500004FA02F0084318601420414600FB025000
:10E5600000F0FCFB204603E03B68DB6AC36201204D
:10E57000BDE8F0811368C06CDC6AA0422CBF0020AB
:10E580000120F5E76414002070140020E814002036
:10E59000F8B5044608B90020F8BD1F4B1B6883423C
:10E5A00004D040F67A711D48F3F7A6FF236D23B916
:10E5B00040F67B711948F3F79FFF236DE16AE26C27
:10E5C000013B91422365E6D0002BE4D1251D28466E
:10E5D00000F0E7FB124E134A50B91421E76A794361
:10E5E00073582BB901201368B84023EA0003136065
:10E5F000E36CC3F10501A161E3620124116804FA2F
:10E6000003F0084310601420294600FB036000F06B
:10E61000A5FB2046C0E700BF641400207EBA0108B5
:10E6200070140020E8140020F8B50D4604460028B8
:10E6300045D0036D23B940F6C9712148F3F75CFF5B
:10E64000E36C9D4238BF1D46E36AAB4237D0236D71
:10E65000012B34D11B4B1B68A34204D140F6E4715B
:10E660001748F3F749FF1426A269E36A002AE56216
:10E67000A4BFC5F10505A561134D626906FB0353EF
:10E680009A421CD1271D384600F08BFBE26A0F4CE2
:10E6900040B95643AB592BB901212368914023EA75
:10E6A0000103236001231420216893400B4323605E
:10E6B000394600FB0250BDE8F84000F04FBBF8BD02
:10E6C0007EBA01086414002070140020E8140020B1
:10E6D000044B1A681AB119680A6D01320A65186884
:10E6E000704700BF641400202DE9F041214C1E4604
:10E6F00080460F461546FEF7F5F9236893F8B830C3
:10E70000022B16D001212368D3F8B42022EA080294
:10E71000C3F8B420236883F8B81056B13046FFF729
:10E720004DF84FF08052144B1A60BFF34F8FBFF378
:10E730006F8FFEF7F7F9FEF7D5F91DB12368D3F80F
:10E74000B4302B602368002293F8B830022B09BF45
:10E75000012500252368D3F8B41004BFB943C3F8DA
:10E76000B410236883F8B820FEF7DCF92846BDE82A
:10E77000F08100BF6414002004ED00E0F8B50E46FF
:10E7800017461D46044620B941F219212E48F3F7D9
:10E79000B3FEFEF7A7F915B1D4F8B4302B6002230D
:10E7A00094F8B85084F8B830EDB2042F1AD8DFE8E6
:10E7B00007F00E0309061500D4F8B4301E43C4F860
:10E7C000B46004E0D4F8B4300133C4F8B430012D9F
:10E7D00012D00124FEF7A6F92046F8BD022DEED195
:10E7E0000024F7E7D4F8B4300133F0D041F24A21E5
:10E7F0001548F3F781FEEAE7261D304600F0D1FA0E
:10E800001420124AE36A11689D400D431560104AB6
:10E81000314600FB032000F0A1FAA36A23B141F2C4
:10E8200059210948F3F768FE0A4BE26A1B68DB6A64
:10E830009A42CED94FF08052074B1A60BFF34F8FE8
:10E84000BFF36F8FC5E700BF7EBA0108E814002050
:10E85000701400206414002004ED00E02DE9F8435A
:10E86000DDF820800E4691461D46044620B941F24F
:10E870008C213848F3F740FEFEF70EFAEFF31187CC
:10E880004FF0500383F31188BFF36F8FBFF34F8FA7
:10E8900015B1D4F8B4302B60022394F8B85084F842
:10E8A000B830EDB2B9F1040F1AD8DFE809F00E0361
:10E8B00009061500D4F8B4301E43C4F8B46004E06F
:10E8C000D4F8B4300133C4F8B430012D12D0012093
:10E8D00087F31188BDE8F883022DEED10020F7E719
:10E8E000D4F8B4300133F0D041F2CF211948F3F716
:10E8F00003FEEAE7A36A23B141F2DA211548F3F7F0
:10E90000FBFD154B1B6803BB251D284600F049FA8B
:10E9100001231249E26A08689340034314200B6004
:10E9200029460F4B00FB023000F018FA0D4BE26A4B
:10E930001B68DB6A9A42CAD90123B8F1000F01D0E3
:10E94000C8F80030084A1360C1E704F1180107480D
:10E95000EAE700BF7EBA0108E0140020E8140020B6
:10E96000701400206414002064150020201500207D
:10E9700038B5054608B9084B1D680024FEF7B2F803
:10E9800095F8B830022B04BF85F8B8400124FEF793
:10E99000C9F8204638BD00BF64140020F8B50F4CFC
:10E9A000FEF7A0F82568ADB90D4F0E4E384600F0C1
:10E9B000C7F9304600F0C4F90B4B2A461F600B4BD9
:10E9C0000C210A201E60FEF7ABFA206010B1084946
:10E9D000FEF76AFEBDE8F840FEF7A4B89C150020DB
:10E9E0007015002084150020681500206C1500208B
:10E9F00051CC0108914208B5416000610AD8D21A91
:10EA000083699A420DD2084B011D186800F0B2F9D3
:10EA1000002008BD9A4201D2994202D2011D034B47
:10EA2000F3E70120F5E700BF6C1500206815002012
:10EA300007B5FFF7B3FF0C4B1B6843B90B484FF406
:10EA40008971F3F759FD002003B05DF804FB084B12
:10EA5000C822019301230749009307480023FEF7CA
:10EA60002DFF0028EAD0EFE79C1500207EBA0108B0
:10EA7000A015002056CC010895EB00082DE9F041C7
:10EA800080462C200D4617461E46FEF76BF90446BD
:10EA900088B125B94FF4B6710848F3F72DFDFFF79B
:10EAA0007DFF069BC4F80080C4E9065726626362B6
:10EAB000201D00F050F92046BDE8F0817EBA010823
:10EAC0002DE9FF410D4690461F46064620B94FF4FA
:10EAD000C3710F48F3F710FD0E4C206878B1052D77
:10EAE000CDE9015803960DDCFFF7F0FC0023022866
:10EAF0000CBF0A9A1A4601A92068FEF735FA04B03D
:10EB0000BDE8F08100233A4601A9FEF7E3FAF6E7F3
:10EB10007EBA01089C1500202DE9F74300271A4D05
:10EB2000DFF86C802B681A6832B9184A11681360D4
:10EB3000296003B0BDE8F083DB68DC681E6804F17F
:10EB40000409484600F02DF9636A20469847E369B6
:10EB5000012BE7D1A36933449E4206D2636024614E
:10EB60004946286800F006F9DCE7002300973246A2
:10EB700019462046FFF7A4FF0028D3D140F2723196
:10EB80004046F3F7B9FCCDE7681500206C1500206E
:10EB90007EBA01082DE9F04F4FF00108624D89B0AF
:10EBA000DFF898B1DBF80020136843B30024D36882
:10EBB000D3F80090FFF7BCF8FFF7C2F85B4B824632
:10EBC0001A681F4690425A4E1CD31860002C4CD035
:10EBD000584B1B681A68B2FA82F25209A9EB0A0173
:10EBE0003068FEF799FDFFF74FF998B94FF0805262
:10EBF000514B1A60BFF34F8FBFF36F8F0AE00124B0
:10EC00009946D7E70393FFF787FF039BC3F800A05C
:10EC1000FFF73AF9002205A93068FEF7FFFA00284D
:10EC2000BED0059B002BF5DB079C636913B1201D4B
:10EC300000F0B7F8FFF784F83B688146984201D2AC
:10EC4000FFF76AFF059BC7F80090092BE2D808FA86
:10EC500003F313F4047A57D113F0C70F33D19B0693
:10EC6000D8D52046FEF780F8D4E7814529D8FFF7AC
:10EC70000BF9DBF80030DB68D3F80CB00BF10400C3
:10EC800000F08FF8DBF81C30012B15D1DBF81810E1
:10EC90004B46524649445846FFF7ACFE60B10094DB
:10ECA00023464A4621465846FFF70AFF20B94FF44B
:10ECB000F4712846F3F720FCDBF8243058469847D7
:10ECC000A8E722468AE7A169069B4A4619442046DE
:10ECD000FFF790FE00289DD0636A20469847E369BD
:10ECE000012B97D1A2690699CDF800A00A4453469A
:10ECF00051462046FFF7E4FE00288BD140F2013157
:10ED00002846F3F7F9FB85E7069BA36123B94FF487
:10ED100046712846F3F7F0FBA1694B464A46494441
:10ED20002046FFF767FE75E77EBA010898150020B8
:10ED30009C1500206C15002004ED00E068150020F3
:10ED40004FF0FF3200F108034360C0E90223036182
:10ED500000230360704700230361704743689A688B
:10ED60004B608A609A68516099600368086101335A
:10ED7000036070470A6830B5531C0AD103695A68AA
:10ED80004A6091608B6059600368086101330360D9
:10ED900030BD00F108035C6825689542EFD8234632
:10EDA000F9E70369D0E901128A6082685160596805
:10EDB000814208BF5A60002202611A68013A1A6053
:10EDC00018687047021C18BF012200210148F8F79B
:10EDD00081BE00BF00040240F9F72EBB38B50546DE
:10EDE0000C460020FFF7EEFF45F08000FFF7F4FF30
:10EDF0002046FFF7F1FFBDE838400120FFF7E2BFF2
:10EE000008B50120F8F770FC0A20F8F76DFC0B201C
:10EE1000F8F76AFC0720F8F767FC0520F8F764FCB0
:10EE2000BDE808400420F8F75FBC0000204B70B537
:10EE30009D780446EDB958B902211E48F8F744FE02
:10EE400023461A460221BDE870401A48F8F78CBDE7
:10EE5000012805D102211748F8F730FE2B46F0E7CC
:10EE6000022823D102460146BDE870401148F8F758
:10EE7000B9BD012D14D138B904210E48F8F724FE8C
:10EE8000002304211A46DEE7012804D104210948A1
:10EE9000F8F714FEF4E7022808D102460421E3E75C
:10EEA0006A21BDE870400448F3F726BB70BD00BF7F
:10EEB000A4150020000002407EBA010808B5002019
:10EEC000FFF7B4FFF8F752FB0120FFF7AFFFF8F7A9
:10EED0004DFB0220FFF7AAFFBDE80840F8F746BB4C
:10EEE00008B500210120F9F729FA0120FFF76AFF90
:10EEF0000023094819461A46F8F736FDB521402087
:10EF0000FFF76CFFA0214120FFF768FFBDE8084034
:10EF100000210120FFF762BF0004024010B5FFF797
:10EF20006FFF0120FFF74EFF00233A481A461946AB
:10EF3000394CF8F719FD00210120F9F7FFF9227883
:10EF40007AB1002306211A463248F8F70DFD062152
:10EF50003048F8F7B3FDF8F709FB19215820FFF7FF
:10EF60003DFFFFF7ABFFFFF7BBFF63785BB100230B
:10EF700004211A462948F8F7F7FC00230D211A4608
:10EF80002748F8F7F1FC002201212248F8F72AFD72
:10EF900000220A211F48F8F725FD00220B211D48F9
:10EFA000F8F720FD002207211A48F8F71BFD002280
:10EFB00005211848F8F716FD002204211548F8F736
:10EFC00011FD0523022201211248F8F7ABFB0523AE
:10EFD00002220A210F48F8F7A5FB052302220B2184
:10EFE0000C48F8F79FFB0523022207210948F8F790
:10EFF00099FB0523022219460648F8F793FB094BB3
:10F000001B782BB9BDE81040BE210748F3F774BA4E
:10F0100010BD00BF00040240A41500200000024003
:10F0200000080240A71500207EBA010882B00190B6
:10F0300002AB33F8041D054A9B78118093700122BE
:10F04000034B1A7002B0FFF769BF00BFA415002080
:10F05000A71500201A4B10B55B78D3B10128194CC5
:10F0600018D104211848F8F729FD0D211748F8F7A1
:10F070002BFD23786BB1002304211A461248F8F7C0
:10F0800073FC00230D211A461048F8F76DFC00238D
:10F09000237010BD40B904210B48F8F715FD0D2170
:10F0A0000A48F8F70BFDE4E7022204210648F8F7C6
:10F0B00099FC02220D210548F8F794FC0123E7E7AB
:10F0C000A415002044010020000002400008024076
:10F0D00008B5FFF795FEFFF7F1FEFFF701FFF9F71F
:10F0E00087F9012200211F48F8F77CFC0220FFF776
:10F0F000B1FF0220FFF79AFE022201211948F8F71A
:10F1000071FC02220A211748F8F76CFC02220B213D
:10F110001448F8F767FC022207211248F8F762FC4E
:10F12000022205210F48F8F75DFC022204210D4858
:10F13000F8F758FC0C4B1B781BB9E2210B48F3F78E
:10F14000DBF90B4B1B785BB1002306211A460548FF
:10F15000F8F70AFCBDE8084006210248F8F7B4BCFD
:10F1600008BD00BF00040240A71500207EBA0108B8
:10F17000A415002010B5064C022220460021F8F705
:10F1800031FC2046BDE8104002220121F8F72ABCDC
:10F1900000140240F8B50F4CD4F88032984723464B
:10F1A00010F5617641F1000704F52072D3E90845B6
:10F1B000A04271EB050401DAC3E90801D3E9064571
:10F1C000A64277EB050401DAC3E9066728339342C8
:10F1D000ECD1F8BDB015002010B5044618B9BB211C
:10F1E0000748F3F789F9074BD3F880329847D4E9F9
:10F1F0000623904271EB0304B4BF101A002010BD27
:10F200007EBA0108B01500202DE9F84F064628B94E
:10F21000BDE8F84FDC213448F3F76EB90023334AD8
:10F220001C469246D118097A2833B14208BF0134EE
:10F23000B3F5207FF6D1002C54D0062E03D94021FF
:10F240002948F3F759F92A4B53F83650002D47D186
:10F25000E7212548F3F750F94FF0000B65430AEB1F
:10F260000B04227AB24235D16268002A32D0226978
:10F27000012A03D1D0211C48F3F73EF9D4E9062333
:10F2800019461343104624D0D4E90889B0EB08008E
:10F2900061EB090107F090FF07462069013807F08C
:10F2A00071FF0146384608F079F80746284607F00E
:10F2B00069FF394607F0BEFF394607F0B1FE08F096
:10F2C000A5F918EB000249F1000310461946C4E9FC
:10F2D000060125610BF1280BBBF5207FBFD101E0B2
:10F2E000012DB9D1BDE8F88F7EBA0108B015002014
:10F2F00060CC01084FF47A73B0FBF3F341F6583257
:10F30000A3F55223A3F6183393422DD81B4B1C4A66
:10F310000344934228D91B4B1B4A0344934223D9ED
:10F320004CF24E32194B034493421DD9184B98426C
:10F330001CD903F5371303F5D863984218D903F5A0
:10F34000122303F5F863984214D903F5122303F549
:10F35000F863984210D903F5DB2303F5BA639842AA
:10F3600094BF052006207047002070470120704799
:10F370000220704703207047042070473F373ACC83
:10F380009E8601007F0F31CC3E0D0300AF312ACCA9
:10F3900040DA8E332DE9F04385B0E0B1D0E903982F
:10F3A0004FF47A740D4B4168D3F88C62037AB1FB49
:10F3B000F4F4062B96BF0A4A0A4D52F823500778F8
:10F3C000FFF70AFFCDF80080CDE901903B462A46C1
:10F3D00021460548B04705B0BDE8F083B0150020D0
:10F3E00098CC0108B8CD0108C5CD010870B5134C03
:10F3F000054694F894320E4623B94FF4967110489E
:10F40000F3F77AF825B940F22D110D48F3F774F8A7
:10F4100026B94FF497710A48F3F76EF800232822B3
:10F4200002FB03F0215CA94203D120444168B142B0
:10F4300003D00133102BF3D1002070BDB015002094
:10F440007EBA01082DE9F04F2E4F9A4697F8943274
:10F4500093B00191934623B940F241112A48F3F742
:10F460004BF80025FFF796FEA9464FF0FF382C46D3
:10F47000282303FB0576019AF368934218DBBBF15E
:10F48000000F10D13046FFF7A7FE80B3404536D3BA
:10F490000ED1D4E90823D6E90801FBF7FEF80028CD
:10F4A00018BF344604E000213046D8470028E9D18F
:10F4B0000135102DDCD1BAF1000F01D0CAF800805F
:10F4C000B8F1000F0FD1B9F1010F0CD909F1FF31DB
:10F4D0004046FBF7E1FA12AB03EB8000282350F81B
:10F4E000404C03FB0474204613B0BDE8F08F12AB10
:10F4F00003EB890343F8405C09F10109C6E7804644
:10F500003446D5E7B01500207EBA010838B50B4C5B
:10F5100094F8942222B940F279110948F2F7ECFFED
:10F5200010236FF027050020002105FB0342013B5B
:10F5300002F52672C2E90001F7D138BDB0150020EE
:10F540007EBA0108000000002DE9F14F0D46044687
:10F5500020B94FF4C2712048F2F7CEFF236923B9D6
:10F5600040F285111C48F2F7C7FFDFF87490D9F814
:10F57000803298478B4682462069C4E908AB07F081
:10F5800001FE294607F056FE294607F049FD07F01F
:10F59000E1F90FA3D3E9002307F05EFB06F01CFF9F
:10F5A00007F0CAFC1AEB00064BF100078046C4E9DD
:10F5B0000667284608F004F8D9F88C5202464346FC
:10F5C000AC466168054801B0BDE8F04F604700BF38
:10F5D0000000000080842E417EBA0108B4CC0108EE
:10F5E000B01500202DE9F0410E461746054620B91A
:10F5F0004FF4C8711348F2F77FFF26B940F291111A
:10F600001048F2F779FF0021384607F0CFFF20B904
:10F610004FF4C9710B48F2F76FFF0024DFF8288020
:10F6200014F80830AB4207D108EB04004368B3423A
:10F6300002D13946FFF788FF2834B4F5207FEFD197
:10F64000BDE8F0817EBA0108B015002008B5FFF7CB
:10F6500051FE003018BF012008BD00002DE9F04721
:10F660003F4F94B097F8943206460D4623B94FF4B5
:10F67000D9713C48F2F740FF2846FFF7E7FF044600
:10F6800058B94FF47A713848D7F89032B5FBF1F198
:10F690009847204614B0BDE8F08729463046FFF76A
:10F6A000A5FE0028F6D18046282303FB0879D9F867
:10F6B00004202AB108F10108B8F1100FF5D1E9E7EB
:10F6C00097F894321BB977212648F2F715FF1EB937
:10F6D00078212448F2F710FF282200210DEB0200C8
:10F6E00008F0B7FB2846FFF705FE062804468DF80C
:10F6F000300003D940211B48F2F7FEFE0B956D4602
:10F700004FF0280A194B8DF8286003EBC4025268A9
:10F7100053F834300AACCDE90D230FCC0FC50FCC14
:10F720000AFB087A0FC594E803006E46544685E844
:10F7300003000FCE0FC40FCE0FC495E80300D7F817
:10F740008C3284E803004146094898474846FFF751
:10F7500021FE9AF80800FFF757FD48469AE700BFD8
:10F76000B01500207EBA010868CD010860CC010800
:10F7700097CD01080D4B10B593F89432044623B988
:10F780004FF4EA710A48F2F7B7FE6CB163685BB1F7
:10F790000848FBF733F82046FFF7FCFD0023207AEA
:10F7A00063602372FFF730FD002010BDB01500200C
:10F7B0007EBA010828CE01082DE9F041124D074616
:10F7C00095F89432884623B94FF4F6710F48F2F752
:10F7D00093FE27B940F2ED110C48F2F78DFE00249C
:10F7E00026462B5DBB4208D128194368434504D106
:10F7F000FFF7C0FF002818BF06462834B4F5207F65
:10F80000EFD13046BDE8F081B01500207EBA010886
:10F8100070B5114C064694F8943223B94FF4FE713A
:10F820000E48F2F769FE26B940F2FD110B48F2F7D7
:10F8300063FE0025635DB34204D1601943680BB1D8
:10F84000FFF798FF2835B5F5207FF3D1D4F88C3237
:10F850000348BDE870401847B01500207EBA010883
:10F860000CCE01082DE9F843154D06460F4690468B
:10F870000024A946635DB34209D12B195A6832B1FD
:10F88000002398450DDC09EB0400FFF773FF2834D3
:10F89000B4F5207FEED10024A04508DC0120BDE8AE
:10F8A000F88357F823108A42F1D00133E9E757F87B
:10F8B00024103046FFF7D2FE0028F0D00134EBE7E9
:10F8C000B0150020014B93F894027047B01500204A
:10F8D00010B5074C2378FA2B04D94FF40D71054865
:10F8E000F2F70AFE20780130C0B2207010BD00BFD0
:10F8F000A81500207EBA010884B070B504AC84E875
:10F900000F001C4B93F894121C4631B1BDE87040B7
:10F91000D3F89032184804B018474FF426721846AE
:10F9200004F5207504AE08F094FA0FCE0FC53368C5
:10F930002B6013B9114BC4F89032D4F88C3213B940
:10F940000E4BC4F88C32D4F8883213B1D4F8843218
:10F950004BB9D4F88C320A4898470A4BC4F888321D
:10F96000094BC4F88432012384F89432BDE8704016
:10F9700004B07047B0150020F4CC0108F5A70008CA
:10F980002DCD01089D7D01088D7D01082DE93008F0
:10F990000F4B03F52072D3E908BC5BEA0C0405D0D9
:10F9A0001BEB00044CEB0105C3E90845D3E906BC99
:10F9B0005BEA0C0405D01BEB00044CEB0105C3E92A
:10F9C000064528339342E6D1BDE83008FFF7E2BB95
:10F9D000B015002010B50A4C22681AB92721094831
:10F9E000F2F78AFD4FF0FF312068FDF7A9FC28B936
:10F9F000BDE8104028210348F2F77EBD10BD00BFCE
:10FA0000701800207EBA010808B5002306481A467F
:10FA100019460068FDF7A8FA28B9BDE808402E216C
:10FA20000248F2F769BD08BD701800207EBA0108CF
:10FA3000014B00201B68184748180020014B01208B
:10FA40001B681847481800202DE9F84300232C4D67
:10FA50002C4C6F692370DFF8B890DFF8B8808FB155
:10FA6000AB6839462848C9F8007098476B69B3F508
:10FA7000004F04BF01232370FF2488F80040204674
:10FA8000BDE8F883FFF7A6FFFFF7D2FF6B689F2062
:10FA900098476B68FF2098476B680446FF2098479B
:10FAA0006B68FF2098470646FFF7C8FFFFF7ACFFDB
:10FAB000AD6833463A4621461448A8477F2C04D106
:10FAC0004FF48023C9F80030D7E7042C13D106F097
:10FAD0001F00032805D14FF400530624C9F8003055
:10FAE000CBE7062805D14FF480330524C9F8003050
:10FAF000C3E70828E4D00024C9F80040BDE700BFF0
:10FB0000481800206C180020C3CE0108E2CE01087E
:10FB1000681800206418002008B5FFF789FF044B1F
:10FB200006205B689847BDE80840FFF787BF00BF25
:10FB30004818002008B5FFF77BFF044B04205B68E2
:10FB40009847BDE80840FFF779BF00BF481800207C
:10FB5000014B1868704700BF6818002038B5FFF7E0
:10FB600073FF094D10B10120287638BD2B6905209F
:10FB70009847FFF769FF04460028F4D12876AB6860
:10FB8000024898472046F0E74818002002CF0108B5
:10FB90002DE9F041184F154606468846FFF71AFF33
:10FBA0003A780AB9FFF7B8FF144CFFF741FF6368D2
:10FBB00002209847124B1B68B3F5803F03D9636856
:10FBC000C6F3074098476368C6F307209847636801
:10FBD000F0B298474544A84509D1FFF72FFF3B787D
:10FBE0000BB9FFF7A7FFBDE8F041FFF70DBF636852
:10FBF00018F8010B9847EEE76C1800204818002011
:10FC0000681800201C4B2DE9F041984206468846B2
:10FC1000174603D9F2211948F2F76EFC184DFFF789
:10FC2000D9FE2A780AB9FFF777FF164CFFF700FFD5
:10FC3000636802209847144B1B68B3F5803F03D9D3
:10FC40006368C6F3074098476368C6F30720984780
:10FC50006368F0B298474FB9FFF7F0FE2B780BB905
:10FC6000FFF768FFBDE8F041FFF7CEBE636840468E
:10FC70009847013FEFE700BFFEFF03007EBA01088F
:10FC80006C1800204818002068180020F8B5194B9F
:10FC9000064698420D46174604D940F20D11164803
:10FCA000F2F72AFC154CFFF795FEFFF7C1FE6368DB
:10FCB00003209847124B1B68B3F5803F03D9636854
:10FCC000C6F3074098476368C6F307209847636800
:10FCD000F0B298472F44BD4205D1FFF7AFFEBDE813
:10FCE000F840FFF791BE6368FF20984705F8010BC5
:10FCF000F1E700BFFEFF03007EBA010848180020AC
:10FD00006818002008B5FFF765FEFFF791FE054B68
:10FD1000B9205B689847FFF791FEBDE80840FFF700
:10FD200073BE00BF4818002007B5FFF753FEFFF76A
:10FD30007FFE002340F6FE720193019B934206DD95
:10FD4000FFF77CFE03B05DF804EBFFF75DBE019B9F
:10FD500001330193F1E7000084B070B504AC84E88E
:10FD60000F00204C0023254604AEA3610FCE0FC523
:10FD700096E8030085E803000AB91B4BA3602368DB
:10FD80001BB9A7211948F2F7B7FB63681BB9A82173
:10FD90001648F2F7B1FBA3681BB9A9211348F2F783
:10FDA000ABFB0120FDF784F9114B186018B9AC21A9
:10FDB0000E48F2F7A1FBFFF7B7FFFFF7CFFE0D4BA1
:10FDC00005461B784BB1FFF733FE63680120984767
:10FDD000636840209847FFF731FE2846BDE8704031
:10FDE00004B0704748180020F5A700087EBA010843
:10FDF000701800206C180020F0B508B90020F0BD84
:10FE0000002746684D1CB5421760F7D803685C1898
:10FE10005B5C03F01F03A3F1180103298FBF384671
:10FE20000D49C91811F8180C0544AE42E6D3042850
:10FE30000DD8DFE800F00403070C0C0063781360B2
:10FE40000130DCE7B4F801305BBA9BB2F7E7D4F8D5
:10FE500001301BBAF3E700BF12CF0108F7B51F4608
:10FE6000436816464A1C9A4205460C4617D8036852
:10FE70005B5C03F0C003402B11D196B101AAFFF7E0
:10FE8000BBFF50B1019A04446B68A118994206D88F
:10FE9000296810440C4434603A6003B0F0BD00207F
:10FEA000FBE73046F9E72DE9F743994643681746E3
:10FEB0004A1C9A4280460D4624D803685B5C03F0D6
:10FEC000C003402B1ED1FFB101AAFFF795FF0446E6
:10FED000A0B1019E09F10109B14513D30544D8F839
:10FEE000043072199A420DD8D8F8001032462944CD
:10FEF000384607F08AFF00233444BB55204603B040
:10FF0000BDE8F0830024F9E73C46F7E7F0B50029A7
:10FF100031D0172A1CD8D3B2A3F11804032C8CBFFC
:10FF20000024164C8D689CBFE41814F8184C6F1C04
:10FF30004E6804EB070CB4451DD20E6818438F6061
:10FF4000705500200130231A5D1C0BD1601CF0BDE0
:10FF5000FF2A05D9B2F5803F2CBF1A231923DBE70E
:10FF60001823D9E78E680D68DB00771C22FA03F3AB
:10FF70008F60AB55E6E70020E9E700BF12CF01082C
:10FF8000172BF8B50D4616461C4612D8DBB2A3F166
:10FF90001802032A8FBF0022144A9B1813F8182C4A
:10FFA000AB680132234413446A6893420BD30020A8
:10FFB000F8BDFF2B05D9B3F5803F34BF19231A23B1
:10FFC000E5E71823E3E722462946FFF79FFF0746A8
:10FFD0000028ECD02868AB683146184407F015FFBC
:10FFE000AA68E0192244AA60E2E700BF12CF010824
:10FFF00018B10023C0E9001283607047436873B5ED
:020000040801F1
:1000000014464A1C9A4206460D4602D9002002B008
:1000100070BD03685B5C13F0C00FF7D1002CF5D006
:1000200001AAFFF7E9FE0028F0D03268019B525D7B
:1000300012F0E00F18BFDB432360E8E70A1EABBFF6
:10004000014601460020D243B8BF2020FFF75EBF23
:1000500003685B5C03F0E001E02907D132B1A3F152
:10006000F5014B424B41137001207047002070474F
:10007000836810B544685A1CA24208D2002914BFF4
:10008000F524F424016882600120CC5410BD0020C6
:10009000FCE7F0B446684F1CB74208D805686C5CB2
:1000A00004F0E004402C02D1F0BCFFF7D7BE0020E2
:1000B000F0BC704713460A4601464020FFF760BF78
:1000C000F0B446684F1CB74208D805686C5C04F071
:1000D000E004602C02D1F0BCFFF7E5BE0020F0BCCC
:1000E0007047F0B446684F1CB74208D805686C5C8E
:1000F00004F0E004602C02D1F0BCFFF7AFBE00209A
:10010000F0BC704770B5054608460C4608F095FEF1
:10011000224603462946BDE870406020FFF730BF05
:10012000836841685A1C8A423FBF8260BF220168CF
:10013000012034BFCA54002070470368585CA0F106
:10014000BF0358425841704713B5036814465B5CBF
:1001500003F0E003A02B07D142B101AAFFF74CFE48
:10016000019B236002B010BD0020FBE71046F9E7B9
:10017000836841685A1C8A423FBF8260FF2201683F
:10018000012034BFCA540020704730B18068013864
:1001900088428CBF0020012070470120704708B5BD
:1001A0000246FFF7F2FF30B91268505CA0F1FF037E
:1001B0005842584108BD0120FCE743688B4207D9EB
:1001C00003685B5C13F0C00F0CBF01200020704778
:1001D0000020704743688B4208D90368585C00F0E0
:1001E000E000A0F14003584258417047002070479A
:1001F00043688B4208D90368585C00F0E000A0F126
:1002000060035842584170470020704743688B4252
:1002100008D90368585C00F0E000A0F1A003584240
:10022000584170470020704710B50446FFF7EEFFB5
:1002300050B163688B4208D92368585C00F01F00F6
:10024000A0F11F035842584110BD0020FCE743684D
:100250008B4208D90368585C0C30C0B201288CBFAF
:10026000002001207047002070470023C0E90133BF
:1002700003690160C3607047F8B503680446002B4A
:100280000D46164603DC3E212948F2F735F9324681
:100290000021284607F0DDFDD4E90170B8420CD0FA
:1002A0000021236801EB070C9CFBF3F203FB12C255
:1002B000904205D10020884204D14FF0FF3031E058
:1002C0000131EFE7C21992FBF3FE03FB1E2ED4F8B7
:1002D0000CC01CF80EE0BEF10A0F26D128B3013A7B
:1002E00092FBF3F103FB1122002106F1FF3E714561
:1002F0000ED2E7686368FB5C6B5467682668013759
:1003000097FBF6F306FB1377013188426760EEDA5C
:100310001CF802300D2B4FF0000304D1054405F802
:10032000013C0138F8BD2B54FCE70130C3E700BFA6
:100330007EBA010870B50446044E451814F8011B36
:100340003046FAF75BFAAC42F8D170BD1FDA01080B
:1003500070B515460022C0E901150270C0E90332EC
:10036000C0E90522C0E907224262DDE90412044621
:1003700000F11C06F2F77EFD38B929460748FAF766
:100380003DFA2B210648F2F7B7F8DDE904233146A0
:100390002046F2F75CFD204670BD00BF63A901084E
:1003A0007EBA01082DE9F04100259DF81860C0E9EA
:1003B00001120570C0E90335C0E90555C0E90755CC
:1003C000456231460446174600F11C08F2F756FB19
:1003D00038B939460748FAF711FA20210648F2F7EA
:1003E0008BF8324641462046F2F736FB2046BDE800
:1003F000F08100BF63A901087EBA0108F0B50125AC
:10040000044608270E468DB0564B574A294600959C
:1004100002A8FFF7C7FF02A92046F3F7A3FE02A830
:10042000EFF794FE514BCDE900671A460DEB07003C
:100430000421FFF78DFF0DEB07012046F3F792FE35
:100440000DEB0700EFF782FEF319494A019700937D
:100450000DEB0700474B0421FFF77AFF0DEB070177
:100460002046F3F77FFE0DEB07001027EFF76EFE37
:10047000F3190093404B01971A46042102A8FFF795
:1004800067FF02A92046F3F76DFE203602A8EFF7BA
:100490005DFE3A4B3A4A01970096042102A8FFF705
:1004A00057FF02A92046F3F75DFE02A8EFF74EFEC4
:1004B0000C23344A00930221334B02A8EFF7E2FEEB
:1004C00002A92046F3F74EFE02A8EFF73FFE2F4B9E
:1004D0002F4A2946009502A8FFF764FF02A920468B
:1004E000F3F740FE02A8EFF731FE0723294A0093F5
:1004F0000221294B02A8EFF7C5FE02A92046F3F717
:1005000031FE02A8EFF722FE1423244A00930221B1
:10051000234B02A8EFF7B6FE02A92046F3F722FE0E
:1005200002A8EFF713FE1F4B1F4A2946009502A8A9
:10053000FFF738FF02A92046F3F714FE02A8EFF7F1
:1005400005FE0A23194A00930221194B02A8EFF76E
:1005500099FE02A92046F3F705FE02A8EFF7F6FD83
:100560000DB0F0BD16CF01080FC201089FAC010805
:10057000C6D20108ADD2010830CF0108CED20108A1
:10058000F8D20108EBC1010837CF010890CF01086C
:10059000EEC10108F2C10108FFD20108FBC1010848
:1005A0003DD3010878D3010856B9010804C20108F7
:1005B00094D3010870B5044690B00146924A01A850
:1005C000F3F779FB914A214604A8F3F774FB904AAC
:1005D000214607A8F3F76FFB8E4A21460AA8F3F7D6
:1005E0006AFB8D492046F3F75DFB05468B48FAF719
:1005F00005F9DDE901239B1A082B06D08848FAF794
:10060000FDF8B1218748F1F777FFDDE904239B1A54
:10061000082B06D08448FAF7F1F8B5218148F1F7A4
:100620006BFFDDE90A239B1A102B06D07F48FAF7EF
:10063000E5F8B9217B48F1F75FFFDDE907135B1AA5
:10064000102B0CD101234A1E01F10F0012F8016F8B
:10065000002E18BF00239042F8D1002B53D07448CD
:10066000FAF7CCF85DB37348FAF7C8F8674A214641
:100670000DA8F3F720FB7048FAF7C0F8082101989D
:10068000FFF758FE6D48FAF7B9F808210D98FFF703
:1006900051FE6B48FAF7B2F810210A98FFF74AFEAC
:1006A0006848FAF7ABF80D980A9A019900F00AFF2A
:1006B0000DA8F0F721FD6448FAF7A0F861E063485F
:1006C000FAF79CF86248FAF799F80A99019800F04D
:1006D0005BFE6048FAF792F8042101980844FFF79E
:1006E00029FE5D48FAF78AF810215C48FFF722FEE0
:1006F0005B48FAF783F810215A48FFF71BFE514870
:10070000FAF77CF8D7E710220A9807F06FFB5649F2
:10071000444B002818BF19465448FAF76FF8002DCB
:1007200040D04448FAF76AF8384A21460DA8F3F752
:10073000C2FA4F48FAF762F808210198FFF7FAFD6C
:100740004C48FAF75BF808210D98FFF7F3FD4A488B
:10075000FAF754F810210798FFF7ECFD4748FAF72D
:100760004DF810210A98FFF7E5FD3648FAF746F8EC
:100770000D98079B0A9A019900F0BAFE0DA8F0F7B0
:10078000BBFC3048FAF73AF80AA8F0F7B5FC07A81E
:10079000F0F7B2FC04A8F0F7AFFC01A8F0F7ACFC4E
:1007A00010B070BD2948FAF729F83548FAF726F84D
:1007B000079A0A99019800F029FE2648FAF71EF8D0
:1007C000042101980844FFF7B5FD2E48FAF716F802
:1007D00010212248FFF7AEFD2B48FAF70FF8102141
:1007E0002A48FFF7A7FD2A48FAF708F810212948F8
:1007F000FFF7A0FD2848FAF701F81A481021FFF783
:1008000099FD104858E700BF9FAC0108C6D2010807
:10081000F8D2010830CF01080FC20108C2CF010889
:10082000D9CF01087EBA0108E9CF0108FACF010843
:100830000AD0010825D001082BD001083CD00108BE
:100840004ED001087DBA0108F6D001086ED001082B
:1008500073D00108A5D00108B7D00108E402002038
:10086000E3D0010814030020ABCF010815D1010823
:1008700032D1010844D1010857D1010877D10108CC
:10088000C2D10108FCD1010868D20108F40200209D
:100890007FD201080403002096D2010810B5084C4D
:1008A000D4F834221AB95A210648F1F725FED4F8B3
:1008B00034020023BDE8104003222021FDF75EBF73
:1008C000480100207EBA0108F0B51F461446C7B0A3
:1008D00005460E46F122002109A807F0BAFA09AA36
:1008E0001021384603F068F8204608F0A6FA0746BB
:1008F0001022002101A807F0ACFA102F3A46214639
:1009000028BF102201A807F080FA09AA05A901A8AA
:1009100003F0CCF8324605A9284607F076FA47B02E
:10092000F0BD000037B50E4C0E4D94F82F30022B61
:1009300012D194F8213094F8F3210093D4F8F411F3
:100940000823012002F0EAFF6B6B00209847042384
:1009500084F82D3003B030BDEB6A98470123F7E7E8
:100960004801002018CB0108044B5A7F22B993F8A4
:10097000330080F0010070470020704748010020DC
:10098000F0B570279DB006460D463A4600216846F0
:1009900007F05FFA08212B460DEB010004AC0B4A6F
:1009A000FFF792FF2B462046094A102108ADFFF7BA
:1009B0008BFF94E80F0085E80F003A466946304601
:1009C00007F023FA30461DB0F0BD00BF13D5010873
:1009D0001BD50108014B83F8000270474801002035
:1009E000014B83F8010270474801002008B5054813
:1009F000F9F704FF044A92F8F831013382F8F8312C
:100A000008BD00BFC5D40108480100200022024BE8
:100A100083F8F821704700BF48010020014B93F88C
:100A2000F90170474801002084B070B58AB00EAC5F
:100A300084E80F00734C4FF41072254600212046C5
:100A40000EAE07F006FA0FCE0FC596E8030014AB02
:100A500085E803000FCB04F1180585E80F000E9B15
:100A60000BB9694B23600F9B0BB9674B2360109B3D
:100A700023B940F285116548F1F73EFD129B23B979
:100A800040F289116148F1F737FD119B23B940F21B
:100A90008D115E48F1F730FD139B23B940F291119F
:100AA0005A48F1F729FDA3690BB90323A36101F0AB
:100AB00047FF94F8203013B9012384F8203001F067
:100AC00037FF94F8213013B90D2384F82130636A7D
:100AD0000BB94F4B636201F01FFFFAF7FBF9C4F843
:100AE00030020138033008D94A486368984700202B
:100AF0000AB0BDE8704004B0704700220421012014
:100B0000FCF70EFA0322C4F83C0200210120FCF796
:100B100007FAC4F8380220B94FF4DD713B48F1F709
:100B2000EBFC002204210120FCF7FAF9C4F83C0197
:100B300020B94FF4DF713548F1F7DEFC00220421C3
:100B40000120FCF7EDF9C4F8400120B940F2C111D1
:100B50002E48F1F7D1FC4FF48163A4F80032002352
:100B600084F83430012384F80432FEF7ABFE05AD7F
:100B700068B9A36822690593236807920893E2681D
:100B800063680692009395E80F00FEF7B5FEFEF746
:100B90009FFE84F8320001F013FF23681E4E079376
:100BA000636806F1A0020893236904960693E3683C
:100BB000F03605930AAB43F81C2D93E803008DE84B
:100BC000030095E80F0002F033F90196A3694FF492
:100BD000CD720093114901231148FCF76FFE0128E3
:100BE00004D04FF4F3710948F1F786FC0023032287
:100BF0000421D4F83402FDF7C1FD012084F831004E
:100C000076E700BF48010020F5A700087EBA01087A
:100C100008E6D33327D401088C0200205AD40108F7
:100C20005511010810B50F4CD4F8343223B940F2F5
:100C3000EF110D48F1F760FC002303220421D4F8E2
:100C40003402FDF79BFD42F21071D4F83802FCF734
:100C500077FB0023D4F838021A46BDE81040194645
:100C6000FCF782B9480100207EBA010838B50E4D64
:100C7000D5F8383223B94FF400710C48F1F73CFC39
:100C80000021D5F83802FCF75BFB0128044608D1A7
:100C90000023D5F838021A461946FCF765F92046B4
:100CA00038BD0020FCE700BF480100207EBA0108E3
:100CB00010B5FFF7DBFF68B1074C0023D4F834020E
:100CC00003220821FDF75AFDD4F83402BDE8104094
:100CD000FCF7A2BF10BD00BF48010020002313B5E0
:100CE00002A941F8043D4EF65E224EF66023441EF2
:100CF00094428CBF02461A46034BD3F84001FCF7DE
:100D00008DFA019802B010BD4801002008B5044BCF
:100D1000D3F84001FCF7A2FC003018BF012008BD49
:100D20004801002038B5FFF7A1FF194B20B15B68DF
:100D300018489847002038BDD3F83C01FCF78EFCDA
:100D400004460028F6D1014602F06EF90546002857
:100D5000F0D0047001F0F4FC044618B9284602F003
:100D6000B1F9E7E70C4A13680133136073B91368EC
:100D700001331360636004232046237001F004FDF7
:100D800010B9204601F0EEFC6068D4E71368F1E783
:100D90004801002062D401087418002010B500201A
:100DA00001F0CEFC01230370044601F0EDFC40B9D4
:100DB000204601F0D7FCBDE81040024B02485B68BA
:100DC000184710BD480100208ED40108F0B58BB043
:100DD00005460C4617460193FFF748FF10B1002067
:100DE0000BB0F0BD4B4ED6F83C01FCF737FC0028A9
:100DF000F5D1002F5CD1002CF1D12846214602F01C
:100E000013F905460028EAD09DF80530002B52D092
:100E100004230370FFF7EAFD0F2206A903A809F0D7
:100E200055FC9DF804303BB10D230AA901F8203D83
:100E3000012203A809F058FC9DF806303BB10223BB
:100E40000AA901F8203D012203A809F04DFC96F8FB
:100E50002E2096F82F30934203D196F830309342EB
:100E600017D02023022A18BF00228DF8083095F8E9
:100E7000783002A90BBF43F0040343F001038DF85F
:100E800009208DF8092003A885F87830022209F09E
:100E90002BFC96F81432059996F8F0011944C9B262
:100EA00001F014FF844209D9284602F00BF996E7B5
:100EB000E02F94D8A1E702230370ADE7059A32B181
:100EC000D2B20399284600F0CDFF0028ECD06F770E
:100ED000284601F035FC07460028E5D000230E4ADD
:100EE000836013680133136083B91368013313609F
:100EF0007B60022338463B7001F046FC40B938461F
:100F000001F030FC73680548984768E71368EFE71D
:100F1000786865E74801002074180020F9D40108BA
:100F200013B51C460023ADF804308DF806308DF85B
:100F30000520019B2246FFF749FF02B010BD0000CB
:100F4000034B93F8141293F8F00101F0BFBE00BFF9
:100F5000480100200E2808BF0120024BD87783F8F3
:100F6000F001704748010020024B83F8200083F80D
:100F7000F101704748010020014B83F821007047C0
:100F80004801002008B5F9F725FD024BC3F84801D8
:100F900008BD00BF48010020034630B5054C00F1F4
:100FA0001005224618685968083303C2AB4214463C
:100FB000F7D130BD04030020034630B5054C00F1E5
:100FC0001005224618685968083303C2AB4214461C
:100FD000F7D130BDF4020020034630B5054C00F1D6
:100FE0001005224618685968083303C2AB421446FC
:100FF000F7D130BDE4020020034630B5054C00F1C6
:101000001005224618685968083303C2AB421446DB
:10101000F7D130BD1403002010B50446FFF7BCFF24
:101020002046FFF7C9FF2046BDE81040FFF7D4BFB8
:1010300030B51025C3B0224CF122002105A806F0DE
:1010400008FF2A46002101A806F003FF94F85B314F
:1010500005AA8DF8053094F85A3129468DF80630E6
:1010600094F8593104F5B6708DF8073094F858317A
:101070008DF8083094F857318DF8093094F85631CE
:101080008DF80A3094F855318DF80B3094F85431BE
:101090008DF80C3002F090FC052305AA04F5C6710A
:1010A00001A88DF8043002F001FD062305AA04F51D
:1010B000BE7101A88DF8043002F0F8FC43B030BDD9
:1010C000480100200246024B0068516803C3704784
:1010D000940200200246024B0068516803C3704727
:1010E0009C020020034630B5054C00F11005224655
:1010F00018685968083303C2AB421446F7D130BDB3
:10110000A4020020034630B5054C00F1100522462C
:1011100018685968083303C2AB421446F7D130BD92
:10112000B4020020014B9877704700BF48010020AF
:10113000014B83F82E0070474801002038B5044663
:1011400000680D46884203D008B101F00BFB256012
:1011500038BD00002DE9F041F9F7B6FC0123764CCB
:10116000DFF8DC81754E84F82D300A23744A4FF085
:10117000FF310020FDF7B8FA012866D1D8F8000049
:1011800043071AD5337833B1F9F704FE0020F9F795
:1011900055FE00233370FBF7A5FCFBF7C3FC0223CD
:1011A00084F82D300023D4F838021A461946FBF78C
:1011B000DBFE0020FCF79AFFD7E710F0080721D0EC
:1011C00033787BB941F28830F9F710FE18B99B21CA
:1011D0005C48F1F791F95C48F9F730FE0123337070
:1011E000FFF7A0FB0020FDF7C3FB4FF4FA61D4F832
:1011F0003802FCF7A5F80028B7D1A2215148F1F731
:101200007BF9B2E710F020003FD03378D3B194F8E7
:101210002D30042B16D14D4D3A462946D4F83002D4
:10122000FCF73EF901280DD12B78072B2AD03A463E
:101230002946D4F83002FBF7F1FF012802D12846F5
:10124000F9F702FE0020FDF793FB3378002B8CD0DA
:1012500001F0AEFA0546002887D00378012B1AD199
:1012600094F82C10A26A01B192B9B2FA82F238480D
:101270005209F9F7C3FA284601F0FCFA284601F0B2
:1012800071FA72E701F024FADCE7FDF771FB6CE715
:1012900001F068FAA56A032384F82D302B78052B1A
:1012A00046D8DFE803F003450A0A3A3AD521254833
:1012B000F1F722F9FFF736FB57E729462548FFF7F4
:1012C0003DFFFFF751FB68B101F084FA054618B9FC
:1012D000E1211C48F1F710F9022328462B7001F098
:1012E000A3FAE7E701F076FA074618B9E8211548AE
:1012F000F1F702F93946284600F028F97B7E53B110
:101300004FF47A70FCF774FE3946284600F01EF957
:101310007B68002BF2D03846E1E70E480021FFF74A
:101320000DFF284600F03AFE284601F01BFAC1E7FF
:10133000636809489847F7E74801002078180020BB
:10134000881800207EBA01089D0801087C1800203A
:10135000C3D301087001002003D4010813B5002491
:10136000074802AB90F8F11143F8044D054A90F894
:101370003200FEF767F82146019802B010BD00BFA9
:10138000480100202515010830B50430C7B00D46CE
:10139000FFF7F8FD1B4B0DF1050203F10C0153F8AB
:1013A000040B8B4242F8040BF9D11B8801241380F3
:1013B00000238DF81330022309AA102128468DF846
:1013C000043002F0F9FA09AA05A901A802F06EFB9F
:1013D00005A8FFF711FE09AA102128468DF8044040
:1013E00002F0EAFA09AA05A901A802F05FFB05A824
:1013F000FFF712FE1022044B5C771A7783F8442122
:1014000047B030BDB6D401084801002030B50430E3
:10141000C7B00C461546FFF7B5FD284B0DF1050288
:1014200003F10C0153F8040B8B4242F8040BF9D181
:101430001B882046138000238DF8133002230124DB
:1014400009AA10218DF8043002F0B6FA09AA05A9FC
:1014500001A802F02BFB05A8FFF7CEFD09AA102179
:1014600028468DF8044002F0A7FA09AA05A901A8A8
:1014700002F01CFB05A8FFF78FFD032309AA05A9AD
:1014800001A88DF8043002F011FB05A8FFF794FDC8
:10149000042309AA0DEB030005A98DF8043002F01E
:1014A00005FB05A8FFF798FD1122054B5C771A771D
:1014B00083F8442183F8FD4147B030BDB6D401081C
:1014C0004801002038B50D461446FFF7FBFD2846BD
:1014D000FFF700FE2046FFF705FE2046FFF712FE4D
:1014E0000022024B5A7710221A7738BD480100209B
:1014F00070B50E4615461C46FFF7E4FD3046FFF773
:10150000E9FD2846FFF7EEFD2046FFF7FBFDBDE8AD
:1015100070400022024B5A7711221A77FFF788BDDC
:1015200048010020002310B54168074C1A19106CBF
:10153000884202D192F83C0020B91033B3F5807F85
:10154000F4D1002010BD00BF480100202DE9F04F6C
:10155000064689B00C4619B918216C48F0F7CCFF43
:1015600016B13378022B03D01A216848F0F7C4FF74
:1015700033691BB91B216548F0F7BEFF33691B783F
:10158000042B05D0022B03D01D216048F0F7B4FFD7
:1015900000225F4D337895F8F1716370D5F8F4311E
:1015A0003946039308AB43F80C2D95F83200594A9D
:1015B00095F8F0B195F8F2A195F8F391FDF742FF97
:1015C000804620B90123237009B0BDE8F08F059B48
:1015D00033B101F0FDFB03232370059B6360F3E748
:1015E000B3680133012BB36011D1D5F8E421306920
:1015F0000132C5F8E421B5F8FE2185F82C3001321E
:10160000A5F8FE2100F0DEF8306900F04BFCD5F8BB
:10161000482133695A60D5F8E4215A8195F8F921B7
:1016200042B1002285F8F9211A7A42F004021A72B6
:10163000B5F8FA21A3F87A20404601F0E7F903460D
:1016400095F8F02105EB001130694FF0000880F8A3
:101650007D3080F87C2095F804224FF47A7312F0E4
:101660000F0208BF01225A4307AB019306AB009358
:101670003C3102F57A73CDF8188000F0F9FE0028AD
:10168000A0D0FCF75DFBF060D4F8A00084F80080E7
:1016900008B101F017FD069B0798C4F8A030C4F804
:1016A0000A00224631461C4800F05EF8802231696B
:1016B00004F1200006F0A9FB0021039B0798636159
:1016C00095F83330C4F80A00C4F8881084F810B0D4
:1016D000677484F812A084F8139021702376B2689E
:1016E00095F80232D4F8A0009A4200D258B161763F
:1016F00085F82C10003018BF0120617E009007484B
:10170000F9F77CF860E701216176F3E77EBA01081A
:1017100048010020251501087001002022D501088C
:1017200008B5104A10B10023A2F8FE31937FBBB177
:10173000B2F8FE3192F800128B4211D95B1A92F87E
:10174000011293FBF1F201FB12334BB901F000F9E6
:1017500030B901F00BF918B9BDE8084001F016B92D
:1017600008BD00BF4801002070B5D2F8A040064671
:101770001546E4B10021204601F08AFBFFF746F947
:1017800023782046052B01BF012386F8D1316389D8
:10179000A6F8D231FFF7C4FFD5F80A10204600F0B2
:1017A000B7FB237A5B0701D501232B7270BD20465E
:1017B000FFF7B6FFD5F80A102046BDE8704000F0EC
:1017C000A7BB0000134B10B49A7F02B3027A93F8C0
:1017D000F01142F001020272DA7F914208D193F8CF
:1017E0003C40A4B193F84C408CB193F85C4074B188
:1017F000B3F8FE4193F800329C4208D9914206D0DA
:10180000037A10BC43F002030372FFF7EFB810BC79
:10181000704700BF48010020431EDBB21F2B96BF5C
:101820000D4A0023D35C0A280BD8012202FA00F0EB
:1018300010F4A46F05D0094A92F814221A440E2A13
:1018400007DC074A107818440E28CCBF002001207E
:1018500070470020704700BF5FD501084801002095
:101860009B18002070B5057804462846FFF7D4FF82
:1018700088B1094A094E1378F5540133137051B1F8
:10188000074A247892F81432D01880F805420846A6
:10189000013382F8143270BD9B1800208C18002090
:1018A00048010020000000002DE9F04F002593B012
:1018B000CDE907019DF87080B74E09920593454523
:1018C0000AD2059B595D5F190846FFF7A5FF0290F4
:1018D00028B9B248F8F792FF13B0BDE8F08F01398C
:1018E0001F2900F2A682DFE811F02000A4022C00DC
:1018F00054027D016101C40142025402EB01A402C1
:1019000056022C016D026F02A402A402A402A402DA
:10191000A402A402A402A402A402A402A402A40297
:10192000A402A402A402A4029102A8EB0503DBB264
:10193000012B4FF0000400F0028186F8FD410224E3
:10194000FDE0A8EB0503DBB2039307238DF83830E5
:1019500000231C460193039A231D934202DA3B5D48
:10196000032B10D0019B2BB19DF838306FF300038F
:101970008DF838309DF83830072B40F0D2800024A5
:10198000DFF81C92C6E03B19D3F8012005345FFA5A
:1019900082FB0BF00F034FEA1B1B0693BBF1060FF4
:1019A000C2F30F23E4B24FF000090F92049303D95E
:1019B00002F0F003F02B2FD14FF6FF73C2F3076252
:1019C000049902F07002602A08BF194600230A46F3
:1019D0009A4611465FFA8AF00B930A9201F088F852
:1019E000DDE90A2380B106EB0A11096C61B106EB4F
:1019F0000A1191F844104FEA111C01F00F015945EA
:101A000002D8E34598BF03460AF1010ABAF1100F64
:101A1000DFD10BB14FF00209069B072B05D99DF8CA
:101A20003C3003F00F030F2B01D149F004099DF85E
:101A30003FA00AF0700ABAF1600F0CD149F0010919
:101A4000BAF1000F0FD0DDE90132BAF1600F18BF13
:101A50001346019307E0BAF1000FF4D1049801F0A6
:101A600025F80028EAD19DF83830C9F3400269F31F
:101A7000000362F34103C9F3800969F382038DF81F
:101A8000383068E73B19D3F801A09DF838300534A9
:101A900003F00703072BCDF840A0E4B23AD19DF83C
:101AA0004030C3F30311CAB286F8F0110AF00F01F7
:101AB0000F290BD021B9012161F303038DF84030C8
:101AC0009DF84030C3F3030386F8F1319DF84310CD
:101AD000CAF30F20C1F3021101F010F820B940F24F
:101AE00075114846F0F708FD96F84431102B09D1DE
:101AF0001AF0706F01BF01229DF8433062F30303B7
:101B00008DF843309DF843301A0703D0C3F3030325
:101B100086F80232039A231D9A4202DD3B5D032BB5
:101B2000B0D054B1032312A8002100F8083DFFF7FC
:101B300099FE00210EA8FFF795FE01F049F92C440B
:101B40004AE0A8EB0503DBB2052B40F27081781C5C
:101B5000F8F747FF97F905300021002B22DB0CA393
:101B6000D3E9002312184B41002196F8040210EB30
:101B7000020941EB030A099B022B03D119F1010968
:101B80004AF1000A079BC3E91C9A0624D7E700BF65
:101B90006E3DD51200000000480100207FD50108ED
:101BA0007EBA0108A8A3D3E90023DBE7062312A825
:101BB00000F8103D0021FFF755FE089B12AC03F022
:101BC0001F0304F8083D00219B48FFF74BFE204609
:101BD0000021FFF747FE6C1CE4B2A5423FF47CAE47
:101BE00025466CE6A8EB0503DBB2042B4FF000049E
:101BF000A5D9D7F801308DF834401093DBB2C3F388
